:020000040000FA
:0400000A9901C0DEBA
:1000000000400020218E01005D8E01005F8E010006
:1000100000000000000000000000000000000000E0
:10002000000000000000000000000000618E0100E0
:100030000000000000000000638E0100658E0100DA
:10004000678E01005D3D000065950100678E01002F
:10005000678E010000000000218F0100678E010003
:1000600069E80000D59A0100D9930100678E01006C
:10007000678E0100678E0100678E0100678E0100A8
:10008000678E0100678E0100678E0100678E010098
:10009000678E01000D8A0100D98A0100A5E90000E0
:1000A000B5E90000678E01000000000000000000BC
:1000B0000000000000000000000000000000000040
:1000C00010B5064C2378002B07D1054B002B02D02E
:1000D000044800E000BF0123237010BD2001002070
:1000E0000000000098870300044B10B5002B03D0DC
:1000F0000349044800E000BF10BDC04600000000F6
:100100002401002098870300164B002B00D1144BCC
:100110009D46402292029A1A924600218B460F4633
:100120001348144A121A28F050FE0F4B002B00D02F
:1001300098470E4B002B00D0984700200021040068
:100140000D000D48002802D00C4800E000BF20F050
:10015000E3FB2000290028F08EFB20F029FBC0469D
:100160000000080000400020000000000000000027
:1001700018010020E02F0020000000000000000017
:1001800010B54A68014926F045FE10BDC43B030086
:1001900010B50400080021F08CF90300002C03D0F6
:1001A000012C06D0002003E00348002B00DC0348AC
:1001B00010BD40002043FBE7CCE70200C4E702008B
:1001C00043684B6083688B60C3680800CB60014B59
:1001D0000B607047A890020030B5040087B00D0096
:1001E0000020042A25D1200021F063F9AB0722D199
:1001F000184B2A689A421ED103AA290011F034FB39
:10020000102026F056F8144BE2680360039B6168E7
:1002100053435B184360049B6168019353435B182D
:10022000059983604A43C260002902DAE2689B1A9A
:10023000836007B030BD002301002A00206802F06F
:10024000F5FCE36858436368C01801234000184375
:10025000EFE7C046E8A402006C900200F0B50E0083
:10026000002785B0110003901D00012203233000F8
:10027000009712F021F8102026F01BF8039B0400D1
:10028000036001234760C36028689E4205D102F0E5
:10029000F5FBA060200005B0F0BD02F0EFFB606050
:1002A000686802F0EBFBA060032EF3D1A86802F0AF
:1002B000E5FBE0600028EDD101480DF087F8C0466D
:1002C000D6FB020070B50D004A688B68084904002F
:1002D00026F0A0FDEA68012A04D10649200026F094
:1002E000D8FC70BD0449200026F094FDF9E7C04613
:1002F000E0FB0200A0020300EDFB0200136810B552
:100300001400002B05D1A42904D1406825F0D8F9A8
:10031000206010BDB9235B00994201D18068F5E7E8
:10032000024B9942F5D1C068F0E7C046BF02000019
:100330000023820708D10068044A0133904203D0A9
:10034000034BC01A434243411800704720910200FA
:10035000E4900200044B88600B60044B08004B6083
:100360000023CB607047C0466C98020097150200CE
:1003700030B585B00500080069460CF0F7FB0400B5
:1003800020000CF055FC011E02D1064805B030BD1E
:100390002B1D0022180023F085F80028F0D0024819
:1003A000F4E7C046CCE70200C4E7020070B50500E0
:1003B000102025F07EFF0400074B696808C023F079
:1003C00067F8AB68E968A3606B68E0689A0028F09A
:1003D000E0FC200070BDC04620910200F7B504008B
:1003E0000D0000268B0704D10B68214E9E1B734223
:1003F0005E41AB68002B0AD1002E03D01D492000BE
:1004000026F047FC1C49200026F043FCF7BD002ED7
:1004100003D01A49200026F03CFC1949200026F0A0
:1004200038FC002701236A68BA4207D81549200022
:1004300026F02FFC002EE9D01349E4E7BA00019220
:10044000EA68B9005258002A0FD0042A0DD0002BB8
:1004500003D10E49200026F01CFCEB68B900595866
:100460000122200002F03AFA00230137DBE7C04600
:10047000E49002002BFC020032FC020038FC020077
:1004800043FC02005E070300A002030045FC0200DB
:1004900010B5830707D1044B02689A4203D1034980
:1004A000034824F0C7FA10BDE4900200F3FB0200F9
:1004B000E0A7020070B50D000400FFF7E9FF290076
:1004C000201D012222F0EEFF004870BDE4B30200BF
:1004D00070B50D000400FFF7DBFF2900201D02228C
:1004E00022F0E0FF004870BDE4B3020070B50600E2
:1004F00008680D000124FFF7CBFFB44201D3044884
:1005000070BDA300E958286820F0E3FF0134F4E748
:10051000E4B3020070B50D000400FFF7B9FF280036
:1005200000210CF023FB050028000CF081FB011ECC
:1005300001D1044870BD231D0322180022F0B2FF30
:10054000F2E7C046E4B3020010B50400FFF7A0FFD5
:10055000201D23F035F8014810BDC046E4B3020069
:1005600010B5012220F0E6FF004810BDE4B3020000
:1005700070B504000D00FFF78BFF201D022229003B
:1005800022F090FF002804D1034822F03EFE0CF038
:10059000A5F8024870BDC046C0A90200E4B302003D
:1005A00010B50400FFF774FF201D22F0EAFF0028B9
:1005B00003D10249024824F03DFA10BD15FC0200A7
:1005C000C0A90200F8B50D0001280BD0002803D007
:1005D00002280BD0002004E08B681448002B00D1C7
:1005E0001348F8BD8B685B001843FAE7032400202A
:1005F0000C408442F5D10F4B0E6820009E42F0D192
:100600004F68A74203D1012076003043E9E7EA684A
:10061000A3009958002906D0042904D002200CF028
:100620003DF9401036180134EBE7C046CCE7020034
:10063000C4E70200E4900200F8B5040010200D00A9
:1006400025F037FE0600094B210008C607003000E0
:1006500022F01EFFA4002C19A54201D13800F8BDDC
:10066000012202CD300022F01DFFF5E720910200AB
:10067000F7B504000E00171E2CD0FFF709FF194D27
:10068000B4422DD000210800FFF7D6FF002105005D
:1006900030000CF06BFA019001980CF0C9FA061EBC
:1006A0000CD1002F1CD0E06825F032FE6B6863602F
:1006B000AB68A360EB680B4DE36011E0201D0022E6
:1006C000310022F0EFFE0028E6D031002800FFF7CD
:1006D000F1FEE1E78842D5D1200020F00DFF0500B2
:1006E0002800FEBDE4B30200F0B589B00400039019
:1006F000029101920027FFF71BFEB84207D13A0092
:1007000003AB0121224820F06BFF04000137029D5A
:1007100000262800FFF70CFEB04207D1320002ABE2
:1007200001211B4820F05CFF05000136019B002BD6
:1007300005D00023AA680193A36893420DD0154BFE
:1007400006940493144B05930023079304A820F008
:1007500022FF011E12D101230193002F02D020009D
:10076000FFF7F2FE002E02D02800FFF7EDFE019BFE
:100770000A48002B00D10A4809B0F0BD2B1D002209
:10078000180022F08FFE0028E0D10190E5E7C04676
:10079000209102006C98020097150200CCE702003D
:1007A000C4E7020073B50C00150000910192002609
:1007B0008B0704D10B68394E9E1B73425E41320099
:1007C0001F2868D819F0A0FA2810176767671C67F8
:1007D0006767676767212D346767673B6767676788
:1007E0006740464A5358675D2900200020F095FE77
:1007F0000400200076BD2900200020F0E6FEF7E787
:100800006946022020F0C2FEF2E7002E04D06946BD
:100810000220FFF76BFEECE72900200020F073FEBA
:10082000E6E729002000002EE0D0FFF773FEE0E7A6
:1008300029002000FFF71CFF002EDAD1D8E7694617
:10084000022020F077FED3E7012229002000FFF7E5
:100850004BFFCDE7012221002800F8E72800FFF731
:1008600067FD002815D0A368AA68934211D129001A
:10087000200020F0E6FEBBE72900200020F0D9FE92
:10088000B6E7201D0022290022F00CFE044C0028AF
:10089000AFD1044CADE70024ABE7C0462091020085
:1008A000CCE70200C4E70200F0B50F00496885B04C
:1008B00005001600002901D0002A05D139002800C2
:1008C00020F0D0FF05B0F0BD0F321309C918009316
:1008D00020F039FF0F22A868B9687C68324000D147
:1008E0001032009B1E19234BF3185B00C018214BDC
:1008F0000290E3185B00CB18019010209C46210069
:100900000023801A002921D1C3401A48029A844644
:100910006400141B2380009B5B00E41A009B0234DC
:1009200063445A00200028F050FA002E04D07300CF
:10093000023BE35A002B1BD001216E603B78DB07A2
:10094000DA0F2B788B4313432B70BBE76246128878
:10095000013913431A00C2400393019B1A80019A84
:10096000039B023A0192022252421B049444C9E7BB
:10097000013EDAE7FFFFFF7FF0B54B6815005268D4
:1009800089B006000C00934201D22C000D00012119
:10099000227863680A4201D12A781140C9183000D0
:1009A00020F0D1FEB36822780193A3681700029368
:1009B000636829789C46AB684F4003930123180075
:1009C0001F408B4306936346904302006046591EC6
:1009D000019B04936B681B1A07934B1C18D1634649
:1009E0005900019B5918002F02D001230B800231BE
:1009F000019820F02BFE0121706022782B78534063
:100A00003278DB078A43DB0F1343337009B0F0BD44
:100A1000029B13481B881B189B180593079B5B18A8
:100A20008B421AD8039B039A1B8802321B1803922D
:100A3000069A01399B18059A5A4092B21B0CD71995
:100A40000693049A059B17801A0C049B3F0C0233F3
:100A50000493029B02330293BFE7014BE8E7C046D1
:100A6000FFFF0000F0B5060095B0069353680D0037
:100A7000591C0492009320F066FE049B00215B68E1
:100A8000B0685A1C5200009328F09FF9002373604D
:100A9000049B28005B68591C009320F054FE0499C5
:100AA000280020F0DFFEAB686F680193069B9B680F
:100AB0000393069B5B680293B3680793029BBB4258
:100AC0002DD82ED3039A3900019820F07FFE0028FC
:100AD00023D10123079A686013807360049B1A78FE
:100AE000069B1B785A4001231A4214D032781343D4
:100AF00033706B68002B0ED0012111A8494220F001
:100B0000D0FE11AA3100300021F0D2F8069A290057
:100B1000280021F0CDF815B0F0BD002801DA00233F
:100B2000DBE7824A029B9B185B009C460022039BEA
:100B3000634405931B8800921AB2002A63DA0022EC
:100B4000019B7C001A537B1C102709936B60019B4F
:100B5000A01C00991B180893791A019B0A91089907
:100B60008B4256D3059B009A1B8893400893029BA7
:100B7000012B0AD91022039B00996344023B1B8876
:100B8000521AD340089A1A430892019B029A1C19E0
:100B9000099B9B1A654A73609B18079A5B00D318E0
:100BA0000A93634602330E936B680B930B9A029B76
:100BB000934239D313005D4A102194460024019AD0
:100BC00063445B00D318009A891A019A9A4200D8AC
:100BD0009EE07368002B07D0544A07999A18520078
:100BE000525A002A00D19DE06B68002B00D175E7B6
:100BF0004E4A01999A185200525A002A00D06DE7C5
:100C0000013B6B60F0E7009A5B0001329BB292B24D
:100C100091E71988009F0800B84002431A800A9A99
:100C20000233D1408AB29AE7A31E20880D931B8815
:100C300000041843089919F07BF80E9B0022E31A70
:100C40000C931900039B05909C4609928C4212D884
:100C500023889A4234D3D31A5A42190C9BB2228069
:100C60005A1E9341CA18002A2CD003990C9B8C461B
:100C700000210F0041E0099B009F180C63461B8870
:100C8000BB4018436B4609909F8C059B5F430B88C4
:100C90009F4203D2D81B0F9090420CD8D31AFF1852
:100CA0007B420B80BBB23A0C5F1EBB41D2180223C1
:100CB00002319C44CAE70F9B9A1A0A800022F6E789
:100CC0009A1A22800A9B059A023B5A800A930B9B30
:100CD0000D9C013B6B6067E7380C09906046009FF4
:100CE0000088B840099F074318884118B8B24118D6
:100CF000022019808444090C02339C42ECD82388DA
:100D00005918059B2180013B090C521A0593AAE74B
:100D10001A88009F100038418A402043188094B2FE
:100D2000023B52E7013B736053E7C046FFFFFF7F82
:100D3000436870B55A00002384680A4DA218944293
:100D400006D30278D20700D55B4201200B6070BD4C
:100D5000023AAB4203D816881B043343EFE7002066
:100D6000F5E7C046FF7F0000032230B502400121B5
:100D7000002A04D1084C05680B00A54209D00B00DD
:100D8000034006D1002A04D1036804481B1A5842C4
:100D90004341180030BDC046D4E702002CB9020020
:100DA00010B50400FFF7E0FF012200280AD1032359
:100DB00002002340022B05D103480440063C2200D8
:100DC000541EA241100010BD070080FF044B886034
:100DD0000B60044B08004B600023CB607047C0469B
:100DE0006C980200F125020010B501F05FFD084B80
:100DF00042680848D31859424B41AC215B428B43AF
:100E0000B02189005B18044907F04CFB0BF066FC2D
:100E100040FDFFFF90AC020048FC0200F7B5040063
:100E20000E00019301208B180A0000210093009B03
:100E3000934212D82725002900D0053D224F2A00D1
:100E40003900200025F0E6FF009B9E4214D32A00C3
:100E50003900200025F0DEFFF7BD1378272B08D0DE
:100E6000223B5D426B41DBB20132002BDFD02725F4
:100E7000E4E700230100F7E73278AA4205D12A000F
:100E80001249200025F0C6FF1AE011495C2A14D04F
:100E90001F2A09D97F2A15D0019B002B02D053B2FB
:100EA000002B07DB3900ECE70A490A2A05D00A497A
:100EB0000D2A02D0092A05D10849200025F0E9FEB3
:100EC0000136C1E70649DCE7820003008100030028
:100ED00085000300880003008B0003008E000300E0
:100EE00091000300194B70B506000C0098420FD119
:100EF0004968A0680FF0AEFD051E09D0200026F05D
:100F000024F90023ED00236006331D43280070BD43
:100F1000102025F0CEF96168050081600660A068A8
:100F20000FF07AFD63686860591C2368994208D104
:100F3000A368EB600023EA68A9685354A3602360A8
:100F4000E4E7A06825F0D3F9E860F3E70C9A020023
:100F500070B504000D00002A05D00FF0ADFDC300F0
:100F60000620184370BD0FF075FD0028F7D12A0048
:100F70002100024821F014FAF4E7C0460C9A02005E
:100F800010B50A000100024821F00AFA10BDC0465F
:100F9000A0920200094B10B50340062B01D1C008F6
:100FA00010BD830708D1064B02689A4204D18168BC
:100FB000C0680FF081FDF3E7FFF716FF070080FF21
:100FC0000C9A0200064B10B50340062B03D1C00853
:100FD00024F0D5FC10BD8368C0680B60FAE7C046FA
:100FE000070080FFF0B50F00002589B01100060052
:100FF0001C003800009503232A0011F05DF90E2033
:10100000AF420FD0012F0FD102AA102104A814F073
:10101000F7FE216802A82A0001F060FC04A9300054
:10102000FFF760FF09B0F0BD2068830722D1164B9F
:1010300002689A421ED104A9FFF7C4FF134B0500B2
:1010400020680340062B13D1C00824F089FC04005B
:10105000002C04D1049928000FF0DEFC04001020BD
:10106000049F25F026F906608760C5604460D9E7D3
:101070004468EDE704A9012201F0BAFE00220599B7
:101080000498FFF765FFCDE7A0920200070080FFFC
:10109000F0B58DB00400039101F008FC04A906002E
:1010A0002000FFF78FFF039B01902F489A0705D17F
:1010B0001B6883420AD02D4A934207D0C36800229E
:1010C0000293012103AB029CA0470390002406AACF
:1010D00005A9039801F074FD2500059BA3420ED8D5
:1010E0002900002508A826F01FF80A9C059BAB42A2
:1010F00021D808A93000FFF7F5FE0DB0F0BD069B22
:10110000A700D85901F0D2FBB04202D018480CF029
:1011100021FB002C01D0049BED18069BD859154BE0
:101120000340062B05D1C00824F01FFC2D18013404
:10113000D3E78068FAE7002D06D02000049A0199D1
:1011400027F027FE049BE418069AAB00985807A9DD
:10115000FFF738FF079A0100200027F01AFE079BCF
:101160000135E418C2E7C04688E702004CA002003F
:10117000BE000300070080FFF0B58BB00490086844
:101180000D000692079301F091FB0400686801F0DE
:101190008DFB0600A04202D06868FFF725FE08A973
:1011A0002868FFF70FFF040009A96868FFF70AFF26
:1011B000089A0590A3180393049B2700022B19D9C2
:1011C000AB681D498B4206D00121300000912100FF
:1011D00004F04AF80700049B032B0BD0EB68164A77
:1011E000934207D00122210000923000089A04F0B7
:1011F0003BF80390039B059AD91B069B380000938C
:10120000099B21F0AEF8002806D1079B0138002B7E
:101210000CD00A480CF0DAF8094B9E4208D10100C4
:10122000200022F054F84400012020430BB0F0BD10
:10123000041B6400F8E7C046E4B30200AA00030000
:101240000C9A0200F0B5070087B008680D0001F0A5
:101250002DFB04A906002868FFF7B4FE05A90400C9
:101260006868FFF7AFFE03902000022F07D9012323
:101270000093AB68049A2100300003F0F5FF059A53
:10128000041B049BA418064D9C4205D8039927F023
:1012900071FD002800D1034D280007B0F0BDC04605
:1012A000C4E70200CCE7020073B50D0006006946F2
:1012B0002868FFF787FE01A904006868FFF782FE2F
:1012C0000100022E02D908480CF072FA019A009827
:1012D000064D824206D8801A201827F04BFD0028C0
:1012E00000D1034D280076BD98000300C4E702003A
:1012F000CCE70200F0B58FB0079010680C00160024
:1013000001F0D4FA0690012C31D0706801F0CEFAC9
:10131000069B984202D07068FFF766FD0DA97068C1
:10132000FFF750FE0D9B089009930DA93068FFF759
:1013300049FE0D9B0B900493079B012B1CD1049B32
:101340005D1E01235B420A9300242700049B039443
:101350000593059B002B13D1039B002B23D1214B1D
:10136000069A0E209A4200D01F480FB0F0BD072306
:1013700009931E4B0893D8E7012300250A93E3E75E
:101380000B9B09995A1901230898009320F0E9FF53
:10139000002816D1039B002B19D1079B002B09D1E4
:1013A0002F00049B5C1E049B0134E21B934212D16C
:1013B0003068DAE7079B2C00012B0AD001232F00AD
:1013C00003930A9BED18059B013B0593C1E72C0095
:1013D000F7E7039FE7E70B9B0698D91920F0E0FF9A
:1013E000C3E7C0460C9A0200909202001701030066
:1013F000F0B589B0049008680D0001F057FA0400B8
:10140000686801F053FA0700A04202D06868FFF74D
:10141000EBFC06A92868FFF7D5FD060007A9686858
:10142000FFF7D0FD069A0590B3180393049B340090
:10143000022B19D9AB681E498B4206D00121380016
:101440000091310003F010FF0400049B032B0BD02C
:10145000EB68174A934207D001223100009238000E
:10146000069A03F001FF03900025079BAB4212D1BF
:10147000039B2000191B21F039FF0130450001209A
:10148000284309B0F0BD0599200027F073FC00281F
:1014900008D101353400079A039BA6189E42F2D961
:1014A0006D00ECE7200021F009FF0600F2E7C046DE
:1014B000E4B3020010B50100014821F063F810BD4B
:1014C0000D33020010B50100014821F05BF810BD9A
:1014D0001F330200F7B50600080001A9FFF772FDEF
:1014E000019B0500002B01D11348FEBD134B0400E6
:1014F0009E4207D10027019A631B9A4211D8002F00
:1015000007D1F1E70E4B9E42F4D0019A631B9A4239
:1015100001D80C48E9E72078B04701340028F4D11D
:10152000E2E7207807F098F8002803D02078B04749
:10153000071ED9D00134DEE7C4E70200C1860000EF
:10154000D9860000CCE7020010B501000148FFF782
:10155000C1FF10BD4186000010B501000148FFF732
:10156000B9FF10BD5986000010B501000148FFF712
:10157000B1FF10BD7186000010B501000148FFF7F2
:10158000A9FF10BDC186000010B501000148FFF79A
:10159000A1FF10BDD9860000F0B585B006000C0093
:1015A000170001F083F9694605003000FFF70AFDD6
:1015B0000600042F23D10098A30715D1114B2268F0
:1015C0009A4211D101AA210010F04EF9002802D14F
:1015D0000D480CF0EDF80199029A2800521A711882
:1015E00020F0DEFE05B0F0BD00230100220028003F
:1015F00001F01CFB335C01205B001843F2E7002084
:10160000F0E7C046E8A40200A6FC020070B51D0089
:101610008EB0002900D174E018683B4C03002340D1
:10162000062B05D0830726D1384B02689A4222D177
:101630000239012962D80AA9FFF7C4FC060028680C
:101640000440062C15D1C00824F08AF90400002CAF
:1016500004D10A9930000FF0DFF9040010200A9D30
:1016600024F027FE2A4B85600360C66044600EB0FC
:1016700070BD4468EBE7012940D80122104210D028
:10168000441021000AA825F04FFD0C9B00212200E8
:101690001800019327F099FB0AA91D48FFF722FCC7
:1016A000E5E703A920F0DAFF002805D0049A0399A2
:1016B000174820F075FEDAE7286801F0F9FA1021E2
:1016C000002800D0411006A825F01DFD0AA92868B1
:1016D0000BF04CFA040020000BF0AAFA002801D10C
:1016E00006A9DAE701F0CAF9FF2802D909480BF088
:1016F0006DFEC1B206A825F066FDECE706480CF0C9
:1017000029F80648B3E7C046070080FF0C9A02009C
:10171000A092020073FC02008CFC02009092020076
:1017200073B50400080001A91600FFF74BFC050083
:10173000042E06D10300019A0749200025F06AFB18
:1017400073BD0649200025F0A4FA0123019A29005F
:101750002000FFF763FBF3E703010300CF59030009
:101760000A001B4B73B51A4005000C000340062B02
:101770000CD1062A04D1441A60426041C0B212E082
:10178000C00824F0EDF80600606805E04668062A07
:10179000FAD1C80824F0E4F8002E05D0002803D0C0
:1017A000B04201D0002076BD69462800FFF70AFC50
:1017B00001A905002000FFF705FC009A019B01002C
:1017C0009A42EFD1280027F0D5FA44426041D5E78C
:1017D000070080FF084B07B50340062B08D083079E
:1017E00004D10268054B92699A4201D0FFF7FCFAD6
:1017F00001A9FFF7E7FB0EBD070080FF9D1D00005C
:101800000A4B13B503400C00062B08D0830704D104
:101810000268074B92699A4201D0FFF7E5FA01A9E5
:10182000FFF7D0FB019B236016BDC046070080FF79
:101830009D1D0000F0B59BB00B9005910892102102
:101840000EAA12A8099314F0DBFA059B089A93429A
:1018500008D30B9A12AB13CB13C21B6813600B98FF
:101860001BB0F0BD059B19785D1C7D290ED1089B2E
:10187000AB4208D9059B59787D2904D112A825F0DF
:10188000A2FC059507E0BC480BF0A0FD7B2906D023
:1018900012A825F098FC059B01330593D5E7089B1A
:1018A000AB4216D9059B59787B29E7D02B007D29BF
:1018B00003D0212901D03A290DD100252E001A7814
:1018C000212A11D0002206921AE0089A01339A4286
:1018D00001D1AA48D8E71A787D2A03D0212A01D05D
:1018E0003A2AF2D11E00EAE708995A1C91421CD903
:1018F0005A780692723A012A17D802339942E8D9E7
:1019000000211A7805913A2A1FD15A1C5B7805925A
:101910007D2B1DD1089B059A9342DAD90027059BA0
:101920001B787D2B17D09648AEE79648ACE7197820
:101930007B2905D10132013308998B42F7D3C8E7DF
:101940007D29F8D1013A002AF5D1059F0593E6E7F4
:10195000059B0122F0E7002D48D00023287816933C
:1019600006F086FE00283DD0099B1B680793002BDC
:1019700001DD854888E716AA3100280020F0D9FC4F
:10198000209A169B013A04009A4203D87F49804866
:1019900023F050F8219A01339B009D580122099BA6
:1019A00052421A60B44231D27A480BF001FF01343E
:1019B000B44204D223782E2B01D05B2BF7D1611BCC
:1019C00001222800FFF7C4FA002205000100229836
:1019D00007F0D2F8002807D129006F4821F01BFC3E
:1019E0000AF07CFE2C00E3E74568DBE7099B1B68F7
:1019F000002B01DA694847E7209A013A9342C5D2A1
:101A0000013321999A005558099A1360002F00D08C
:101A1000A6E1069B3C00002B04D0069C733C631E91
:101A20009C41E4B210AA102116A814F0E9F929008B
:101A3000220010A800F052FF16A95948FFF752FAE9
:101A400001235B4205000D931093002F00D18FE01E
:101A50000EF096FF229B059A0293219B3900019379
:101A6000209B16A80093099BFFF7E4FE16A825F01B
:101A700098FB0026179B0400C3180A93037806936B
:101A8000B34208D0474F1900380027F0DAF9B042C6
:101A900000D16EE1013423782B2B4ED000272D2B63
:101AA00002D0202B01D1043701342378232B02D11B
:101AB000133B1F4301342378302B07D1069B002BA7
:101AC00001D13D330693002E00D130360DAA0A997C
:101AD000200020F02EFC037807902C2B04D10C3B27
:101AE0001F43030001330793079B1B782E2B06D15E
:101AF000079810AA01300A9920F01BFC0790079B59
:101B00001C78002C1BD02100274827F09AF90028C8
:101B100003D0079B5B78002B11D02448B4E631003A
:101B2000380027F08EF9002804D033000234069ED6
:101B30000693B0E706900600ADE70227B4E716A8C3
:101B400025F003FB069B002B08D12800FFF728F99E
:101B50003C230693002801D002330693002E00D1C7
:101B6000203606231F4229D0732C23D110488BE640
:101B70003C003E00E9E7C046D1FD020012FE020033
:101B80002AFE0200F9FD02004EFE020098FE02004D
:101B900084A90200B1FE0200C0A90200CEFE02002C
:101BA0000C9A020018FF02001DFF02002DFF020028
:101BB00046FF0200632C01D1714865E6069B3D2B70
:101BC0001FD05E2B1FD03C2B01D13B3B1F43280075
:101BD000FFF7CAF800282DD0632C50D026D8472C08
:101BE00013D8452C26D2002C40D0252C22D02800FA
:101BF00020F01DFD220003006249634806F052FCFC
:101C0000EEE64023E2E78023E0E7582C53D0622C35
:101C1000EDD1002303930D9B0222029361230196D1
:101C2000009729000EA813F0FFF834E6672C17D8A8
:101C3000652C1BD32800FFF7B3F800286CD0002CCC
:101C400056D06E2C54D0472C3FD8452C41D2252C51
:101C500050D0280020F0EBFC220003004B49CCE7D9
:101C60006F2C1AD0782C26D06E2CC0D10023039371
:101C70000D9B01960293009761230A22D1E7280069
:101C800000F0FCFE0D9B16A90870012201933B0099
:101C900000960EA813F06CF8FDE5FB0602D5802334
:101CA0009B001F43002303930D9B01960293009713
:101CB00061230822B5E70022230003920D9A173B07
:101CC0000292019600971022ABE72300653B022B9E
:101CD000BFD8280000F036FF109B220002930D9B16
:101CE000011C01933B0000960EA825F04EF8D2E5AA
:101CF0006724EEE72800802400F024FF244918F030
:101D000071FE109B640002930D9B3C430193011CE8
:101D1000009623006622E7E7069B3D2B01D11D4874
:101D2000B2E5002C01D0732C13D116A92800FFF7BF
:101D300067FD109B0100169A002B00DA1092109B91
:101D40009A4200D916930D9B00960193169A3B0078
:101D50009FE7280020F06BFC220003000E494CE7AF
:101D6000069B002B00D058E601235B420D93109395
:101D70006EE66678002E00D0D1E606968BE6C04669
:101D800072FF0200A5FF020008AD0200D6FF0200AC
:101D90000000C8420A0003003F000300F0B5A1B0F4
:101DA00005000C000D920A2800D0E4E10DAB0F9362
:101DB0000123073D1093059215403CD11368BF4A9B
:101DC000934206D10FAA10A9059821F02CF8059589
:101DD00002E0BB4A9342FAD1109B11A907930F9BD3
:101DE00020000893FFF7EEF8002309900A93A30759
:101DF00005D1B44A23689B1A5A425A410A9214AA3E
:101E0000102118A813F0FCFF119A00279446099B93
:101E1000099C63440493049BA3420FD8079BAA48E0
:101E2000BB4229D10A9BA948002B00D0A54818A97C
:101E3000FFF758F8BAE100230593CDE7217825296B
:101E400004D018A825F0BFF90134E4E7049B661C10
:101E5000B34202D89E480BF0B9FA6178252904D123
:101E600018A825F0B0F93400EEE70025282915D18F
:101E7000059BAB4202D197480BF06CFCA01C0600FE
:101E80003378292B23D1311A0122FFF761F80100A1
:101E900005980EF083F80127050001360023340071
:101EA00040220026302104200B9320330693049B0C
:101EB000A34213D800231293049BA34231D9237861
:101EC0002A2B70D1079BBB4221D88348D4E7049BBF
:101ED000B34201D88148BEE70136D1E723782D2BE4
:101EE00003D12C3B1E430134E1E72B2B01D1293BCD
:101EF000F8E7202B01D10643F5E7232B04D0302B44
:101F0000D8D116430691EEE710230B93EBE77B1C29
:101F10000C93089BBF00F85800F0B0FD0C9F129086
:101F2000013401235B421393049BA34292D923788B
:101F30002E2B17D1049B601C83428BD963782A2BEC
:101F400038D1079BBB42C0D97B1C0C93089BBF00B8
:101F5000F85800F093FD0C9F13900234049BA342A9
:101F600000D877E7002D06D1079BBB42ADD9089A70
:101F7000BB009D5801372278672A45D8652A00D3CF
:101F8000B8E0582A5DD01DD81300453B022B00D87D
:101F9000B0E0099B5249E41A00941300514806F03E
:101FA00081FA0AF09BFB200012AA049920F0C1F9E3
:101FB0000400B6E7002313AA0499139320F0B9F99B
:101FC0000400CBE7632A49D0642AE2D103222B0024
:101FD0001340022B0AD1444B2B40062B06D0FF2383
:101FE000DB05E81890430AF0CBF90500139B0A22A1
:101FF0000393129B00960293069B01936123290091
:1020000014A812F011FF1FE7732A16D8722A00D302
:1020100080E0692ADAD06F2ABBD10B9B002B02D05B
:1020200084239B001E43139B00960393129B08225C
:102030000293069B01936123E1E7752AC6D0782AB3
:10204000A7D11300139A173B0392129A0292069A91
:1020500001920B9A164300961022D0E7224B2B4098
:10206000062B05D0AB0716D1184B2A689A4212D11D
:102070001CA92800FFF7C4FB1C9A0100012A01D00B
:102080001A48F9E6129B019320230093330014A809
:1020900012F06EFED8E62800FEF766FE00280BD090
:1020A000280000F0EBFC129B1CA908700193202370
:1020B000012200933300EAE70D48DDE64CA0020060
:1020C00074C20200A09202009CFD02000C9A020061
:1020D000D7FC0200E9FC020016FD020000FD020030
:1020E00067FD020008AD0200070080FF3DFD020011
:1020F00056FD0200280000F025FD139B2278029374
:10210000129B011C0193069B14A80093330024F03A
:102110003CFE99E616AA10211CA813F071FE237844
:102120001A00723A51424A41D2B2722B09D00A9B2C
:10213000002B06D0AB0704D1594B2968994200D136
:102140000422290016A800F0C9FB139A1D9B002A3F
:1021500000DA1393139A9A4200D91A00129B1E991F
:102160000193202314A80093330012F001FE1CA851
:1021700024F0EBFF68E6080000F098FB16A90700C2
:102180002000FEF71FFF0590072D22D118A90D98FA
:1021900000F0B2FC03000020834207D0189981426E
:1021A00006DC404B40489F4200D10E2021B0F0BDDC
:1021B000169B1CA8594324F0B7FF1E9B01210493D2
:1021C00000930598189B169A23F013FD1CA938005C
:1021D0002EE60D9800F06AFBB8420FD11CA90D98AD
:1021E000FEF7F0FE1C9E04901D2D17D8192D4ED21F
:1021F000052D21D0122D1FD00020D7E7284B0D9898
:102200009F4209D101221CA920F028FA0028CDD034
:102210001C9B1D9E0493E7E7FEF7E6FD1F2DEBD107
:102220000123049A009316993300059820F099F839
:1022300000282AD01D48B9E7169B002B07D10D981E
:1022400000F034FBB84202D10D9C2000AEE7002E16
:10225000FBD0169B1CA8F11824F066FF1E9B169A53
:1022600005991800069326F094FD169A1E9B944635
:102270000593634418003200049926F08AFD1CA9D6
:102280003800FEF72FFE0400DFE709488EE70096CE
:10229000049B169A0599280023F0E1FCC8E7C04684
:1022A000A09202000C9A020090920200CCE7020079
:1022B000C4E70200F0B5050087B008680C0000F024
:1022C000F5FA0090012D28D96668022D26D0A06865
:1022D00000F0D4FB05000021080024F0C1FB04A994
:1022E00001902068FEF76EFE049B0400C7183E4B69
:1022F0009E4241D1BC422AD2207806F0A1F90028A2
:102300000FD1002D0FD121003A1B009820F048F882
:102310000100019811F060FF19E0334E01256D4274
:10232000D9E70134E6E72600307806F089F900287D
:1023300002D10136B742F7D82100321B009820F0B5
:102340002FF80100019811F047FFB74209D8019812
:1023500007B0F0BD0136B74203D1002DF7DD013DD6
:1023600006E0307806F06CF90028F3D1002DF6DC99
:10237000BE42ECD23400C4E7300000F097FA009B74
:10238000984202D03000FEF72FFD05A93000FFF77C
:1023900037FA059B0390002B13D114480BF016F865
:1023A0003E002100321B00981FF0FAFF0100019847
:1023B00011F012FFBE42CAD2059BF418002D00DDB9
:1023C000013D2600059B0293002DE9D0029BF318E6
:1023D0009F42E5D3029A0399300026F0CBFC0028F7
:1023E000DFD00136F0E7C046E4B30200710003001D
:1023F000F0B507008BB00D00022807D8290038007F
:10240000FFF758FF050028000BB0F0BD086800F08A
:102410004DFA08A9049028686E68FEF7D3FD019074
:10242000A86800F02BFB041EE8DB431C1800002109
:10243000059324F015FB2F4B05009E4202D12E4838
:102440000BF0B6F909A93000FFF7DAF9099B0690FD
:10245000002B02D129480AF0B9FF089A019B944643
:1024600063440293A3000393099F029BDE1B002C8D
:102470000BD0019BB34208D83A000699300026F0F1
:1024800079FC002821D0013EF1E7EB68A6009F19F6
:10249000019A029B01999A1A04981FF081FF3860F3
:1024A000002CB0D0059B1C1BEB68A70099193A00C3
:1024B000180026F077FC6B6800211A1BEB6892006D
:1024C000D81926F082FCAC609DE7039AEB6894462D
:1024D00063440793029BF1199A1BD21B04981FF0C7
:1024E0005FFF079B013C1860039B0296043B03932C
:1024F000BAE7C046E4B3020008010300710003001C
:1025000070B50C008AB0050004A920681600FEF71B
:1025100059FD00230593049B0100C218029605ABE8
:1025200006A801940095FFF785F906A90248FEF771
:10253000D9FC0AB070BDC0460C9A020010B5040068
:10254000002906D0044B8A6B03600968002306F05B
:1025500015F820000AF0C2F818AC0200F0B504002B
:1025600087B0039202936618002A06D0023A222A04
:1025700003D935480AF02AFF0134B44229D2207821
:1025800006F05EF8071EF7D123782B2B1CD10134FF
:10259000311B200003AA20F014FA23181C00002588
:1025A0000193B44217D3002F00D06D4201236D0078
:1025B0001D43019B9C422FD12449039A244805F0D6
:1025C00071FF0299FFF7BAFF2D2BE1D101340127EA
:1025D000DEE70027DCE723781A00303A0092092A68
:1025E00007D9202213431A00613A192ADBD8573B36
:1025F00000930399009B9942D5D9280005F004FC6B
:10260000002816D1039B5D43009BED186B006B40C7
:102610000FD40134C5E70134B44205D2207806F066
:102620000FF80028F7D1C7E7B442C5D1280007B09A
:10263000F0BD019B3A000593F11A05A8039B23F016
:1026400065F8059C0500B4E7550103007801030017
:1026500008AD0200F0B504008BB008934318049253
:102660000193019B9C4200D3F6E0207805F0E8FF3F
:10267000071E38D123782B2B37D101340590019BCD
:102680009C4200D3EAE0202322781A43692A33D1FE
:102690000199A21C914200D8E6E062781A436E2AA2
:1026A00000D0E1E0A2781A43662A00D0DCE0E21D07
:1026B000E51C914214D9E2781A43692A10D1227993
:1026C0001A436E2A0CD162791A43692A08D1A27979
:1026D0001A43742A04D1E2791343792B00D10535CA
:1026E000FF26F6051BE00134BBE705902D2BCAD170
:1026F0002C3B01340593C2E76E2A2ED10199A21C0E
:10270000914200D8B0E062781A43612A00D0ABE071
:10271000A27813436E2B00D0A6E05D4EE51C059B0E
:10272000002B02D080231B06F618A5427BD1594905
:102730008CE03D002B786F1C18003038092834D805
:10274000022E15D10A23029A53431B180293019BB0
:10275000BB42EED8002304934DE000220792029280
:102760004D4A250006920022002603920993E1E7D4
:1027700018F0AEFC051C012E0DD1069918F032F9A7
:10278000011C039817F0BCFD43490390069818F00C
:1027900029F90690DBE74149039818F023F9291C31
:1027A00017F0AEFD00260390D1E7002E03D12E2BAB
:1027B00003D10126CBE7022E16D0099A1A43652AC7
:1027C00012D1019BBB4256D96B782B2B05D1AF1C84
:1027D000019B9F42ABD00226B9E702262D2BA8D140
:1027E0002C3BAF190793F3E7049A002A04D0202268
:1027F00013436A2B13D13D00079B002B02D0029B91
:102800005B420293029818F019FC011C23481BF04C
:10281000D5F8039918F0E6F8049F061C7FE700231B
:102820000493E9E70135019B9D4205D2287805F024
:1028300007FF0028F6D17AE7019B9D4200D076E79A
:10284000089B002B01D1002F1AD01549154820F004
:10285000E9FC1099FFF772FE002305930023039310
:10286000002325000493CCE7059B002B00D15EE7F5
:102870002500002656E7019BBB4200D157E769E7D8
:10288000032302209E43084B3043C0180BB0F0BD19
:102890000000C07F3B010300CDCCCC3D00002041B7
:1028A0001E01030008AD020000008080074BC20734
:1028B0000AD4074A074B0240062A05D00322064BDA
:1028C0000240022A00D00368180070472CB90200A9
:1028D000070080FF0C9A020088B0020070B50D005E
:1028E000040016000EF04CF82800FFF7DFFF8368A5
:1028F000002B04D0320029002000984770BD4268A8
:102900000249200024F086FAF8E7C046E4020300FA
:1029100010B50A0001000248FFF7E0FF10BDC046F5
:1029200084E80200F7B5050008000E0020F07EFCE8
:10293000002810D001AA6946300005F053FE009B24
:10294000002B08D01749280024F0A3F9009CE71EAB
:10295000A400002F09DA310028000222FFF7BEFF91
:102960002800114924F095F9F7BD019B28001A1998
:1029700011000C3A08390B6812680C4924F04AFA25
:10298000019B1B19043B1A68002A06D1064928003E
:1029900024F07FF9033F0C3CDBE70549280024F0D5
:1029A00039FAF7E7A2020300654F0300C6020300ED
:1029B000DB02030010B50400FFF778FF054B006948
:1029C000984203D0431E9841C0B210BD200021F0B0
:1029D00067FFFAE7F5BA000070B505000C000120AA
:1029E0008D4203D0214B9D4201D1002070BD994200
:1029F000FBD001231D4204D01942F6D12B000D005B
:102A00001C002A001A4B1A40062A05D0AA0711D129
:102A1000184A296891420DD12340062B05D0A307FF
:102A2000E3D1144B22689A42DFD121002800FEF73F
:102A300097FEDBE72340062BD7D0A30703D10D4B2E
:102A400022689A42D1D02800FFF730FF8369002B1B
:102A5000CBD0220029001B2098470028C5D0064B68
:102A6000C01A43425841C0B2C0E7C046E4B30200B6
:102A7000070080FF0C9A0200CCE70200104B10B553
:102A8000984219D00F4A0123904217D0184201D022
:102A9000184110BD830706D10B4B02689A4202D140
:102AA0000CF036FFF5E71FF0C2FD084902000848A8
:102AB00005F0F8FC09F012FE0020EAE71800E8E74C
:102AC000C4E70200CCE702002CB90200690203004F
:102AD00090AC020010B5C30705D4830706D1054B9F
:102AE00002689A4202D122F028FE10BDFFF7C6FF0D
:102AF000FBE7C0462CB902000F4B70B50D00012456
:102B0000984204D100230B602300180070BD0B4BCA
:102B1000984201D10C60F7E70300234002D0401037
:102B20002860F1E78207F0D1054A01689142ECD1B3
:102B30000CF0EEFEF4E7C046C4E70200CCE702006A
:102B40002CB90200184B10B5984228D0174B984268
:102B500027D0C30703D5401018F070FA10BD032327
:102B6000184206D1124A0168914202D122F0EEFDCC
:102B7000F4E702001A40022A08D10E4A0240062A4F
:102B800004D0FF22D20580189843E7E71FF04FFDDD
:102B900009490200094805F085FC09F09FFD002065
:102BA000DCE7FE208005D9E7C4E70200CCE702009D
:102BB0002CB90200070080FF4F02030090AC020016
:102BC00010B583070CD103680A4CA34202D120F050
:102BD0002AF910BD084CA34202D123F058FFF8E7B0
:102BE0001FF025FD05490200054805F05BFC09F0D2
:102BF00075FDC0464CA0020088E70200FF010300FB
:102C000090AC020013B50C0001A9FFF7D9FF019B9E
:102C1000A34206D022000349034805F043FC09F013
:102C20005DFD13BD2202030008AD0200F7B50500EB
:102C30000C0017001E00D3070ED557100197019BFB
:102C4000002B1FDA1B190193002E1DD0002B15DA63
:102C5000002301930198FEBD01A91000FFF74CFF6E
:102C60000028ECD138006C681FF0E1FC2200030062
:102C70000B490C4805F016FC09F030FDA342E9D9D8
:102C80000194E7E7002EF9D1019B002B01DBA34261
:102C9000E0D36A680449054805F004FCECE7C04647
:102CA000C501030090AC0200E901030084A9020001
:102CB00010B50400830710D10D4B02689A420CD165
:102CC0000C4B0340062B06D1C00822F04EFE4300F9
:102CD0000120184310BD8068F9E72000FFF7E6FDEA
:102CE0004369181EF6D0210001209847F2E7C0463C
:102CF000A0920200070080FF164B70B50400002070
:102D00009C4203D0144DAC4201D1012070BD134B45
:102D100000209C42FAD001262640864203D0601053
:102D2000431E98410DE02000FFF7C0FD4369002BD2
:102D300009D0210030009847002804D0401B4342AE
:102D40005841C0B2E2E72000FFF7B2FF0028DCD014
:102D50000138E5E7C4E70200CCE70200E4B3020073
:102D600010B50400FFF7A4FF002809D120001FF0D0
:102D70005EFC04490200044805F094FB09F0AEFC37
:102D800010BDC0468102030090AC020070B5040083
:102D90000D001600FFF78AFD036A002B05D03200F4
:102DA000290020009847002818D10D4D2000002E42
:102DB00008D11FF03CFC02000A49280005F072FB14
:102DC00009F08CFC042E04D11FF031FC06490200EE
:102DD000F3E71FF02CFC05490200EEE770BDC0468A
:102DE00090AC0200E9020300140303003503030062
:102DF00010B51FF033FC002802D102480AF0AAFCEB
:102E000010BDC046A001030070B5050000291CDB01
:102E1000032905D80800002416F076FF18180606C6
:102E20000123023999430C00FE26B52109023143E2
:102E300028001FF02DFC002C04D005492800214358
:102E40001FF026FCAE61EC6170BD0024F226ECE7B9
:102E500080B0000010B50D4C206824F053FC002811
:102E600007D00B4B1B78002B03D1206803685B68ED
:102E700098470023074A1370074A13700BF030FC81
:102E80000CF05CFA0EF038F810BDC0465C2900204A
:102E9000CB2D0020CA2D0020392E002070B5050052
:102EA00094B0002804D13F481DF0D4FD14B070BD8B
:102EB00008A809F0EDFB041E19D12E68290004A80A
:102EC00001220EF0C7FE23002200310004A808F002
:102ED00099F90400032001F0A1F8200021F05FFD22
:102EE0000120404201F09AF809F0F0FBDEE70120F2
:102EF000404201F093F809992B48FFF713FD099818
:102F0000FFF7D4FC2949040008F0E6FE0028CDD1E3
:102F10002749200008F0E0FE0028C7D1099C01AA3B
:102F20006946200005F05EFB02AA322104A812F0D7
:102F300067FF009B022B05D9019B1E495A6802A816
:102F400023F068FF2000FFF7B1FC1B4BC2689A42D8
:102F500010D1236819495A6802A823F05BFFE3687F
:102F6000002B07D05A68002A04D00022996802A8D2
:102F7000FFF7B4FC032001F051F804A824F011F984
:102F800006F034FC04A824F0E0F80120404201F0EF
:102F900045F80B4B9A6C002A00D187E700229A640F
:102FA00084E7C0469803030084E8020054AC0200A2
:102FB000FCA90200C503030065830000CE030300E3
:102FC0007C2E0020F8B54E4C1321200025F0BEFCCD
:102FD0002000032125F050FD4A4C01234A4A1321C9
:102FE000200016F017F801220221200016F042F806
:102FF000464C200013F0F2F9454F3860200013F0E2
:1030000009FC444D2860102025F059FE0400296871
:103010000025414E3A68330013F042FF3F4B1C60DD
:103020003F480DF08DFCE120C0000DF099FC3D49BA
:103030003D480AF07FFE09F071FB06F053FB01F0FA
:10304000A5FE13F031F8300024F0A3FF22F04AFA75
:1030500000F064F904F0E0F901F07EFC0AF0D4FC21
:10306000324C3348230088331D600BF0ADFB0BF06E
:1030700089FB0AF0DBFC2F4F3B78012B0ED100239C
:1030800007211A002C4800F051FA031E1DD0010040
:10309000F720400000F0D2FBFFF700FF3B78002B49
:1030A0002AD112F0ABF90028F8D0244820F004FB14
:1030B0000BF078FB08220021214825F086FE230032
:1030C00098348C331D602560AAE7F82292021178AB
:1030D0004D2909D15178502906D1F7205288194934
:1030E000400022F05FFDD7E70122174917200AF0C0
:1030F000A5F821F07EFCD1E712F0D0F9D3E7C04665
:103100003C2900205429002017280200DC29002037
:10311000582900205C290020642900206029002013
:10312000004000203C2900203C0100207C2E002093
:10313000552E0000EA000020D2030300DA0303004A
:10314000FC2E002004E0030044A0020010B5084C4F
:10315000084A0621200013F075FF074A074920009E
:1031600025F0A6FD00221E21054824F01CFF10BDFD
:10317000642900208C94020000000020FD6F0100F3
:10318000DC29002070B505000C200C0023F091F81C
:10319000024B45600360846070BDC046A494020089
:1031A00010B524F09CF8014810BDC046E4B30200FD
:1031B00010B5C30708D483070ED10368094A9342A8
:1031C00002D0094A934207D1FFF758FC002801DDDD
:1031D00020F07FFA054810BDFFF7B4FC17F00EFF92
:1031E000F4E7C0462CB90200D4E70200E4B30200C1
:1031F00001220B4B10B51A600A4A51680029FCD015
:1032000000215160A1220131D2009A585960032354
:10321000D01718408018801022F052FA10BDC04616
:1032200000C00040FCC0004010B5002804D1044894
:1032300012F05CFE034810BD0868FFF71FFCF7E7BB
:10324000E7030000E4B3020080235B051869034B29
:103250001B7843438020C002C01A7047C72D00204E
:1032600080235B051869034B1B7843438020C00211
:10327000C01A7047C82D002070B5084DC4012B68D6
:103280000021181921F0E3FB2868054B00197F3055
:1032900000781B788342F0D270BDC046F42900202C
:1032A000C62D002010B5C3790400002B08D0064AB3
:1032B000037981791068DB01C018013021F0C7FB68
:1032C0000023237210BDC046F429002010B5124B14
:1032D00001001A684379DB01D31818007F300478A5
:1032E000FF2C08D10879C00112185278FF2A0FD09C
:1032F000887990420CD08A799B180132D2B25878E2
:103300007E2A01D08A7110BD00234C718B71FAE7BF
:1033100001204042F7E7C046F429002070B5F824A8
:103320008025A40223786D054D2B4CD12B6980207C
:10333000E41A2B69C002E41A2969001B16F0F8FC94
:103340002B4B2C4918702B69E21852185D4215401E
:10335000294B2A4A9B1A2A4A9B1880225205116936
:103360009D4234D38020C002401B16F0E1FC254B67
:10337000641B1870E411244BE4B21C70A1200123DB
:103380000025224A22491360C0004D604B68002B83
:10339000FCD01358DBB2A342F7D21E4901330B70A5
:1033A00001235360FFF750FF037805001A4CFD2BF3
:1033B0000FD180235B051869184BC009C018C001E4
:1033C0002818206070BD80242B69E402AFE76D18D7
:1033D000C5E7FFF745FF0378803DFD2B01D1256050
:1033E000F0E7FFF73DFFFD2121F031FBF7E7C04695
:1033F000C82D0020FF87FFFF1401002000000020DF
:10340000A4870300C72D0020C62D002000D0004057
:10341000FCD00040C92D0020F4290020FFFFFF014F
:10342000F7B5254B254F1A78254B14001B783968C2
:103430000133E001405CFF2829D00134E4B29C4212
:1034400000D101249442F4D1802300265B051B693E
:10345000DB090193E30100933B68E2019D182B789F
:1034600028005A425341F61821F007FB002810D0DB
:10347000002304E0DA01AA5C002A0AD10133019A90
:103480009342F7D13868009BC01821F0ECFA200075
:10349000FEBD0B4B01341B78E4B201339C4200D1DA
:1034A0000124054B1B78A342D4D1072E02D91FF06B
:1034B0000CFAB6E7FF24EAE7C92D0020F429002022
:1034C000C62D0020F7B507000D0001240E4B1B7818
:1034D00001930E4B1E68019BA34202D2FF242000E1
:1034E000FEBDE10171180B78FE2B09D18B78AB4240
:1034F00006D103312A00380025F03CFC0028EED02C
:103500000134E4B2E7E7C046C62D0020F4290020CC
:1035100010B5054A03791068DB01C01881780022D4
:103520000330FDF715FD10BDF4290020F0B585B07E
:1035300002900D0016000393782948D8FFF7C2FFC8
:103540000400002E3BD0FF2801D0FFF795FEFFF7C7
:1035500067FF0400FF2803D11E491F4821F06AFAC3
:103560001E4FC0013B680190FE21181821F06FFA30
:103570003B68019AE9B29818023021F068FA38687D
:10358000019B2A00C018033002990BF037FA0C2077
:1035900022F08FFE039A0300002A16D0104A1A6008
:1035A0000E4A1C7112685C71E4011419A278DE7174
:1035B00002329A7101221A72039A5A7202E033009F
:1035C000FF28E4D1180005B0F0BD064AE7E7002364
:1035D000F8E7C046E803030028AB0200F429002006
:1035E000ECBA020098BB020007B501A9FEF708F982
:1035F0000199FFF767FFFF2803D10449044821F030
:1036000019FAFFF739FE03480EBDC0461B0403003C
:1036100028AB0200E4B30200F7B50192027A04007D
:103620000091002A02D1244809F0D0FEC579002D6E
:1036300006D1224A17680279D201D25D002A05D14B
:10364000092201251A606D422800FEBD61797E22A3
:10365000C901791808007F30A3790078D21AFF28B1
:1036600009D12079C00138184078FF2819D0C01A34
:10367000824200D902000198461B964200D91600EA
:10368000002EE1D0009A01335019C918320025F0FC
:1036900080FBA3799B19DBB27E2B04D0A371AD19FB
:1036A000D4E70022E7E70023A3716379DB01FB186D
:1036B0007F331B786371F2E7FE030300F4290020D7
:1036C000F0B585B00393037A040002910192002BB8
:1036D00002D1304809F07AFEC379002B08D02E4A77
:1036E00003791268DB019B5C019A0092002B25D1C3
:1036F0000923039A13600A3B0193019805B0F0BDBA
:103700007E22A379D71A009A974200D917006079D0
:10371000214E0133C001C01833683A0018180299CD
:103720000BF06CF9A379DB19DBB27E2B0AD0A37105
:10373000029BDB190293009BDB1B0093009B002B79
:10374000DED1DAE70023A371FFF76AFE0500FF2848
:1037500009D12079FFF790FD002323721C23039ADF
:1037600013601D3BC8E760793368C0011818290051
:103770007F3021F06CF93368ED015819617921F03F
:1037800066F962793368D2019B187F331B786371C5
:10379000CEE7C046FE030300F4290020002170B5E7
:1037A000080023F05DF9012405000C4B1B78A342AF
:1037B00001D2280070BD0A4AE3011068C0180378DE
:1037C000FE2B08D1817800220330FDF7C1FB0100F8
:1037D000280010F001FD0134E4B2E6E7C62D002018
:1037E000F429002073B501A9FEF70AF80199FFF743
:1037F00069FEFF2803D10E490E4821F01BF9002570
:103800007E260D4B1C68C301E31859789B78023360
:10381000DBB2C201A2187F321078FF2804D1C81A87
:10382000401921F04DFF76BDF31AED180023F0E7A3
:103830001B04030028AB0200F42900201FB5034A33
:10384000034B22F072F905B000BDC046CD32000036
:10385000A5320000044B054A05481A60054A5A6023
:1038600000221A817047C046FC290020200307006F
:10387000E4B3020074696275F7B51600314A0B00B3
:1038800088321768002F02D12F4809F09FFD0221CE
:103890002E4C2F4DE167A324E4002C592D4AE4B2AD
:1038A00006343C192C4F3D68A54204D12B4B1160C6
:1038B00001930198FEBD2578002832D1601C002BB1
:1038C00004D12900FDF75CFB01900BE05A68AA4285
:1038D00000D92A000100186825F064FA01226B0063
:1038E0001A430192002E0ED0621953785B42336066
:1038F000D37811791B0209040B43917852790B4359
:103900001206134373603E68A91D6118721A2000E5
:1039100025F048FA0223751B0E4A063D3D601360F0
:10392000C7E7022D04D8002303600E330193D9E7C3
:103930002100042225F02DFAE91E201D0022FDF7AA
:1039400007FBC1E77C2E0020AC04030004E100E08B
:103950000010004000E100E0082A0020E4B302006B
:103960007FB5002101AA0800FFF786FF0A4B9842A5
:103970000FD00121019B03905A00029B0A438B4008
:103980000492064A032013400B4303A9059302F057
:1039900071FE07B000BDC046E4B30200FEFFFF7F2A
:1039A000002213B501AC11002000FFF765FF094BA1
:1039B00098420ED02378022B08D96378012B05D1C9
:1039C000A378002B02D1E378012B02D0024809F042
:1039D000FDFC16BDE4B302008C04030002220B4B75
:1039E00010B5DA6700220121094B5A61094A1161B9
:1039F0005A69002AFCD0084C88342068002803D07B
:103A000022F086FC0023236010BDC04604E100E0E4
:103A1000FC100040001000407C2E002010B5FFF785
:103A2000DDFF014810BDC046E4B30200F8B5FFF762
:103A3000D5FF364C26786578063601357543280063
:103A400022F037FC324A861916600022314B4519A4
:103A500088331860304B01211D60304B5A60802242
:103A6000D20511605A68002AFCD003212C4B615604
:103A70002C4A00259950A178043A9950617A08326D
:103A800099506168284A08269950217A274A284F78
:103A900099500121274A9D5004329950264A9E5040
:103AA0008122247892042243A324E4001A510224A0
:103AB000224A9C50224A9F50224F043A9F50182776
:103AC000214A9F50214AC0279850C12292009E50FF
:103AD0001F4ABF00D0591F4E0640C020000230438D
:103AE000D051C020400014501460102280301C5867
:103AF00022431A50184A5560596051680029FCD079
:103B00000021116101229A60F8BDC046FC29002005
:103B1000082A00207C2E0020F8290020FC0000400C
:103B2000001000400C0500001C05000024050000EA
:103B3000FFFF00002C050000140500003405000004
:103B40003C050000211001005405000004050000A0
:103B500000E100E0FF00FFFFFC10004010B5FFF7A0
:103B600065FF014810BDC046E4B30200F0B5050092
:103B70008DB01600002802D0694809F0EBFD694BB2
:103B800009AA190091C991C21A781F7A06925A7827
:103B900005929A78039203229A5604925A685B7AA5
:103BA000019202937368AB424CD9EB000793B36860
:103BB000EA009B181A68002A1BD0042A19D05868FA
:103BC000FEF788FFB368EA0004009858FDF7E2F9B1
:103BD0000200B338FF3806282ED816F095F8040CEA
:103BE000131920262800631EFA2B00D995E0E3B2B2
:103BF00006930135D6E7631EFD2B00D98DE0E3B2B5
:103C00000593F6E7532C00D987E0E3B20393F0E77E
:103C1000072C00D981E0444B1B570493E9E7022CA1
:103C200000D97AE0E3B20293E3E70194E1E7FF2CE5
:103C300000D972E0E7B2DCE73C493D4804F032FCD1
:103C400008F04CFD3B4B09AC88331B68002B12D1AC
:103C5000069B27722370059B6370039BA370049BD4
:103C6000E370019B0A93029B63722E4B07CC07C340
:103C700031480DB0F0BD069B2A4D2370059B637043
:103C800022882B889A420FD0FFF7A8FE039B277249
:103C9000A370049BE370019B0A93029B63720ECC9A
:103CA0000EC5FFF7C3FEE3E70222244B2449DA677F
:103CB0000022244B4A6101321A614A69002AFCD071
:103CC000039809AA907004981772D07001980A900E
:103CD00002985072134870CA70C01B4A04989850DA
:103CE0000398043A98500298083298500198174A5D
:103CF0009850174A9F5000224A6001325A604A6821
:103D0000002AFCD000220A61C02101329A60114BC6
:103D1000013249005A501A60AAE70F498DE7C046A0
:103D200036040300FC2900202E0403005104030084
:103D300008AD02007C2E0020E4B3020004E100E0A4
:103D4000FC100040001000400C0500001C050000A5
:103D50002405000000E100E067040300214BF7B5F3
:103D60005A68214D002A03D000225A600132AA600D
:103D70001A69002A34D000221A61A323DB00E85814
:103D80001A4BC2B2883319680C78A24201D21400CF
:103D900008708023DB00EB58012B1FD1144E154A0D
:103DA0003768A31D12680193FB189A4216D3621C50
:103DB000380024F0EEFFA923DB00EB58621CBB5453
:103DC00015F0F6FE3368020A1C19E270020C22712B
:103DD000019AA0709B18000E607133600123AB60E4
:103DE000F7BDC046FC100040001000407C2E0020B3
:103DF000082A0020F8290020F7B5314F00933B0036
:103E0000883301921A680E00002A02D12D4809F069
:103E1000DDFA02212C4B2D4CD96700232C4D636118
:103E200001332B616369002BFCD0A323DB00EB582B
:103E30000099DBB27118994203D9B3423DD39B1B61
:103E40000093009B8837F31813703B68010001331F
:103E50001800320024F09DFF009B002B06D038682C
:103E6000013680191A00019924F093FF0023636042
:103E700001332B606368002BFCD00123AB6000236F
:103E800023612369002BFCD00023636101332B6184
:103E90006369002BFCD00023636001336B606368AF
:103EA000002BFCD00023C021022223610133AB6030
:103EB000084B49005A501A60F7BD1E000023BFE7A7
:103EC0007C2E0020AC04030004E100E0FC10004064
:103ED0000010004000E100E007B501A9FDF790FCEB
:103EE000019B020003210248FFF786FF01480EBD37
:103EF0002A040300E4B302001FB5012201A9FEF762
:103F000077FF002301981A000299FFF775FF014817
:103F100005B000BDE4B30200030010B50548002B56
:103F200003D11FF072F908F0D9FB09681FF073F98B
:103F3000F9E7C04654AC020010B503480968FEF723
:103F4000F1FC024810BDC04684E80200E4B3020060
:103F5000F0B5802787B02B4D02907F422C78002C43
:103F60001CD063B2002B12DA6E787C40E4B2002ED3
:103F700014D0013CE4B2FF2C02D101350135EDE74C
:103F800004AB981D0121067005F0F2FBF1E704ABCC
:103F9000D81D0121047005F0EBFBEFE7052702981F
:103FA0001FF097FB0124BC4227DA0025164E2200A1
:103FB000290030000BF0A2FB6B4601901B79002B0F
:103FC00015D0631E1A002900300003930BF096FBF6
:103FD000031E0CD12200290030000BF05BFBFF22F6
:103FE000019B290013403000621E0BF053FB01358A
:103FF000052DDBD10134E4B2D5E7013F002FCED14E
:1040000007B0F0BDC70403001C00002010B5C82095
:10401000FFF79EFF004810BDE4B3020010B5040096
:10402000431C02D0024804F09BFA024B1C6010BDF6
:10403000A42E0020782E0020014B024A9A6470477B
:104040007C2E0020A42E002030B507240278084DD5
:10405000A24314000222224302707F22039C41608B
:104060002240D400028883602A402243028030BD6F
:1040700007FCFFFF10B50B00072401782340A14384
:1040800019437F23017004990A4C0B40D90003881F
:10409000426023400B430380039B04685905064B91
:1040A000C90A23400B430360029B8360059BC360E6
:1040B00010BDC04607FCFFFFFF03E0FF70B513789B
:1040C00004000A3BD8B20F2809D90A001048114948
:1040D00004F0E8F90025636A1860280070BD002527
:1040E00052781B021A43E36AAB420AD1238C0025A3
:1040F000042BF2D10849064804F0D4F9636A186029
:10410000EBE7206BA90009589142E6D00135EBE7B7
:1041100018AC0200E8060300FD060300F0B5040039
:1041200085B00D00100003A9A26A1E0021F03EFF19
:10413000002809D12A000B490B4804F0B3F9636A3F
:104140001860002005B0F0BD0398FEF7C3FC030023
:10415000B343F7D0030000962A000449024804F054
:10416000A1F9ECE7A406030018AC0200BC060300AA
:10417000F7B51F0013780E000A3BD9B2050021489D
:104180000F2904D850781B02184321F0F3FB1524A3
:104190000378009315231C491B1B0193A300CB1A22
:1041A000190055310978009A91421FD119005631F2
:1041B000427809788A4219D1573381781B788B422B
:1041C00014D1002B0FD1019B9A000F4BD05CB84249
:1041D00008D93B0032000D490D4804F063F96B6AC1
:1041E00018600020FEBDC378002BECD0013C002CF1
:1041F000D0D132000749064804F054F96B6A1860C0
:104200002000EFE73B83030060070300140703006F
:1042100018AC02002D070300F0B5137885B0050037
:104220000E00462B47D101A9100021F0EFFE019BA3
:10423000834240D003781A000A3A0F2A0AD80200B3
:104240000F2331002800FFF793FF01248440200052
:1042500005B0F0BDB32B2ED121F0D3FE040021F028
:10426000CBFE02900378B62B25D10127A73B220075
:1042700031002800FFF77CFF3C0003A9844002982E
:1042800021F0C4FE039B02909842E0D09D2102A839
:1042900021F0CBFE029A039B9A42D8D00F23310023
:1042A0002800FFF765FF3B00834002981C4321F084
:1042B000A3FE0290EEE732000349044804F0F2F84E
:1042C0006B6A00241860C2E74507030018AC0200BF
:1042D000F0B50E0087B0040004A930001F00019261
:1042E00021F04DFB019B0500002B0FD1A4239B0067
:1042F0009E4205D1BF21090220001EF0C9F919E034
:10430000BE4B9E4200D088E0BD49F5E7019B012BE2
:1043100000D09AE00A23FF339E420DD101003A6893
:104320002000FFF7CBFE010020001EF0FBF9002863
:1043300000D116E207B0F0BDB24B9E4209D1010098
:104340003A682000FFF7BAFE010020001EF042FA92
:10435000EDE7AD4B9E420AD101000F233A682000E1
:10436000FFF706FF8E21C000C9010143C4E70378AF
:10437000622B3BD1049B032B07D0052B36D1C3788E
:104380005F2B33D103796E2B30D101230E265B4294
:1043900069789E480293B300F31AC3181A002B32AF
:1043A00012788A4209D1AA7894461A002C321278DF
:1043B000944502D12A331B780293013E002EEAD1A4
:1043C000029B013329D03A6829002000FFF776FECE
:1043D000049B0200052B03D12E79773E73425E4188
:1043E0003300029920001EF0B9F9A0E7884B9E42E5
:1043F00001D1884980E7884B9E4201D187497BE7FC
:10440000874B9E4212D129003A682000FFF704FF33
:10441000FF231B02B421184215D0019B2A008149B9
:10442000814804F03FF8636A186083E77F4B9E423F
:10443000F3D13A6829002000FFF7EEFEFF231B02AC
:104440001842EAD1BC2109028FE7019B022B00D060
:1044500021E17B68764A1B780A3B0F2B48D89642AD
:1044600012D13A6801000F232000FFF781FE7A681D
:10447000060029000F232000FFF77AFE310002001A
:1044800020001EF038F955E700226A4B02929E4246
:104490001AD18026F6013A68290007232000FFF789
:1044A00067FE7A680190290007232000FFF760FE6D
:1044B000019A0300310020001EF016F93AE7029B32
:1044C000013302930F2BA8D0029B03229E005A4B6C
:1044D0002800991924F0D4FC0028F0D1EB78002BA7
:1044E000EDD1564BF65C80233601DB011E43D2E74B
:1044F00096421AD1802607233A6829002000FFF748
:1045000037FEFF23019029007A682000FFF706FE9E
:104510000100019BB6011B0231431943ECE6A026C2
:10452000E9E7C026E7E7E026E5E787239B009E4210
:10453000F5D01E3B9E42F4D0414B9E42F3D0414BFE
:104540009E4251D0404B9E4250D0404B9E424FD055
:104550004F339E424ED03E4B9E424DD03D4B9E42ED
:1045600000D05AE705233C4A9B009B5A290002933E
:104570003A6807232000FFF7FBFD7E68039033783D
:10458000452B6BD1300021F07CFD002866D1300036
:1045900021F037FD0378A62B60D105A921F036FD67
:1045A0000599060021F01CFD022857D1300021F0AA
:1045B00023FD07233200070029002000FFF7D8FD64
:1045C000029B0600DB0451D51F233A00290020007E
:1045D000FFF7A4FDF100039B029E80011E433143BF
:1045E000F826F6003040C0E60023BCE70123BAE716
:1045F000019BB8E70323B6E70423B4E7E602000013
:1046000030BF00000B0200000F0200006505030030
:104610002202000072B600002302000062B6000011
:104620009F0200001F06030018AC02009A0200005F
:104630008902000001020000690603006806030009
:10464000C50200006E0200006F020000710200004F
:10465000C1020000C302000098F602002A0044498B
:10466000444803F01FFF636A1860D6E66B460822D1
:104670009B5E002B07DA3E233A0029002000FFF75B
:104680004DFD4008A6E77C233A0029002000FFF7F3
:1046900045FD80089EE7019B032B00D0BDE69E23CD
:1046A0009B009E4222D100263A6807232900200061
:1046B000FFF75EFD7A680190072329002000FFF7CD
:1046C00057FD1F230290BA6829002000FFF726FD3E
:1046D000019F029B374381013943DE0031430BE6E2
:1046E00080263601E0E780267601DDE7224B9E42F8
:1046F000F6D0224B9E42F6D0093B9E422BD1C026DB
:1047000007233A6829002000FFF732FD07230190B4
:104710007A6829002000FFF72BFDBA68760113782C
:1047200002900A3B0F2B0DD8072329002000FFF72A
:104730001FFD029BD900019B194331430F008101EA
:104740003943D9E58023DB001E43290007232000DD
:10475000FFF7E4FCEDE70A4B9E4200D05DE6D02671
:10476000CEE708490348646A1EF05CFD2060E1E57D
:10477000F405030018AC02007902000007020000F3
:10478000C502000054060300F7B50E000700110033
:10479000300021F025FC0025040004281ED97C6A85
:1047A000134914481EF03EFD206000242000FEBD89
:1047B00073780002184321F0DDF80236019024F0EE
:1047C00058FB022811D1019B1B78722B0DD1019B44
:1047D0005A782B0030339A4207D10135A542E5D0F3
:1047E00030780A38C3B20F2BE2D97C6A0249D8E785
:1047F0008F05030018AC0200C2050300054B10B57D
:10480000186822F07BFF044B002800D1034B1800EE
:1048100010BDC0465C290020CCE70200C4E70200BE
:1048200010B5034B186822F071FF024810BDC04656
:104830005C290020E4B3020010B5034B186822F095
:10484000D3FF20F03DFF10BD5C29002010B5034BC5
:10485000186822F0D0FF20F033FF10BD5C29002043
:1048600010B5034B186822F0CDFF20F029FF10BDD2
:104870005C29002010B5034B186822F078FF20F067
:104880001FFF10BD5C29002030B593B009F08AFFEE
:10489000184C200023F078FB174D286812F068F8B8
:1048A000200023F076FB09F06DFF20F01BFE1EF0C8
:1048B0008EF90400296803A822F016FF0F4B200090
:1048C0000A93039B0B93049B0C93059B0D93069BF0
:1048D0000E93079B0F93089B1093099B01931193D1
:1048E00020F0C1F8200020220AA90AF087F8044825
:1048F00013B030BD642900205C29002055BA11C0D6
:10490000E4B30200F8B5114D0400286822F0F6FE69
:10491000002802D12000FFF7B7FF0D4B1B78002BBA
:104920000DD10C4E3478E4B2002C08D10127286850
:10493000377003685B689847054B34701F702868B0
:1049400012F0F2F820F0BCFEF8BDC0465C29002051
:10495000CA2D0020CB2D0020F0B58DB01EF037F908
:104960000E4B02689A4217D1046941680894446961
:104970008268C36809948469C0690A9484466C4655
:1049800005910692079308A8E0C8E0C4604620603D
:104990000348006822F092FE0DB0F0BD55BA11C078
:1049A0005C290020F0B58FB00692426809939446C6
:1049B0000368040002939B6804300093634403601F
:1049C0000E001EF011F9059060681EF023F9431CDB
:1049D00063600378A24A0193831C636043780021DB
:1049E0000093C31C63608378B5000393031D636069
:1049F000C3782000049323001033A360059B143078
:104A00009A1893000793C318E360079B0C331A00AE
:104A1000089324F0DAF9099B009A5B190B93059B24
:104A20009B1A039A0A939D1A2F1D009ABF00E7193B
:104A30000123B24264D2019A1A4207D13300009A8C
:104A40008849894803F02EFD07F048FE009B033596
:104A50009900099BAD005918009B6519F01A01F0E7
:104A600009FE009E043F68600022964200D070E07C
:104A7000069B002B03D1019B1B0700D4D6E0022329
:104A80000026019A1A400992B24204D0069820F0FA
:104A9000BAFE060038600027029B0B9DDB68089376
:104AA000069B9F425ED10A9B029805339B00E1184A
:104AB0000A00049D0C30002D00D080E0049A920082
:104AC0008918079A2032A2188A4200D980E0143B44
:104AD0000693009B089A9B00D3180793039B9D4263
:104AE00000D27FE065680DA80D951EF07DF82818AE
:104AF0000578461CFF2D00D0A7E066600FB0F0BD22
:104B0000019A1A4205D00335AD00584B6519043F90
:104B10006B60069B002BA7D1019B1B07A4D4009BB5
:104B2000049A9A1AB24212D8009A049B991A320037
:104B30008900009B9A4297D29300029D581828182A
:104B4000089D0069EB1AE31818610132F1E73300A0
:104B500076E7099908989300C958C31AE3181961B0
:104B6000013282E7009B039800221B189C462968AB
:104B7000944505D8099B002B1CD1CA083C490EE07E
:104B8000089B90001858884212D1059B013B9B1A44
:104B90009B00E3185A69002A05D0CA0835493248F3
:104BA00003F080FC50E76A685A610137083577E7FF
:104BB0000132DDE76A68300020F05EFEF5E7166836
:104BC000002E02D1AE0086591660013D043272E714
:104BD000081D0968002903D1121A92102649DEE740
:104BE000010071E7069AAB00D71AE7193A69002A63
:104BF00016D1082000996E180899B6008E190799E9
:104C0000C958019B03420DD0049B029804339B00BA
:104C10001858043003F0B0FF002803D043683B610C
:104C200001355BE732681549D208B8E7039B002BD2
:104C300002D0134808F08EFD019B9B0700D451E77A
:104C4000039820F0E0FD38604CE7ED43059BED183C
:104C5000AD00651968690AF0EBFD6861300047E74F
:104C6000FDFFFF3FB407030090AC020044A0020028
:104C70001C080300ED0703003D0803006F08030054
:104C80009F0803000048704716FCFFFF004870476C
:104C900016FCFFFF82B007B591B204920593052977
:104CA00009D01B2902D104A810F0C2FD002003B0D6
:104CB00008BC02B0184704AB5B88032BF6D106A9E9
:104CC0000822684624F065F80349049A059B0868A1
:104CD00011F042FFEAE7C046602900200022044BA1
:104CE0005A60044A08321A60034A13607047C0468B
:104CF0000C2A0020A0990200A02B0020F8B5214E1C
:104D00003568696801292DD9AA684B1ED05C0A282C
:104D100028D1002B01DC1C0009E0581E145C0A2C71
:104D2000F9D00300F5E7105D202802D10134A1423B
:104D3000F9D8002B0BDD601C814208D1581E0028D9
:104D400005D00138175C0A2F0CD0202FF7D052184D
:104D5000023AE31A14789B083A3C624254411C1907
:104D6000002C00D1F8BD084F04223900280022F0A1
:104D7000AEF90421380004F0EDFC3369013C043342
:104D80003361EDE7142A0020DB6F030010B5202209
:104D90000021024824F019F810BDC046DC2E002086
:104DA000084B10B5426818600020986018750138EB
:104DB000D86008005A601A6199611EF07DFCFFF707
:104DC0009DFF10BD142A0020F8B503780400002BC5
:104DD0001ED0104D286E002804D0210024F03FF88A
:104DE000002815D0200024F044F8471C380021F09A
:104DF0006DFA061E0CD03A00210023F0CAFF2A00EB
:104E0000054B5C321968043B99609342FAD12E66D7
:104E1000F8BDC0467C2E0020F42E0020F0B5B84C22
:104E200002002068A568436885B00193002D00D07A
:104E3000FDE0531E042B11D8636801998B4200D109
:104E400095E0012A00D12AE1022A07D1236962688C
:104E5000934200D94FE10122524288E0032A00D157
:104E600085E0042A00D12FE1052A00D107E1062AB6
:104E70000ED12369019A9342AD416D42002DEADDC6
:104E80002368290098682369C01804F063FC1FE0B8
:104E90000B2A21D1019B2269991A22F0D8F92368A3
:104EA000019A5B68934204D213002269981A04F0B5
:104EB00087FC2268236951689068C91AC01804F0F9
:104EC00049FC236858682369C01A401B04F066FC3B
:104ED00023695D192561BEE70E2A13D1E368002B13
:104EE000B9DB013BE3606268019B991A22F0AFF9DC
:104EF000E368002B18DB1633824A9B00D3189968AD
:104F000020680FE0102A16D1E368062BA3DC5D1C95
:104F10007C4A17339B00D318996800299BD063689B
:104F2000E560436022F058F963682269D61A226866
:104F30005568ED1A0AE0152A0CD123696268616888
:104F40009A1A22F08CF9236962689E1A0127002EB2
:104F50002FDCA4E70D2A0DD16B481EF0ADFB2068B5
:104F600022F01FF96368C018FFF72EFF002210001F
:104F700005B0F0BD01231B2A62D0082A01D07F2A88
:104F800020D121696268914200D864E700238668D5
:104F9000B618F75C202F13D101339F18B942F8D807
:104FA0000426032B00DC033E891B320022F057F954
:104FB0000127300004F0F2FB23699E1B266178E094
:104FC0000126F1E7092A28D1636822698068D11A8D
:104FD000C0184E4A03AB02F025FB061E00D13AE78B
:104FE0000027431C0BD1A0691EF066FB6368226991
:104FF000D11A22689068C01804F0ACFB4FE723690F
:105000002068F918039B01375A1C03921A7822F082
:105010000CF9BE42F3D1350041E71300203B5E2B73
:1050200000D918E7216922F009F9012537E7012D98
:1050300008D104234F2A03D002235B2A00D0002387
:10504000A36008E7022D20D11300303B092B03D8C1
:1050500003232275A360FEE60023A360412A00D14A
:1050600052E7422A00D139E7432A00D101E7442A16
:1050700000D1EBE6482A12D0462A00D0EBE6002702
:10508000019B22693E009D1A0EE00021032D29D1CB
:105090007E2A24D1237D312B01D0372B0DD1002541
:1050A0002F00236962689E1A0023A3609E4200DDE0
:1050B0007FE7002F00D1E1E6F1E61A00FB25343A44
:1050C0002A42DCD0332B0AD12169019B994206D2B6
:1050D000012222F0C4F8002501272E00E4E7002574
:1050E0002F00FAE7042D04D1462AC8D0482AD6D08A
:1050F000A5E7A160AFE6002501262F0059E7C046CD
:10510000142A00207C2E0020DC3F030084E80200EB
:10511000044B88600B60044B08004B600023CB609D
:105120007047C0466C980200352C020013B504008D
:10513000080001A9FBF746FF002C03D0012C07D083
:10514000002004E0019B0548002B00D1044816BD57
:1051500001991EF0CBF840002043F8E7CCE70200AD
:10516000C4E70200F0B585B00400080003A91500EB
:10517000FBF728FF0600002D07D10300039A2F49F3
:10518000200021F047FE05B0F0BD039B0200C318CC
:10519000002101200193019B934206D82727002973
:1051A00000D0053F3A0026491AE01378272B08D093
:1051B000223B5D426B41DBB20132002BEBD0272753
:1051C000F0E700230100F7E730001EF05CF805006F
:1051D00030001EF073F80600AF4205D13A001949BD
:1051E000200021F017FE14E017495C2D0ED02B0093
:1051F000203B5E2B01D82A00D5E714490A2D05D0A3
:1052000013490D2D02D0092D0CD11249200021F097
:1052100040FD019BB342D7D83A000949200021F054
:10522000F9FDB0E7FF2D02D82A000B49D8E70B4B58
:105230002A000B499D42D3D90A49D1E70301030053
:105240008200030081000300850003008800030042
:105250008B0003008E00030091000300FFFF00009D
:10526000080903000F090300F7B51E0008AB1D78FD
:10527000294B0C001700984206D12B003200390050
:10528000FDF7D4FC2018FEBDF30715D57610019666
:10529000019BE219002B2ADA00213F260127501E2C
:1052A000A04219D2002900D001932000002DEAD19C
:1052B0001A491B481FF0BEFB01A93000FDF71CFC7A
:1052C0000028E5D130001DF0B2F916490200164859
:1052D00003F0E8F807F002FA0278B243802A01D01E
:1052E00039000133421E002BCDD01000D8E720003A
:1052F000012600243F27904204D3002C00D00193C4
:105300001000D3E7013BBED3340001300178B9432C
:105310008029F0D10130F9E7A0920200EE080300E5
:1053200084A90200C608030090AC0200F0B587B063
:1053300004000E001700FDF7B9FA02A905002000CD
:10534000FBF740FE0400042F4ED1B30734D1274BA6
:1053500032689A4230D105AB04AA03A930001DF08F
:105360009EFE059B224FBB4204D0032B02D0214856
:1053700008F01EFA039B2600BB4207D00122210041
:1053800000922800029AFFF76FFF0600029A049B22
:10539000A118BB4206D00121280000912100FFF78F
:1053A00063FF01000E208E4204D88A1B28003100C2
:1053B0001CF0F6FF07B0F0BD0023029A0093210015
:1053C00033002800FFF750FF0278012153B2002B71
:1053D00006DA4023012101E001315B081342FBD1D1
:1053E0000122FBF7B5FDE5E70020E3E7E8A40200B2
:1053F000E4B30200A6FC020010B504000C2020F06B
:1054000058FF034B4460036001235B42836010BD7F
:10541000089B020001220020074B08495A600860DF
:10542000A821DA60064AC9005A5006495A50043188
:105430005A5005495A50704700A000400CAC00403B
:10544000FCFF0000440500004C050000034B04482D
:105450001B78002B00D103487047C046CD2D00209B
:10546000CCE70200C4E70200F8B5A826324A334B65
:10547000F600196813680420CB18C9181160304A67
:105480008C4612781B11170009112E4A2E4C2F4DF5
:10549000002F48D0002B3ADA9051C31AA920C0003F
:1054A000135081239B00002937DA591A13515151A7
:1054B0000123274CD3602378002B22D03F2225489C
:1054C000254B01688C331B6801310A409D5C1C4BE5
:1054D0001B78002B01D0803D6D001C2302606246CA
:1054E0006B4308339B1A154A9B1013601F23194006
:1054F00007D11A4B1A78002A03D01948197009F0FD
:1055000069FA01232278042053402370F8BDA927AB
:105510000433FF00D0519351C3E7535181239B00C3
:10552000C9181151C4E7043390515351A920812364
:10553000C0009B001350F3E7302A0020402A0020CF
:10554000D800002000A000404C05000044050000E9
:10555000CC2D0020342A00207C2E0020D9000020F1
:10556000F32C020030B585B001220400080001A927
:10557000FDF73EFC029A202A00D920220023019D3B
:10558000934204D0E85CE11808710133F8E7014860
:1055900005B030BDE4B3020070B50400080015008A
:1055A000FDF76CFA1F2802D90C4807F00FFF002DF9
:1055B00002D10B4808F0CEF82418042D04D10120A4
:1055C00023795B00184370BD2800FDF757FAFF28C8
:1055D00001D90448E9E720710348F4E748090300CA
:1055E0005C09030079FC0200E4B302000123A0225D
:1055F000834010B5134CD20513510300C133124C34
:10560000FF339B009C50114B8900C918A223DB007B
:10561000CA580F4C00022240CA50F82252011040D2
:10562000C022CC589202224310430322C850CC58C7
:10563000084822432043C850C046C046C046CA500E
:1056400010BDC0460C0500000303000000600040D0
:10565000FFE0ECFF031F0000A0221E21114BD2002F
:1056600070B59C58104D8C439C50A324E4001D51F0
:105670000E4C0F4D0F4E5C5104355E510E4D8000A7
:105680005C51A5240D4DE4001D51084C0C4D001932
:105690000C4C185104341D510B4C185198580143AF
:1056A000995070BD00F0014040A1004000600040F2
:1056B0001C05000044A100402405000048A1004052
:1056C0004CA100402C0500003405000010B504007A
:1056D0000A4903F0F5FB0A4BA0211C600123607905
:1056E000084A8340C9058B500021FFF77FFF002047
:1056F000FFF7B2FF0022044B1A7010BD18B202006F
:10570000382A00200C050000D800002070B50D00DC
:105710000400134E2800310003F0D2FB31002000BA
:1057200003F0CEFB0F4BA0221C600F4BD2051D6077
:10573000607901242100814026000C4BD150697909
:105740008E400021D650FFF751FF68792100FFF706
:105750004DFF2000FFF780FF054B1C7070BDC04659
:1057600018B20200382A00203C2A00200C05000054
:10577000D8000020F8B50025FFF74CFE214B28008B
:1057800090331D6009F0F4F8A0221E201E4B1F4923
:105790001D701F4BD2001D601E4B1F4C1D608B588F
:1057A0001E4F83438B50A223DB00E2581C4E3A402D
:1057B000E250E2581B493243E2500122E5501A4BB5
:1057C000186843799A401300A022D205535003F081
:1057D00061FB164B1B78AB4213D0154B1149E258B5
:1057E0001740E750E25816430122E650E550114BAE
:1057F000186843799A401300A022D205535003F051
:1058000049FBF8BD7C2E0020CD2D002000F001408A
:10581000302A0020402A002000600040FFE0ECFF1A
:10582000001F03000C050000382A0020D8000020CB
:10583000140500003C2A0020F0B53E4E8DB0330028
:1058400090331B680500002B03D1FFF793FF0DB0C9
:10585000F0BD002801D008F097FA684606F018FF5E
:10586000002822D133009033186807F0B9F90400FA
:1058700006F02CFF002D01D008F090FA2E4B2022CC
:105880001D6833006D118C3301356D011B681540A7
:105890005D19002C2DD1903621002800346023F0B2
:1058A00094FA0122254B1A70D1E7002D01D008F09F
:1058B00075FA019B2249186806F00EFA00240500CB
:1058C000A042DBD1019F3800FCF7F0FF1D4B98424E
:1058D0000BD12900012000F0CDFE2A000400F86061
:1058E0001F211948FBF734FBA060019B0024B3641F
:1058F000C4E72000FCF7DAFF144B984209D03300CC
:1059000000229033124913481A601DF08BFCB064DA
:105910009DE763682B60A3686B60E368AB602369F5
:10592000EB6063692B61A3696B61E369AB61236A17
:10593000EB61B6E77C2E0020342A0020D90000203D
:10594000DCAB020074AA020016090300EC9B020003
:105950003609030090AC020010B5FFF70BFF0148B9
:1059600010BDC046E4B30200F0B589B00493734B98
:1059700003901B780E001500002B01D0FFF7FAFEF4
:105980006F4C8C342368002B06D16D4A4020903236
:10599000136020F08EFC206080226A4BD200DA6710
:1059A0000122694C694BE250FFF734FD0023684A3D
:1059B000F021A3500432A3500832A350C22209039D
:1059C0009200A150634F093AFF3AA3500594BE429A
:1059D00000D0A3E0B54200D09DE05F4D07AC2800A9
:1059E00003F062FA002805D001235C4928002370E7
:1059F00003F066FA5A4D280003F056FA002805D045
:105A0000012356492800637003F05AFA554D2800C7
:105A100003F04AFA002805D0012350492800A3705A
:105A200003F04EFA002307AA5F1C9B5C002B39D0C1
:105A30004D4ABB00043BD458A02203213D006379AA
:105A4000D205C133FF339B00995007ABEB5C002BB1
:105A500026D00426444BAA00D3580193012263792F
:105A6000A0219A40A123C905DB00CA50019B053340
:105A7000180002931DF01DF9012811D16379A021AE
:105A800098403A4BC905C85002981DF012F90028F9
:105A900006D1013E002EE1D1019949E00225D4E76B
:105AA000022DFBD10123022FBDD12B4801F0BEFCFA
:105AB000FFF70CFE0021039807F058F80025012499
:105AC0003F221F4B802190331860294B1D70294BBA
:105AD0001C70294B1A601A4B12198C33186823F06A
:105AE00074F92800FFF7A8FE244B144E1C60059B98
:105AF00050221C6022492800347008F005FF049BE6
:105B0000AB4219D00E4B3278002A15D09A6C002A7D
:105B100012D120BFF7E71B4807F01CFE300001F050
:105B200085FC0400BD42C3D0280001F07FFC0100C9
:105B30002000FFF7EBFDBDE709B0F0BDCD2D002043
:105B40007C2E002004E100E000A00040FC0F0000DB
:105B500004050000E4B30200ACA20200E8B10200B8
:105B6000F4A2020004A30200B89B02000C0500008E
:105B7000CC2D0020D9000020342A00200CAC00409D
:105B8000695400008109030010B5084B86B002ACCF
:105B90000093019404230CF0BFFB02982379E26880
:105BA000A168FFF7E1FE024806B010BDC49B0200E9
:105BB000E4B30200014B1878C0B27047CD2D00202D
:105BC00010B5242020F075FB0400044B202208C0EF
:105BD000802123F0FAF8200010BDC046EC9B0200A3
:105BE000F8B5070008000D001600FCF75FFE304B0B
:105BF00098425BD1781F0F2858D814F085F8080810
:105C00003257575757575757575757303055FFF751
:105C1000D7FF04230400EA5CE2540133242BFAD1B9
:105C20003000FCF743FE224B98423FD10121052F63
:105C300002D0122F00D002390422FF20B35CA55CF1
:105C4000803B4B435B19FF2B03D90500DB179D43BA
:105C50002B00A3540132242AF0D12000F8BD2C00DF
:105C6000DEE7FFF7ADFF04230400EA5CE2540133F2
:105C7000242BFAD13000FCF765FF0F211DF03EF810
:105C80002100FF25221D24311378803B4343DB1381
:105C90008033FF2B03D92E00DB179E433300137094
:105CA00001329142F0D1D8E72C00E3E70024D4E799
:105CB000EC9B0200F0B585B00C00FBF76BF903AA72
:105CC000070002A92000FCF77BFF029E039B350022
:105CD0001035AD002800019320F0EBFA04002C22CF
:105CE0001030002123F071F867602700104BE66345
:105CF0002360104B019EA3600F4B403DE3600F4BB0
:105D0000403763610E4B7519A3610E4BE3610E4B77
:105D100023620E4B63620E4B6363AE4202D12000DE
:105D200005B0F0BD01CEFBF735F901C7F5E7C04678
:105D300058B80200555D0000B55D0000196600000E
:105D4000B1660000795D0000B1670000A565000044
:105D50004CA0020070B50C0005000B6805495A689C
:105D600021F058F821682800403122000CF08CF90D
:105D700070BDC046C43B0300136870B5002B10D142
:105D80000568EE6BB34200D170BD9C002C19246CE9
:105D9000A14201D00133F5E702339B001B58136089
:105DA000F2E7024902481EF045FEC046A30903007F
:105DB000E0A70200F0B51700C26B85B0CE19050050
:105DC00001910393964206D033002549254802F0FD
:105DD00069FB06F083FC0021300000F04BFC04005E
:105DE000019B05609B001A0003990830029322F082
:105DF000D0FF0298BA0008302018002122F0E5FFF9
:105E0000029A039B94466344F7191E00019BBB4210
:105E100002D3200005B0F0BD3068FBF7BBF80021CD
:105E20000200EB6B0293029B994204D10E490D488C
:105E300002F038FBCDE78B00E818006C824201D0FD
:105E40000131F0E7E3189968002901D00749EEE72E
:105E5000726808369A60019B02330193D6E7C04608
:105E6000B407030090AC02001C080300ED07030018
:105E7000014B58687047C0467C2E0020014B1868C3
:105E80007047C0467C2E0020F0B5194E87B03368AD
:105E9000050000200C0001931FF0B5FC306000905D
:105EA00020681EF07CFD019B07003360114E022D1F
:105EB00003D0A068FCF7FAFC0600210063680831F3
:105EC000A81E039300F0D6FB009B049005930022CC
:105ED00003AB0321300006F053FD074B04009F4243
:105EE00003D0010038001FF07DFB200007B0F0BD9B
:105EF0007C2E002058B80200E4B302001FB56946AA
:105F000006F034FE0400200006F092FE002802D1C4
:105F1000044804B010BDFCF7EFFE0028F3D102489E
:105F2000F7E7C046CCE70200C4E702001FB56946A8
:105F300006F01CFE0400200006F07AFE002802D1C4
:105F4000044804B010BDFCF7D7FE0028F3D0024887
:105F5000F7E7C046C4E70200CCE7020010B5FCF743
:105F600029FD034B002800D1024B180010BDC0468C
:105F7000CCE70200C4E7020037B5FCF77FFD01ABB8
:105F80007F2806D80121187001221800FAF7E0FFD7
:105F90003EBD1E49820988420BD8402149420A432E
:105FA0001A703F2202408020404210435870423114
:105FB000EAE7174C010BA0420ED82024644221438B
:105FC000197080215F344942224020400A43014336
:105FD00099705A700321D7E70E4CA04212D81024B2
:105FE000850C64422C431C703F2580242940644268
:105FF0002A40284021432243204359709A70D87088
:106000000421C1E7044807F0E1F9C046FF0700009A
:10601000FFFF0000FFFF1000B7090300F0B589B0D3
:10602000019204000D0000222F490198029302F012
:10603000A3FD0090002801D043680093012C16D0E6
:10604000A4002B19002427000193019B9D4224D01A
:10605000009B2E68002B04D0310018001EF0A6FC17
:106060000600002C37D137002C680435EDE70024FA
:1060700004A9286806F07AFD27000390039806F02B
:10608000D7FD051E0CD1002C07D12200174901981D
:1060900002F072FD00281BD04468200009B0F0BD5A
:1060A000009B2E00002B04D0290018001EF07EFC5F
:1060B0000600002C09D03A003100029807F08EF952
:1060C0000B4B984201D025003E002C003700D5E74D
:1060D000084807F07BF93A003100029807F07EF992
:1060E000034B9842C1D1BEE7561300002E110000A9
:1060F000CCE70200D809030037B501A90500FBF77A
:106100007FFB1E4B04002B40062B05D0AB072AD18A
:106110001B4B2A689A4226D1019920001DF0E6F80F
:106120000190012822D1207843B2002B04DB01200A
:1061300023785B0018433EBD7F23013418403F3B6A
:10614000034208D13F22237819009143802905D0CA
:106150001FF0B6FAEFE798435B10F1E780011340B8
:1061600001341843EFE7019B012BE0D0019A054968
:10617000054802F097F906F0B1FAC046070080FF23
:106180000C9A0200F109030090AC0200F0B5140073
:1061900087B00290039100222349200002F0ECFC1A
:1061A000002205002149200002F0E6FC0123040042
:1061B000049305931E4F002D07D068681D4B98422D
:1061C00003D004A9FBF71CFB07001B4E002C07D0D3
:1061D0006068184B984203D005A9FBF711FB060035
:1061E0000024029B154D9C420AD10023059A01937D
:1061F0000093310028000EF0BBFD0E4807B0F0BD43
:10620000002C07D00023049A019300933900280042
:106210000EF0AEFD0399A3000022C9582800FCF738
:106220005DFB0134DDE7C0468E15000096110000CD
:10623000DE6F0300E4B30200654F030084E8020050
:1062400010B5040086B06A4602A810210FF0D8FDF0
:10625000012221006846FCF741FB02A90248FAF737
:1062600041FE06B010BDC0460C9A020070B50C6825
:10627000E30726D4A30703D1174B22689A4220D004
:10628000012820D94868FCF7F9FB06002000FCF73C
:1062900059FC051C300014F0D1FE011C0F4817F00A
:1062A0008DFB011C041C281C14F09CFB16F0F6FF4F
:1062B000211C14F0BFF9032302249843084B044324
:1062C000E418200070BD2000FCF73CFC16F0E6FF4F
:1062D00006F056F80400F4E72CB902000000204153
:1062E0000000808030B50B0085B01400012802D971
:1062F000094807F02FFA09480121C2680192019D5F
:106300000022A8472200039003A901200DF0C4FF3A
:10631000039805B030BDC046450A030088E7020077
:1063200013B504000800FAF735FE6A4601002000A4
:1063300006F09EFB009B0248002B00D1014816BDD1
:10634000CCE70200C4E7020037B50024022800D9D8
:106350008C6848680D68FAF71DFE0A4B0100002C96
:1063600000D0094B6A4628009847009B002B07D0B5
:1063700001991C00002903D01800FCF703FF04005A
:1063800020003EBDD5CA000071CA000070B50400EF
:1063900008001500FAF7FEFD2A000100200006F0B3
:1063A000C1FB014870BDC046E4B30200F8B5032646
:1063B000050007003540022D16D10E4B0340062B79
:1063C00012D0FF23DB05C418B443201C002113F0B6
:1063D00075FE002806D080231B06E418B443064B44
:1063E0002C43E7183800F8BD380009F069FA0700B7
:1063F000F8E7C046070080FF000080807FB50B00F3
:10640000012803D100211868FCF782FA102102A8A4
:1064100020F079FE0C4902A81CF002FC032804D1EC
:106420000A481CF0F2FE06F059F9039B0193002B79
:1064300003D1042801D10648F3E702A90548FAF779
:1064400051FD07B000BDC0463B830300FCA902001C
:1064500058A802000C9A020010B506F0C1FB0028F3
:1064600004D103481CF0D1FE06F038F910BDC04637
:10647000DCAB020010B5022803D0054905481EF028
:10648000D9FA4A680B20096806F0A8FF10BDC0467B
:106490002B0A0300ECAA02007FB50D4D0400A842B0
:1064A00013D00C4E012201003000FCF717FA0A4904
:1064B000300020F0EEFB04230293084B0394DB69C9
:1064C00002AA0321064801939847280004B070BD32
:1064D000E4B3020084E80200654F030098B10200B3
:1064E0005C9D0200F8B50E0000280FD10400284B77
:1064F0001D680021080020F0B3FA00270600BD4205
:1065000032D10025AC423ED13000F8BD0868830787
:1065100014D103681F4A93420DD11CF087FF050078
:106520003068FCF7C3F91C4BC26800249A42E0D1E2
:1065300034680434DDE7194A934201D0FCF7B6F918
:10654000856B002DECD0164B2A689A42E8D00025C6
:10655000E6E7EA68FB009958002904D0042902D034
:1065600030000DF039FE0137AB68BB42F1D8C8E707
:10657000A268EB009958002904D0042902D0300009
:106580000DF02AFE01356368AB42F1D8BCE7C04686
:106590007C2E002098B102007DB6000058B80200A1
:1065A00074C20200044B88600B60044B08004B600F
:1065B0000023CB607047C0466C980200E72D0200B4
:1065C00070B50E0010490400002520F062FB7368CE
:1065D000AB420AD8012B03D10C49200020F059FB13
:1065E0000B49200020F055FB70BD002D03D0094958
:1065F000200020F04EFBAB00F31801229968200028
:10660000FCF76CF90135E2E7E20D0300700A0300C4
:10661000A002030045FC020070B50D0001281ED049
:10662000002803D0022807D0002004E04B680E4861
:10663000002B00D10D4870BD00260D4C6B689E42AA
:1066400003D3012064002043F5E7B300EB189968F9
:10665000022006F023F9401024180136EEE74B68BB
:106660005B001843E7E7C046CCE70200C4E702003E
:1066700044A0020070B506000D000B48002E0DD09E
:10668000B41CA40020001FF014FE084B46600360F9
:10669000002D03D00023083CA34200D170BDE9586F
:1066A000C21891600433F7E744A002004CA0020036
:1066B000F0B5070085B00E0014001D2803D9002591
:1066C000280005B0F0BD01238340324D1D4044D168
:1066D000314A13421FD1F82292051342EFD0200015
:1066E000FCF7E4F82D4B426A9A4205D020002C4971
:1066F0001EF0F8F8041E0CD0230031006268083345
:1067000000920831726838000BF02AF9254D0028F4
:10671000D6D1254DD4E72000FCF7C8F8204905F074
:10672000DBFA0028CBD07368626829009818FFF75D
:10673000A1FF07003100736808379A00050008318F
:10674000380022F026FB210070686368800038184A
:106750009A00083122F01DFBB2E703A91000FCF7F4
:10676000CBF90025A842ABD00398104D0028A7DD37
:10677000736800215843FFF77DFF05002B003000B0
:10678000083300930830039B726804211FF031FA2C
:1067900096E7C0468000100020000400A5650000B8
:1067A0004CA00200CCE70200C4E7020044A00200B3
:1067B00030B5040085B0042A2DD1032540680D4072
:1067C0001FD1164B0A689A421BD101AA0BF04CF854
:1067D000002802D1124806F0EBFF019B0298290025
:1067E000C01AFFF747FF050021006B6808319A00C7
:1067F000019B08309C00091922F0CBFA280005B053
:1068000030BD0A00002301002068FCF70FFA0230B7
:1068100080000559F2E70025F0E7C046E8A4020031
:10682000A6FC0200F0B50C001100002285B01E008D
:106830000092012320000BF03FFD184D002C1ED0CC
:106840003568AB0703D1164B2A689A4217D010203F
:106850001FF02FFD00210400306806F087F90025A5
:1068600004260390039806F0E3F9071E0AD12800D6
:106870002100FFF7FFFE050020001FF049FD280062
:1068800005B0F0BDAE4205D8F10020001FF02FFD8D
:1068900004007600AB001F510135E3E744A002007D
:1068A0004CA002000022104B10491A600300123362
:1068B000FF3341185A701A7004338B42FAD1010029
:1068C0000300002209310833FF311A709A705A70A0
:1068D000DA7004338B42F8D1C3237F229B00C25469
:1068E000034B044A1A607047442A00201103000039
:1068F00004000020720A0300F0B500267E24320056
:1069000031009300C318FF335F7C7F2F4CD09B7CFA
:10691000F618F6B2531CDBB2EF2E2AD9C1267D251C
:10692000B60086193700AC469C4516DA9B00C318A2
:10693000FF3359749974D97419757D230232D2B218
:10694000934211DA9300C318FF335C749974D974BD
:10695000197500260132D2B2D3E73D68043FBD600D
:1069600001256D42AC44DFE73568013B7560043EAC
:10697000E6E77D2FEED80D4DEF5D01252F42E9D0E2
:10698000C1227D26920082189E4208DA9A0082185F
:10699000FF3254749174D17411751A00D9E71568D7
:1069A000013E5560043AEFE7F0BDC046550B0300C9
:1069B00070B5002140250D4C8B00C318FF335A7C65
:1069C0007F2A11D0A25C0131C9B22A42F4D05A7D8B
:1069D0007F2AF1D0A25C7F2AEED9DA7D56B2002E52
:1069E000EADD0132DA74E7E770BDC046040B03004C
:1069F0000300F7B500214B4A1333FF338218197097
:106A000004339A42FBD1FC2300249C462200844498
:106A100053B2002B04DA444B444A1A60002008E0C9
:106A200063461F69BC4205D37F234432920013544E
:106A30000120FEBDDE68355D602D01D9203DEDB23F
:106A4000611CC9B28F4251D0735C602B01D9203BCD
:106A5000DBB2232D4DD1303B092B02D9324B344AC6
:106A6000DBE70234E1B28F4204D8FF2BF6D8437043
:106A70000C00CDE7745C2500303D092DF5D80A25C2
:106A80006B430131303BE318C9B2ECE70136512EBC
:106A900030D10023274C1F5DDEB22A2F0CD1264FA8
:106AA000FF5CAF4208D19300C318FF335E74447893
:106AB00001321C75D2B2DBE70133512BEBD11F4CF5
:106AC000493B08342678AE4208D0013C002B02D165
:106AD000154B1B4AA1E7013BDBB2F3E7002BF7D0D4
:106AE00014004334A4000419A370C1E7232DB5D0CA
:106AF00000230026F7B201970F4FF75DAF42C5D1D3
:106B00000C4FF75D2A2FC1D09F42BFD1930001994E
:106B1000C318FF3359744178013202341975D2B267
:106B2000E1B2A5E71203000004000020750A03008B
:106B3000870A0300940C0300430C0300E50C0300D8
:106B4000950A030010B51130084A0949FF3003784F
:106B50007F2B00D110BD02240457002C03DCCB5C3A
:106B600043700430F3E7D35CFAE7C046F30B03004D
:106B7000A30B0300F0B50023070085B09E00BE19EB
:106B80003100FF314A7C9C467F2A01D105B0F0BD1F
:106B90004F4B02209C5C63460133DBB20442EDD0D4
:106BA000012560462C4242D15419E0B20090494878
:106BB0007C35801840780190C87C097D0290039153
:106BC000C1218900791808009D4226DA9B000098AF
:106BD000FB18FF3358740198941C98740298E4B21F
:106BE000D874039818753B48634682183000FF300C
:106BF0009578027D023300927D22C67CDBB29A42F8
:106C000010DA9B00FB18FF335C749D74DE74009AED
:106C10001A7563460333DBB2B0E70468013D446094
:106C20000438D1E70868013A48600439E7E70130E1
:106C3000C0B2010044318900C95D0029F7D07F2925
:106C400008D008242248405C204297D124390129E9
:106C500000D893E73000511CC9B200911D49FF30A4
:106C6000891849787D250191C17C0291017D0391AC
:106C7000C121890079180C009D421FDA9B00009CFD
:106C8000FB18FF335C74019C124D9C74029CDC74F5
:106C9000039C1C75941CAA1863469678027D0233E7
:106CA00000927D22C57CDBB2E4B29A420BDA9B00F3
:106CB000FB18FF335C749E74DD74A8E72668013D01
:106CC0006660043CD8E70868013A48600439ECE79C
:106CD000040B0300A30B0300F7B500229300C318B5
:106CE000FF335C7C002C03D10132D1B20A00F5E7FE
:106CF0007F2C00D126E1102693490D5D511CC9B2AD
:106D0000354227D0DC7CAD06ED0FA4462C00C12512
:106D10001434AD001F7D019445196D368E4214DA8E
:106D20008D00019C4519FF356C740024AC746446D9
:106D30002F75EC745C7C352C00D0C5E05A7B834CFD
:106D4000A25C5207D2D5102285E02C68013E6C600F
:106D5000043DE3E74E2C1CD118220D24DD7C5C742D
:106D60001E7DC1239B00C31870348C420CDA8B004B
:106D7000C318FF335A740022DD749A741E75B5E788
:106D80001B22EAE71C22E8E71F68013C5F60043B26
:106D9000EBE74F2CF4D0502CF4D06DB2002D2BDA51
:106DA000DD7C002D28D00D004435AD002D5C002D7C
:106DB00022D1961CF5B20195AD004519FF356F7CC7
:106DC0007F2F19D0604EF75D7F2F15D9EF7C002FF4
:106DD00012D0C1237D229B00C318019C944206DD82
:106DE0001F236B740023AB74EB742B757EE71C6858
:106DF000013A5C60043BF0E7172C2ED15C7B013A32
:106E0000D2B2452C1DD11B3C5C7315004335AD003F
:106E10004D4C2D5C655D7F2D00D867E70132D2B205
:106E200092008218FF32557C002D00D180E0645D15
:106E30007F2C00D85AE7D27C002A00D056E71E32B9
:106E400009E0392C01D10D3CDEE73F4A125D7F2A73
:106E500000D84BE712225A7448E7182C07D15A7B06
:106E6000394CA25C7F2A00D840E71322F3E7202C9C
:106E700005D15A7B3C2A00D038E7163AEBE7482C7C
:106E800015D15C7D7F2C02D14B245C7403E02E4D28
:106E90002C5DA406F8D55C7C2B4D2D5DED0700D450
:106EA00048E75D7B202D3CD10C3C5C741EE73C2CFC
:106EB000F1D15A7D7F2A00D118E7234CA25C9206BB
:106EC00000D513E73F22C6E72A2C16D1DA7C1C7DB9
:106ED000C1237D259B00C3188D4209DA2B258B0029
:106EE000C318FF335D740025DA749D741C75FDE6CC
:106EF0001E68013D5E60043BEEE72C2C11D1DA7C6C
:106F00001C7DC1237D259B00C3188D4204DA8B00B4
:106F1000C318FF332D25E5E71E68013D5E60043B85
:106F2000F3E7452C00D170E7392C00D0DEE66CE7A2
:106F3000527D7F2A00D1D9E6A25C7F2A00D8D5E60F
:106F40001E2288E7F7BDC046040B0300550B030063
:106F5000F0B50022060085B0130044339B009B5D12
:106F60007F2B31D05B4CE35CDB072AD51300511E2D
:106F7000C9B244318900584F7118013BDBB2002B74
:106F800023D008787F2803D0385C04397F28F4D9CF
:106F900099007118FF31487C7F280ED02027255C8E
:106FA0003D4204D04C4D285C0425284205D0887C05
:106FB0004508AC460130604488740133DBB293422B
:106FC000E6D10132D2B2C7E70023022712E06B07F5
:106FD00008D4EB070DD56246FF32937CD9085B1AC3
:106FE000937406E0039B039A9B7B99080133CB18AB
:106FF0009373029B9A00B2181100FF3194464A7CA9
:107000007F2A64D034485D1C845CEDB2029565B281
:10701000002D21DA029A9200B218FF320392527CBC
:107020000192855C019C2A0041257F2C00D015002F
:1070300040242242CBD1019C123C012CD9D84022C1
:107040000233DBB244339B009B5DC35C1342D0D060
:107050008B7C013B8B74CCE71E4DAA5C08252A4231
:107060000ED0029B9B00F318FF335A7C7F2AC0D0BE
:10707000825C3A42BDD006229A7405229A73B8E720
:107080003C421AD00133DBB21A0044329200925DC6
:10709000002AF7D07F2AACD00F498A5C3A42A8D0A8
:1070A0009B00F318FF339A7C520801329A746246AF
:1070B000FF32937C5B08013392E710231A4298D089
:1070C0004B7BC35C3B4294D08B7C023BC2E705B058
:1070D000F0BDC046550B0300040B030070B504005F
:1070E000FFF7E0FB2000FFF783FC23000022FC33C6
:1070F000DA601A61904226D02500224E113533689D
:10710000FF35934203D029001F4806F079FB200089
:10711000FFF7E2FD2000FFF74BFC2000FFF712FD18
:107120002000FFF715FF2000FFF724FDC4222B00ED
:107130009200A1181A78502A06D97F2A07D0002079
:10714000124B134A1A6070BD04338B42F2D133687C
:10715000002B02D00F4819F07DFC2000FFF7CCFB7C
:107160003368002B03D029000B4806F049FB2000B0
:107170001BF066FE054B0949186821F070FE43427A
:107180005841E0E7582A0020AC0A03000400002020
:10719000BB0A0300E10A0300F10A0300720A0300BC
:1071A00070B504000800FBF769FC0500431002D02D
:1071B0000F4806F00BF90F49200001F081FE00286E
:1071C00007D0A02203216379D205C133FF339B008E
:1071D0009950012362799340A022D205002D04D05A
:1071E000A121C9000448535070BD0449FAE7C046C4
:1071F0003B0D0300F8B10200E4B302000C050000EF
:1072000070B505000800FBF739FC0B2303410400AF
:10721000DB0702D4094806F0D9F82800084901F034
:107220004FFEFF22A40092001440A0226B79D205E9
:10723000C133FF339B0003489C5070BD0D0D03000C
:10724000F0B10200E4B3020010B50C49040001F0F3
:1072500037FEA022D205002805D004216379C1336E
:10726000FF339B00D150A223DB00D0586379D84074
:10727000012318401EF024FA10BDC046F0B10200F0
:1072800010B5040001F0E8FD0A4B984205D00A4B06
:10729000984202D0200001F0EDFDA0226379D205D2
:1072A000C133FF339B0098580007800F1EF008FA87
:1072B00010BDC046F0B1020008B20200032370B551
:1072C0000B4004000800022B14D1194B0B40062B75
:1072D00010D0FBF737FC15F08BFC0022154B13F098
:1072E00037FF15F015FC144B0500984205D91348DB
:1072F00006F06CF8FBF7C2FBF5E71149200001F03E
:10730000DFFD002807D0A02203216379D205C13315
:10731000FF339B0099506079290006F0B5FB002DE2
:1073200003D10849200001F0CBFD074870BDC046DD
:10733000070080FF0000E03FFF0300001A0D03007C
:1073400038B20200E8B10200E4B3020013B50A4902
:10735000040001F0B5FD05216846615611F084FD79
:10736000684611F0A7FDA0230021044ADB00D1509C
:107370001EF0A6F916BDC046E8B10200007000403C
:1073800010B50800FBF77AFBFA239B00584306F080
:1073900057FB002802D0024806F018F8014810BD3B
:1073A000FE0C0300E4B3020010B50800FBF766FB17
:1073B00006F046FB002802D0024806F007F8024813
:1073C00010BDC046FE0C0300E4B3020010B504007B
:1073D00001F042FD0C4988420DD00C4B98420AD076
:1073E000200001F06DFDA02200216379D205C13398
:1073F000FF339B009950200007F0BCF9044B002894
:1074000000D0044B180010BD20B2020008B20200E8
:10741000CCE70200C4E70200A0230C220249DB05EE
:107420005A5024315A5070474407000010B50400E8
:10743000FBF73CFA064B984208D0064B984205D021
:10744000054B984202D0054806F084F9200010BD93
:107450007CA3020034A2020070A20200EE0C030022
:10746000F0B50D00002785B0110003901E00280024
:10747000104B022200970AF01FFFAB1C9B00180064
:1074800002931EF016FF0400039B013D036045605C
:107490003368029D8360083D0437BD4202D120005D
:1074A00005B0F0BD0021F05905F060FBE3199860CC
:1074B000F2E7C046FFFF0000F7B503780400002B99
:1074C0001FD0402B20D101230193002304221E0052
:1074D0001D00190094462278002A3ED1013200296D
:1074E00010DC002D0EDC002E0CDC033B934209D98E
:1074F000013C23785C2B05D00199002901D00A2B8F
:1075000000D100221000FEBD3F491BF0FAFC00280C
:10751000D9D13E4920001BF0F4FC0028D3D13C49CE
:1075200020001BF0EEFC0028CDD13A4920001BF0D2
:10753000E8FC0028C7D1384920001BF0E2FC0028F5
:10754000C1D1364920001BF0DCFC0028BBD13449F6
:1075500020001BF0D6FC0190B7E76778272A11D1ED
:10756000002B4DD0032B09D1272F05D1A278272A34
:1075700004D10234243AD31A0134ACE7012BFBD8EE
:107580000122F8E7222A11D11A006046824309D16C
:10759000222F05D1A278222A02D102346246EAE7DC
:1075A000002B01D0022BE7D10222E4E75C2A0AD1AA
:1075B000272F03D0222F01D05C2F04D11A00571E91
:1075C000BA41A418D8E7002BD6D15B2A12D006D82E
:1075D000282A0DD0293A57425741C91BCCE77B2AAC
:1075E0000AD07D2A0AD05D3A57425741ED1BC3E7C6
:1075F0000131C1E70135BFE70136BDE7013EBBE719
:10760000272FBDD1B2E7C046876B03005C0D030096
:10761000620D0300660D030072640300948703008B
:1076200081390300F0B58BB007934318039004929F
:1076300001930093009B5C1E039BA34201D900931E
:1076400010E0207801F008F8002801D00094F1E75C
:10765000207801F00DF80028F8D123785F2BF5D0C1
:107660002E2BF3D07D4B1D68009C019B9C4202D2C7
:1076700023782E2B21D1009BE71A019B9C4241D3FA
:107680000024260002940194AB68A34256D8019BC3
:10769000002B00D084E0009B039A93422FD1704CC2
:1076A0003A002100180021F065FB002827D1079B34
:1076B000E41907301C60C01B22E00134D5E7013615
:1076C000AB68B3421BD9F3000293EB68F200985801
:1076D0000028F4D00428F2D009A9FAF791F8099B00
:1076E0000100BB42EBD13A00009821F0C9FB002811
:1076F000E5D1EB68029A9B185868002804D1002055
:107700000BB0F0BD0026DBE7032318420CD1036861
:10771000544A934205D11BF089FE0500631C009377
:10772000A2E7514A934201D0FBF7C0F8856B002DC8
:10773000E5D04E4B2A689A42F0D0E0E7EA68E300D1
:10774000985800281CD004281AD009A9FAF758F82C
:10775000099B06900593BB4212D301003A000098A2
:1077600021F08EFB00280BD1029B002B12D03B0096
:107770009E4202D3059A9A4204D2019B013301939F
:10778000013481E7029AD15C069AD25C914205D11C
:107790000133EDE7069B059E0293EEE71E00ECE742
:1077A000019B012B01D0BE4254D9029B079ADB19E1
:1077B0001360F01BA4E7029BEA68DB0098580028DE
:1077C0003AD0042838D009A9FAF71AF8099B03908F
:1077D0000593BB4230D301003A00009821F050FBE2
:1077E0000190002828D133000F220F33DC171440FA
:1077F000E41824112401A41B012C00DC1034059A88
:1078000033199B18402B0DD9039A194904981FF07E
:1078100001FB099E10E0174904981FF03AFA019BFA
:1078200001330193019B9C42F5DC039904981FF0FE
:1078300030FA099BF6183619029B01330293AB68A4
:10784000029A9342B7D80C4904981FF022FA0120FB
:10785000404255E7002340260293F0E77C2E0020AB
:10786000500D030098B1020058B8020074C2020023
:10787000580D0300DE6F0300654F030010B50400D0
:107880001FF08FFC1AF0CDFF01280BD00649200015
:107890001FF0A2FC20001FF084FC1AF0C2FF022897
:1078A00000D0002010BDC046A60D0300F0B59DB06D
:1078B00000AF0C68032835D9CB68FB60042835D0AD
:1078C0000D6900206D102BD41C232000F918F9F746
:1078D00097FF7861002D5AD0954C9649606808F062
:1078E0005DFB0600606800229349043001F044F912
:1078F0001823FA18D11804003000F9F781FF3B6B08
:10790000013D0100C318002C05D1994203D2013B6F
:107910001A782E2AF9D1013D0ED299420FD187480B
:1079200005F054FD864B0025FB60CDE70025CBE735
:10793000013B1A782E2AEED09942F9D3EBE7FE6983
:107940005C1A2500002E01D0751C2D192B006A46EB
:107950000E33DB08DB00D31A9D46220018003B6182
:1079600021F017FA002E08D02E233A69601C135517
:1079700010187969320021F00CFA2900386909F0F1
:107980009BF806243B69C0000443FD617B61200035
:10799000F9F700FB01F0C4F8061E15D02E21786916
:1079A00021F04FFA00280BD0654BFA689A4207D1B4
:1079B0007B69C11A180009F07FF801F0B1F80600E0
:1079C0003000BD461DB0F0BD182318000125FA187F
:1079D000D2183818103B4021C0181FF0ADFBBE6014
:1079E0003E61FB69AB4205D2554BFA689A42E7D03B
:1079F000BE68E5E7AB4204D07B695B5D2E2B00D00F
:107A000094E02900786909F057F87B6A3860002B08
:107A100017D12A00082479691833F81800191FF0C3
:107A200056FB1823FB181819FFF728FF78607B68AE
:107A3000002B14D13A684349434800F033FD04F069
:107A40004DFE18230824FA182F2110190EF0E4F91E
:107A50003B693969EA1A7B6959181823DDE73868E8
:107A600001F05EF8041E4BD1386801F027F8FB697D
:107A70000400AB4213D1354BFA689A420FD17B68B0
:107A8000012B0FD0324A2B4940681DF0F5FE182219
:107A90000823BA18D11820001BF04EFA30E07B689A
:107AA000012BF4D10022796AB86AF9F751FAF4216E
:107AB0000200FF31200005F035F87B6A18227B6058
:107AC0000823B818C0182F210EF0A6F91822082391
:107AD000B818C0181F491FF07FFB18220823BA18D6
:107AE000D0181FF05EFB1AF09CFE022806D1182267
:107AF0000823BA18D11820001BF01EFA7B687B629D
:107B0000BB68002B0CD07A693B699446E91A634440
:107B1000180008F0D1FF22000100B86805F002F853
:107B2000002E00D126006B1C3B61BC60013558E77C
:107B30007C2E0020860F00009E0F00006A0D0300BF
:107B4000E4B30200890D03000CA90200C4E702009F
:107B5000760F00009E0D0300184BF7B530CB0F00D9
:107B6000160001281AD94B68154A934207D0990785
:107B700011D114491C688C420DD11C001D00022833
:107B80000CD0BB68934209D09A0704D10D4A1968FA
:107B90001C00914202D0002005F0DCFD01A93868EC
:107BA000F9F72EFE019A0100002310201DF0FAFFC4
:107BB0002A003100230005F0C1FBFEBD7C2E002011
:107BC000E4B3020074C20200F0B58BB006000800F6
:107BD00011001A0010AB1F78314B05AD01950093D1
:107BE00005230AF099FB912000011EF062FB2D4B4A
:107BF00004A91860059B476043706B682A4F0370A7
:107C0000AB6804008370EB68C3702B7C30003B6072
:107C1000F9F7F6FD0025254B03900C201D601EF0A2
:107C200048FB234B06000360FDF7CAFFB060FDF779
:107C3000C7FF204B204A1860204B11001D70204BBD
:107C400070601D701F4B30001D602B00FDF78CFE17
:107C50002000049A03991BF0EFF82000FFF73EFA8A
:107C60000400A84207D1FDF785FD0E4B1C60164BA2
:107C7000186805F0ABFB0122144B1A70FDF79AFF50
:107C80000028FBD1124B943318603B68002B04D0C2
:107C90000C4B1048196818F063FE07480BB0F0BD94
:107CA00050A40200102F0020582A00204C2A002047
:107CB0009CA40200482A0020E4B30200D02D00203A
:107CC000CE2D0020502A002004000020CF2D0020BF
:107CD0007C2E0020AA0D030000220D4910B50B7860
:107CE000DBB2934210D10B4A1478002C02D001244D
:107CF0000C701370084B1B78002B07D0074A1368D1
:107D000020331360064B1A68100010BD8268FBE731
:107D1000CE2D0020CF2D0020D02D00204C2A002079
:107D2000482A002073B501A9F9F76AFD019B0600F6
:107D30001748502B17D8802040001EF0BAFA154C77
:107D400005002300943318600023019A9A420CD155
:107D50005B232800AB540AF0C5FF2B00002808D194
:107D6000943420600C4805F031FBF15CE954013398
:107D7000ECE75A1B0133591E09789B29F9D12900D8
:107D800006481AF00DFB00239434236076BDC046EC
:107D9000B90D03007C2E0020C70D03000C9A0200D1
:107DA000D2235B005843134AF0B51368000C83429A
:107DB00006D9114C2368013323601368203B1360FC
:107DC0001F23050001270D4E9D431468A5420BD8C3
:107DD00003401A1D202A00D92022094C246893420E
:107DE00004D3084B1860F0BD3770EEE7E518297131
:107DF0000133F4E74C2A0020502A0020D02D002027
:107E0000482A0020542A002070B506000D000028E2
:107E100014DD002907DD154812F014F80124B042E2
:107E200009DB002407E00100C020000612F00AF878
:107E30000124A842F5DDE4B2200070BD002907DD71
:107E4000C020000611F0FEFF0124B042F3DCE8E799
:107E50000024A042F0D00100044811F0F3FF0123F8
:107E6000A84200DC231CDCB2E6E7C046FFFFFF3F70
:107E700070B504000D0010491EF00BFF6968012267
:107E80002000FAF72BFD0D4E200031001EF001FFFF
:107E9000A96801222000FAF721FD310020001EF020
:107EA000F8FEE96801222000FAF718FD04492000D5
:107EB0001EF0EFFE70BDC046DD0D030045FC020064
:107EC000A002030070B5060010200D0014001EF083
:107ED000F0F9034B466085600360C46070BDC04626
:107EE000E8A4020010B5FAF72DFE054912F07AFD5C
:107EF0000323020002209A43024B1043C01810BD16
:107F0000E02E65420000808010B5FAF71BFE05499F
:107F100012F068FD0323020002209A43024B104333
:107F2000C01810BD35FA8E3C0000808010B5FAF7FD
:107F300009FE011C13F04CF8024B002800D1024B43
:107F4000180010BDCCE70200C4E7020010B5FAF734
:107F5000F9FD440064080849201C13F039F8002892
:107F600005D10549201C12F0BDF8002801D00348B6
:107F700010BD0348FCE7C046FFFF7F7FC4E7020057
:107F8000CCE7020010B5FAF7DDFD034B03400220F9
:107F90001843024BC01810BDFCFFFF7F000080801B
:107FA00010B5FAF7CFFD440064080849201C13F00F
:107FB0000FF8002807D10549201C12F089F8002885
:107FC00001D1034810BD0348FCE7C046FFFF7F7F97
:107FD000CCE70200C4E702001FB500230193FAF7C3
:107FE000B1FD01A915F03CF90322030002209343DF
:107FF000064903435B180293019B934303435B18B9
:1080000002A90393FEF736FB05B000BD0000808097
:1080100070B50D00FAF796FD041C2800FAF792FDE2
:1080200012F0ECFF0100201C15F0F6F8032302000B
:1080300002209A43014B1043C01870BD000080809D
:108040001FB500230193FAF77DFD01A915F0BAF8D9
:10805000032302249843074B2043C0180290019841
:108060001DF02EFB02A903902000FEF703FB04B0D5
:1080700010BDC0460000808070B50D00FAF762FDAB
:10808000041C2800FAF75EFD011C201C15F0B2FB51
:108090000323020002209A43014B1043C01870BD15
:1080A0000000808070B50D00FAF74CFD041C28001C
:1080B000FAF748FDC00FC3076000400818430323C8
:1080C00002249843014B2043C01870BD00008080FB
:1080D00070B50D00FAF736FD041C2800FAF732FDE2
:1080E000011C201C15F00EFB0323020002209A4302
:1080F000014B1043C01870BD0000808010B5FAF726
:1081000021FD14F075FE0323020002209A43024B66
:108110001043C01810BDC0460000808010B5FAF7AB
:1081200011FD15F09DFA0323020002209A43024B31
:108130001043C01810BDC0460000808010B5FAF78B
:1081400001FD15F03BFA0323020002209A43024B83
:108150001043C01810BDC0460000808010B5FAF76B
:10816000F1FC15F091F90323020002209A43024B1F
:108170001043C01810BDC0460000808010B5FAF74B
:10818000E1FC15F043F90323020002209A43024B5D
:108190001043C01810BDC0460000808010B5FAF72B
:1081A000D1FC14F083FF0323020002209A43024B08
:1081B0001043C01810BDC0460000808010B5FAF70B
:1081C000C1FC15F0A3FA0323020002209A43024BDC
:1081D0001043C01810BDC0460000808070B50D006F
:1081E000FAF7B0FC041C2800FAF7ACFC011C201CB8
:1081F00015F0E4FB0323020002209A43014B1043D5
:10820000C01870BD0000808010B5FAF79BFC0021FB
:10821000041C11F053FF002802D0074805F0D6F8DF
:10822000201C15F08BFD0323020002209A43034B10
:108230001043C01810BDC046F50D0300000080803B
:1082400070B5060008680D00FAF77CFC0021041CDC
:1082500011F03EFF002802D0184805F0B7F8201CA6
:1082600015F030FB041C012E06D1032302209C4391
:108270002043134BC01870BD6868FAF763FC0021F7
:10828000051C11F025FF0028E6D1FE21281C8905D8
:1082900011F00EFF002803D00A490B481CF0CAFB5E
:1082A000281C15F00FFB011C201C12F0C3F903233E
:1082B000020002209A431043DBE7C046F50D03009D
:1082C00000008080E40D030044AD0200F0B50E0014
:1082D0001100002285B0B71C03901C0030000D4B2C
:1082E0000092BF0009F0E8FF38001DF0E2FF466091
:1082F00006000500039B083F03600836E719BC42EF
:1083000002D1280005B0F0BD002101CC04F02EFC04
:1083100001C6F4E7FFFF0000F7B505002C200E00B2
:10832000170001931DF0D7FF040005708660878158
:10833000072D01D0012D0FD1337872780A3B1B0233
:108340001343E381019B20206375042363841DF0A4
:10835000B0FFA0622000FEBD014B5B5DF1E7C046AF
:10836000070E0300F7B50D00110000220600009271
:1083700028001F000B4B09F09FFF10201DF0A6FFE7
:10838000041E08D1084B094A094C5A620023266092
:108390002000A360FEBD39002800FEF76BF9E06005
:1083A000F4E7C046FFFF00007C2E002044A002003E
:1083B000942E002010B5013810C9FEF75BF9E0607B
:1083C000004810BDE4B30200F8B57F2553B20400A5
:1083D0000E0017001540002B0ADB6B1E012B07D87F
:1083E0000B6858681DF0C6FA010020001EF051FC11
:1083F000022D16D10F4920001EF04BFCF368002B14
:1084000002D05A68002A04D10B4920001EF041FC1A
:10841000F8BD012A07D1002299682000FAF75EFA18
:10842000F6E7002DEAD03A00F1682000FEF7C8F820
:10843000EEE7C046613A03003B830300C36803488C
:108440005A68002A00D098687047C046E4B302001A
:10845000136810B51400002B0BD0FC23FF33994296
:1084600006D10C4B52689A4202D10023C38023608C
:1084700010BD094B994201D1C368F8E7074B026868
:108480009A42F5D1064B9942F2D1FFF7D7FF20600F
:10849000EEE7C046E4B3020003020000DCAB0200DA
:1084A000E30200000EB470B5050087B010201DF087
:1084B0000DFF041E0BD11A4B1A4A1B4C9D6118620A
:1084C0005A62200007B070BC08BC03B018470021F6
:1084D000056081600120FEF7CDF82521E0600500F0
:1084E0000B9820F0AEFC061E09D10B9820F0C1FCC1
:1084F000320001000B98F8F72BFDA860E1E702A815
:1085000010211EF000FE0CAA0B9902A801920DF09A
:10851000D7FC02A90548E568F8F7E4FCEDE7C0469A
:108520007C2E002044A00200942E00200C9A020011
:1085300010B50300820708D1064A0168914204D1B0
:10854000054AD9680120914203D00449180003F07C
:10855000C3FB10BD58B80200658300001CA80200D0
:1085600010B50400FAF7A2F9034BC2689A4200D092
:1085700024690023A36010BD65830000F8B51600D0
:108580001D0004000F00FAF791F9154BC2689A42DA
:1085900000D02469A068002811D10C301DF096FE8F
:1085A000A06000280AD003236360E288A1689300DA
:1085B000CB180332E2801F605E609D60F8BDE388E7
:1085C000A18802338B42F0DB0331890001221DF0C8
:1085D0009BFE0028F2D0A388A0600333A380E4E7C9
:1085E0006583000070B5150004000E00FAF75EF90F
:1085F000064BC2689A4200D02469A368002B02D1BE
:1086000033602B6070BDE2883260FAE7658300005A
:10861000F8B5050010200C001F0016001DF049FEE3
:10862000054B44608460A4190760C4606B60034B11
:108630002860AB60F8BDC046593202006F320200BC
:1086400000237F2803D8034B1B5C9B07DB0F18001C
:108650007047C0460E0E030000237F2803D8034B4B
:108660001B5C1B07DB0F18007047C0460E0E030093
:1086700000237F2803D8034B1B5C5B07DB0F18002C
:108680007047C0460E0E030000237F2803D8034B1B
:108690001B5C5B06DB0F18007047C0460E0E030024
:1086A00000227F2808D8054B0132195C0C2319429F
:1086B00002D15F3842424241100070470E0E030063
:1086C00000237F2803D8034B1B5CDB06DB0F18005D
:1086D0007047C0460E0E030000237F2803D8034BCB
:1086E0001B5C9B06DB0F18007047C0460E0E030094
:1086F00070B50400FAF7DAF800230C49DA005218D2
:108700001568A54205D1516809481EF0C2FA01203A
:1087100070BD0133612BF1D1064B9C4203D09842CE
:1087200001D00020F4E70449EEE7C04680AD020026
:1087300084E8020088E902008E0E0300FF23032272
:10874000DB05CB1810B59343042804D811F0DCFAEC
:1087500006030F0416000021080010BD0021181C9C
:1087600011F0A6FC0A490028F6D00A49F4E7181CC3
:1087700012F044FC012140000143EDE7802109068D
:108780005B18022193431943034BC918E4E7C04621
:10879000CCE70200C4E7020000008080FF23DB0575
:1087A00010B50400C81803239843002386B0019332
:1087B000063300931022613302A903F00BFB02A9D8
:1087C00020001EF066FA2E2102A820F03AFB0028B5
:1087D0000FD1652102A820F034FB002809D16E21B9
:1087E00002A820F02EFB002803D1034920001EF030
:1087F00050FA06B010BDC046C404030030B50C00EA
:108800001100002285B01D0000920123200009F014
:1088100053FD002C23D02868124B0340062B06D0B2
:10882000032420420ED1104B02689A420AD103A9B8
:10883000F8F7E6FF0022039900921300F9F70AFF08
:1088400005B030BD03002340022BF9D0FAF77AF9C6
:1088500003000220A3431843044BC018F0E7044868
:10886000EEE7C046070080FF0C9A020000008080FF
:1088700002008080F0B5050087B010000191FAF782
:1088800061F9041C0390681F182800D9BDE011F09D
:108890003BFA0D121F24333E6F81BCBCBCBCBC0D27
:1088A000121F24333E6F9FA8ADB2B7000198211C60
:1088B00011F026FD03E0211C019812F0C5F901908A
:1088C00003230198524A9843013B03439B187CE0E1
:1088D000211C019812F086F8F1E70021201C11F00C
:1088E000E7FB002803D04B494B481CF0A3F803A931
:1088F00001A81AF024FDE3E70021201C11F0D8FBA9
:108900000028F0D1211C019811F094FED7E7002136
:10891000201C11F0CDFB0028E5D1211C019814F09A
:1089200069FF0021041C019011F0C2FB002807D050
:10893000039A0023002A01DA80231B060193BFE774
:108940000021201C039E012711F0B8FB002800D154
:10895000071C0021301C012511F0B0FB002800D1BC
:10896000051CFFB2EDB2AF42AAD0311C201C9FE71C
:10897000019D0021281C11F09BFB002805D000213F
:10898000201C11F09BFB0028ADD1211C281C15F0E8
:1089900015F894E70021201C11F08AFB0028A2D1D1
:1089A00003A901A81AF0CBFC03220220019B18495D
:1089B000934303435B180493039B934303435B1864
:1089C00004A90593FDF756FE0300180007B0F0BD9B
:1089D0000199201C11F086FB104B0028F5D1104B9B
:1089E000F3E70199201C11F069FBF5E70199201CC0
:1089F00011F05EFBF0E70199201C11F07DFBEBE725
:108A00000199201C11F064FBE6E70023DDE7C04676
:108A100000008080E40D030044AD0200CCE70200BA
:108A2000C4E7020010B5040048680022043007497A
:108A300000F0A2F8064A002803D04068F8F7CAFE02
:108A40000200044920001EF0E5F910BD860F000069
:108A50003B8303009534030070B5150012680C00C9
:108A60004068002A0AD1CC0006210430214300F0DE
:108A700083F8002801D043682B6070BD03799B0701
:108A80000BD50C4B9842F8D10B4EF36D002B03D154
:108A900001201CF0B8FEF065F06D06216A68E40064
:108AA0002143002A03D11CF0F1FE0023E4E71CF06F
:108AB000E3FEFAE7649D02007C2E002070B50625D7
:108AC000C0000543012229000B4800F055F8446816
:108AD0000600002C0ED108201DF0EBFB074B040014
:108AE000036001201CF08FFE2A00606004491CF026
:108AF000C3FE7460200070BDB82E002098B1020043
:108B0000860F000010B50C000621C00001430122B1
:108B1000024800F031F8446010BDC046B82E002075
:108B200073B50625C3001D43060000222900104826
:108B300000F022F8041E18D1020029000D4800F0B0
:108B40001BF8041E12D0EA216A46FF31406803F088
:108B50008FFF009B002B08D000216A4608001BF005
:108B60002DFF61683000FFF7CDFF606876BDC0461D
:108B7000B82E0020C4B00200F0B587B00092027891
:108B800004000F00930703D5009B002B00D0F5E0F5
:108B9000D307DB0F0ED07A4B3B40062B43D0032389
:108BA0003B4003D177493868884203D0009B012BB2
:108BB00000D0E3E0019353075FD52368A568DE0882
:108BC000F600AE19B54230D3009B012B00D0D5E0A2
:108BD0002368D9086368994210D104316160A068A4
:108BE000C9001DF084FB23686268DB08D21ADB0031
:108BF000A060D200C018002120F0E7F80721236808
:108C0000DD086A1CD2000B4013432360A368ED000B
:108C10005D195B4B2F601F40062F21D00122237866
:108C2000934323701CE00123C4E72868B8421AD19B
:108C3000009B022B14D129002368721BD210083B21
:108C4000013A6F6828002360D200083120F0AAF8AA
:108C50002368DD08A368ED005D1900236F602B60B9
:108C6000280007B0F0BD019B002B04D13900F9F7B3
:108C7000B3FE0028DCD10835A4E76368002B05D1DA
:108C8000009B012B7AD1200000F07EF83C4B3B404A
:108C90000593062B27D1F8081CF062FE039061684B
:108CA000039811F0CBF800260491049B0293029BD9
:108CB000DD00A3685D19286800281BD1009B012BEB
:108CC0005CD107212368DA080132D2000B4013433C
:108CD0002360002E00D0350000236B60059B2F60C1
:108CE000062B9BD1BCE73900022003F0D7FD4310CF
:108CF0000393D4E7042803D1002E1DD12E001BE0DE
:108D0000B84211D1009B022BAAD123680298083BDC
:108D100023600130616811F091F8A368C900CB5855
:108D2000002B25D12B609BE7019B002B04D1390040
:108D3000F9F752FE0028E5D102986168013011F080
:108D40007DF8049B02918B42B1D1009B012B15D180
:108D5000002E0FD023683500083323600023736092
:108D6000059B3760062B00D17AE72378009A57E7F6
:108D70000423D7E7200000F007F890E700256FE70D
:108D8000070080FF0C9A0200F7B5436804000193C6
:108D90005A1C002317495800455AAA4206D90133E4
:108DA000222BF8D15508AD18213B1D43E800A768D8
:108DB0001DF091FA07232268656013400122002507
:108DC000236013432370A060019B9D4203D13800B0
:108DD0001DF09EFAF7BDEE00B959002908D004290C
:108DE00006D001222000FFF7C7FEBE19736843605A
:108DF0000135E9E7B0F60200F8B505000023046884
:108E000086681449621C5800405A824206D90133D0
:108E1000222BF8D15008821801201043002328602B
:108E20006B6080001DF057FA3700A400A860A419F9
:108E3000A74203D130001DF06BFAF8BD3968002954
:108E400005D0042903D0012228001AF02BFB043797
:108E5000EEE7C046B0F602000379044AD35C002B6B
:108E600000D183790248DB00C0187047D12D002063
:108E7000E0B1020010B50400FFF7EEFF22790368AD
:108E800002490348FFF70EFB03F028FCA33403005C
:108E900008AD0200002803D001210379014AD15412
:108EA0007047C046D12D002010B5FFF7D5FF034B0A
:108EB0004068C01A431E9841C0B210BD758E0000B4
:108EC00070B506000C00FFF7C7FF0C4D2B002833D0
:108ED000984204D12A001032002394420BD0002380
:108EE000A04208D0436830009847641B3379044A95
:108EF000E410D4540123180070BDC046E0B1020054
:108F0000D12D0020F0B589B0002807D1664B674805
:108F100019681DF0BEFE664809B0F0BD0D68654BCE
:108F20009D425BD1002108001DF09AFD0024050040
:108F30000590614B5A680192944217D300255F4A0D
:108F400005A901200BF0A8F907AA06A905981DF0AC
:108F50009EFD069B03339B0801939B000393019B9B
:108F6000524EAB4210D156493000D2E79B68019374
:108F7000019AE3009958002904D0042902D028005E
:108F80000BF02AF90134D4E72F00AB000293079BC2
:108F9000029A9858F8F71EFC010030001DF079FE87
:108FA000019BFF18069B9F4212D212231C1A002C11
:108FB00007DD013C07D2039A029B94466344029367
:108FC000E5E71234F3E73F4930001DF062FEF0E7B9
:108FD0003D4930001DF05DFE0135C0E72800F9F77E
:108FE00065FC3A4B42689A4200D16D682800FFF751
:108FF0007FFB061E00D08EE72C4C354920001DF06B
:1090000048FE31002800F9F783FC280019F00FFB17
:109010003049020020001DF0FDFEAB0732D12B6865
:109020002D4A93422BD128001AF000FA1CF039FC8B
:1090300000250600A84200D16DE773689D4200D369
:1090400069E7B268EB00D3181F68002F15D05B6882
:109050002249200001931DF01CFE00213800F9F781
:1090600057FC1F4920001DF014FE00210198F9F75C
:109070004FFC154920001DF00CFE0135DDE7194AB3
:10908000934203D02800F9F711FC0500A86B0028D3
:1090900000D140E7830700D03DE7134B02689A42B6
:1090A00000D038E7C2E7C0460800002084E802008C
:1090B000E4B3020046140000C4B00200D4B10200C0
:1090C000B5340300DE6F0300654F03000D0200009E
:1090D000D9340300E134030098B10200DD6F0300CE
:1090E000F134030058B8020074C20200002803D013
:1090F000012807D0002004E08B680448002B00D131
:10910000034870478B685B001843FAE7CCE702001E
:10911000C4E70200034B48600B60002308008B602B
:10912000CB60704798B202007FB5040001220800AE
:1091300001A9F9F75DFE0022217940200BF0E6FA43
:1091400001000500029810F0F3FD636806001A0A9A
:10915000824218D2A368C1186943E0681DF0C7F8BD
:109160006368E060DBB22A00A06863606843E3687C
:109170007243181801991FF00CFEA36804489E1949
:10918000A66004B070BD121A1202DBB21343EAE704
:10919000E4B30200F7B5FF27456804000191BD4321
:1091A0001DD101792A0040200BF0B0FA6368060057
:1091B0003B408027A1683F011F430831414367605E
:1091C000E0681DF094F86368E0601A0AA368013A49
:1091D000013372435E43290080191FF0F6FD2079A8
:1091E000019BA268E1680BF031FCA36803480133DE
:1091F000A3606368013BFF3B6360FEBDE4B3020014
:10920000F8B5002207000D00010040200BF07EFAA7
:10921000060010201DF04DF8084B0400012F00D06F
:10922000074B2800277123606368A560DBB2704399
:1092300063601DF03EF8E0602000F8BD30B302002E
:10924000F4B2020070B506008AB00C0015001228B6
:109250005CD003D8052826D0002454E01B2800D178
:109260006CE01F28F8D1012207A9280019F0F6F9AF
:10927000032300284FD01C4213D13B4B22689A4253
:109280000FD1012204A920001AF0B8F90123079A8E
:1092900000930599089B049819F063F8334C002853
:1092A00031D1334C2FE0012204A920001AF0A6F995
:1092B0002800012207A9F9F79BFD069B00220393D2
:1092C0006B464020197B0BF021FA0100060008983C
:1092D00010F02EFD069BA16803936B464118050014
:1092E000187BFFF78DFF059B04001A000499C068E6
:1092F00003931FF04EFD2A000598E3687243181887
:1093000007991FF046FD20000AB070BD1100200033
:10931000FFF70AFFF7E7EA070DD41D4203D1154B0B
:109320002A689A4207D003232B40022BB9D1124B53
:109330001D40062DB5D0114804F03AFA012204A9C7
:1093400020001AF05BF9012207A9280019F086F91C
:109350000028A6D0089B059A00930499079B30002B
:109360001CF07DFC9AE7C04630B30200CCE7020057
:10937000C4E702002CB90200070080FF3B83030012
:10938000F0B5050087B00E00012808D08B0726D164
:109390000B68264A934202D0254A93421FD10122EC
:1093A00003A9300019F05AF9002818D0002229002A
:1093B00040200BF0ABF901000700049810F0B8FC56
:1093C000060001002800FFF71BFF320004007A436B
:1093D0000399C0681FF0DDFC200007B0F0BD30002D
:1093E000F9F766FC071E00D0471039002800FFF788
:1093F00007FF00210400300003F0B8FB00260090B6
:10940000009803F015FC031EE6D0002F04D11900CC
:109410002000FFF7BFFEF3E7721C0192E168320003
:1094200028000BF013FB019EEAE7C046A092020061
:1094300030B3020070B50E7904000D00012E0DD17D
:1094400019491DF026FC3300AA68E9682000F7F7E7
:10945000E5FC164920001DF01CFC70BD32001449CB
:109460001DF0D8FCAB68002BF3D0124920001DF092
:1094700010FC0026AB68B34204D80F4920001DF051
:1094800008FCE6E7002E03D00C4920001DF001FC8B
:109490003200E96828790BF0A1F9012201002000CF
:1094A000F9F71CFA0136E5E7F6340300A0020300E1
:1094B000023503000D3503001D06030045FC0200C4
:1094C00070B5050086B0161E44D0032480680C4099
:1094D0002BD1214B0A689A4227D103AA08F0C4F97C
:1094E000002802D11D4804F063F9042E1AD122008D
:1094F000297940200BF00AF9049B06000093039B96
:1095000028790193019A009B991AFFF779FE039934
:10951000049A0400521A71437243EE68C0687118CD
:109520001FF037FC200006B070BD0A0000230100C8
:109530002868F9F77BFB02002879042E04D1E9683A
:109540000BF04CF90400EDE73300E9680BF07EFA0C
:10955000034CE7E71400E5E7E8A40200A6FC0200DC
:10956000E4B3020037B50C00110000221D00009288
:109570000123200008F0A0FE002C05D121000120CD
:10958000FFF73EFE040016E02968CB0705D48B07E1
:1095900013D10C4B0A689A420FD10800F9F76EFA02
:1095A000010005000120FFF72BFE2A000400002126
:1095B000C0681FF00AFC20003EBD0120FFF7E0FE5E
:1095C000E0E7C0462CB9020037B50400A06803F0FC
:1095D0002FFB019000280ED06568074B9D4205D0F7
:1095E00001AB00220121280003F0CAF9F9F784FB3E
:1095F0000028EBD001983EBDE4B3020030B58DB039
:109600000500684603F044F8011E10D12A1D012010
:109610001BF0D4F90122EB6804005B1001335B00FE
:109620001343EB6003F052F820000DB030BD0198F9
:10963000054A0368934205D0044A00249342F3D0BC
:1096400003F04CF80024EFE7DCAB020084A9020031
:10965000044B0B6003684B60436808008B60012378
:10966000CB607047A8B3020010B502491DF011FB92
:1096700010BDC0461135030010B50400034B036054
:1096800040301DF02FFE200010BDC04624B6020061
:1096900010B50F4C20001FF027F8002808D020003C
:1096A0001EF0F4FF0B4B1B68984202D1FAF7C4FC82
:1096B00010BD3F21084A138801330B400749098830
:1096C0008B42F5D01188064C13806054F0E7C046F9
:1096D0005C2A0020782E0020BC2D0020BE2D00200A
:1096E000F12D0020002210B5044B05491A80054BCE
:1096F00005481A801EF0FDFF10BDC046BC2D00209D
:1097000091960000BE2D00205C2A0020034B188893
:10971000034B1B88C01A431E98417047BE2D002082
:10972000BC2D0020084A094B10881988884201D1B5
:1097300030BFF9E713880649C85C3F21138801331D
:109740000B4013807047C046BE2D0020BC2D00206A
:10975000F12D002070B504004518AC4205D02178E9
:1097600002481EF097FF0134F7E770BD5C2A002025
:1097700070B504004518AC420DD02378064E0A2B74
:1097800003D10D2130001EF085FF217830001EF03E
:1097900081FF0134EFE770BD5C2A002070B5040042
:1097A0000825002C08D02100082C00D929000348E6
:1097B000641AFFF7CFFFF4E770BDC0461F35030002
:1097C00070B5050004000826002C08D02100082CE4
:1097D00000D931000448641AFFF7BCFFF4E7280001
:1097E000FFF7DCFF70BDC0461635030010B5010061
:1097F00001481BF04DFE10BD1C000020142313B5C2
:10980000064C00931922182120000DF069FF044A2C
:10981000044920001FF04CFA13BDC0465C2A00200A
:10982000000000207996000010B5024B672219F065
:10983000F2FF10BD3541020010B5024B972219F01E
:10984000EAFF10BD59AA0000F7B50F0011001A0079
:10985000C38A8579868A019300230400837143615A
:109860000F4B19F0D8FFA368002B17D1E18A00290C
:1098700008D0A38A002B05D1206B1BF09FFC206B26
:109880001BF01CFBA38AE28A3900200019F074FF48
:109890006B1E9D41019BA571A682E382F7BDC04668
:1098A00075A6000010B54379C26A012B03D11000E0
:1098B00019F08EFB10BD0B00006B024919F0B2FBD2
:1098C000F8E7C0462CBD02007FB50B7804000D0000
:1098D0004E1C002B0AD0032B0BD103A928001CF02F
:1098E00050FB03990600206B1BF07FFA300004B098
:1098F00070BD012B07D18E1C49780429F6D0006B6E
:1099000005F0F0F9F2E7042B0BD14B788978006B66
:10991000090219431BF0B1FA28001CF06DFB060088
:10992000E4E7052B15D14379042B04D02649006BBD
:109930001BF0AFFAF0E788784B780002184303A9D0
:109940001CF01DF80399246BF7F71AFB01002000A7
:10995000EEE71A000A3A0F2A09D803A9280019F0DD
:10996000DFFE039906002000FFF79CFFBEE7082BEF
:109970000CD103A928001CF0FAFA039B226A9B0071
:1099800006009958206B1BF084FAAFE703AB02AADC
:1099900001A928001CF061FB05000299206B05F06D
:1099A00055F9019B094A9B009B582900039A200006
:1099B0009847A368002B04D0E368002B01D1029BD9
:1099C000E360039E92E7C046E4B302002CB60200B7
:1099D000F7B506000192FFF777FF04270500019B0A
:1099E0009D4200D1F7BDA91C30006C78FFF76CFFD9
:1099F0002F3CE4B205003900082C01D8024B195D58
:109A0000306B1BF0B9FBEAE72835030010B543794A
:109A1000C26A012B03D1100019F0EBFA10BD0B0044
:109A2000006B024919F0FEFAF8E7C0463CBD02009F
:109A300010B54379C26A012B03D1100019F0D9FA8D
:109A400010BD0B00006B024919F0ECFAF8E7C046B4
:109A50001CBD0200836870B504000D00002B09D105
:109A60001100054819F0DEFBA060200029000C3031
:109A70001AF0F3F870BDC04618AC020010B5024AE7
:109A8000FFF7E8FF10BDC04670380300F0B50400D2
:109A90000D00E162002162712B7891B005920161A5
:109AA0009F4A072B3BD1059B012B06D00200836BFD
:109AB00008321B680599406B9847AB6818000893FB
:109AC0001CF09AFA63790890032B0FD10D90402176
:109AD0000DA81CF0AAFAA36B02009B680D99606B9D
:109AE0009847A368E882002B00D0D4E008981CF0C7
:109AF00083FA08900378002B4FD00A3B0F2B47D8EE
:109B00000DA919F00DFE95220D9B9200934244D0B1
:109B10000AD80125483A93420DD0824A089920007C
:109B2000FFF798FF11B0F0BD7F4A934202D07F4A01
:109B30000325F0E7002508981CF05EFA182108902C
:109B400008A81CF072FA089B07900693069B079AD8
:109B5000934224D16379012B15D9A36B29005B684B
:109B6000606B98476379042B0DD10023E06A03955D
:109B70000293C18A626B0191009393680521D268B8
:109B80000069FAF777FAA368002B00D083E0C9E7F1
:109B90000100674A2000FFF75DFF0225CBE7069B27
:109BA00008931B78222B04D106981CF025FA069006
:109BB000CCE71F2B01D05F4AB0E709A906981CF03B
:109BC00025FA03780600432BF5D11CF015FA099B02
:109BD0009842F0D109A930001CF018FA0378070068
:109BE0000A3B0F2BE7D81CF007FA099B06008342BB
:109BF000E1D00378472BDED11CF0FEF9099B984297
:109C0000D9D10AA9380019F08BFD30001CF0F9F900
:109C10009F210B900BA81CF008FA01000B981CF078
:109C2000DFF99B220A9B0600920093421BD1012878
:109C300004D10B9803780A3B0F2B01D93E4A6DE7FC
:109C40002669731C2361059B012B21D00DA919F0F6
:109C500067FDA36B0D9ADB683100606B98470028A5
:109C600016D1364A5AE7364A93421AD1012803D10F
:109C70000B980378032B01D0324A4FE7059B012B49
:109C800006D0666B1CF08CF9010030001CF0B8FAAD
:109C9000A368002B88D0200008990C3019F0DDFF54
:109CA00040E789229200934222D1012803D90B98E0
:109CB0000378032B01D0244A30E7059B012BE7D022
:109CC0000CA91CF05EF901270B900B980378032B6D
:109CD00001D01E4A22E70DA91CF053F901370B9061
:109CE0000D9A0C99606B1CF092FABE42EDD1CFE751
:109CF000059B012BCCD0032800D95CE70B9B1800F7
:109D00000D931CF079F90E901CF076F9A36B0F906F
:109D10001F6932000DAB0A99606BB847B8E7C046BF
:109D2000653703008937030091020000DA02000062
:109D300096370300BE370300E1370300FD37030009
:109D4000FF0100000D380300293803004E380300DE
:109D5000F0B587B001920A000593531E9A410D0099
:109D600006000599019804921CF03AF92C1E039004
:109D700009D02B7800243A2B05D102002100306B4A
:109D80001BF08DFA2C00049B019F0293059B9F42C0
:109D90001ED1002C3BD1039A049B944663441900C6
:109DA000306B1BF070FA002D3ED1019B9F422CD0EE
:109DB000019B9C423BD120001CF023F900220100B2
:109DC000300000F039F801981CF016F90190ECE72A
:109DD0003B783A2B0CD1002C12D1049B306B5A1ECD
:109DE000039B3C00D218029BD21A19001BF057FAB1
:109DF00038001CF001F9029B070001330293C5E70C
:109E00000C4A39003000FFF725FE07B0F0BD002DE9
:109E1000CBD0AC4208D120001CF0F3F800220100A6
:109E2000300000F009F8C0E700222900F8E700221E
:109E30000199C5E79B350300F0B50B7817001A00B0
:109E40000A3A85B004000D000F2A10D803A9280093
:109E500019F066FC03992000002F01D0022F03D1D6
:109E6000FFF7D4FD05B0F0BDFFF71CFDFAE76A4A25
:109E7000192B00D8CBE01A3B2A2B00D182E005DC5D
:109E8000062B08D0292B11D0644AC0E02B2B00D11F
:109E900094E0972BF8D1002F00D0B7E003A9280059
:109EA0001CF0B4F80200039B00219BE002A92800EB
:109EB0001CF0ACF80600022F03D001002000FFF7D1
:109EC00003FD30001CF098F80299060019F01DFC03
:109ED0000028D9D13378A22B13D1300003A91CF06C
:109EE00095F8060030001CF087F8039A0190904224
:109EF00007D2022F03D031002000FFF7E5FC019EBE
:109F0000F0E73378482B21D1022F06D1206B1BF0CC
:109F100060F8206B1BF01CF80EE030001CF071F8AC
:109F200001002000FFF7D0FC206B012FF2D11BF0C5
:109F300024F8206B1AF0F4FF30001CF05DF8029951
:109F400019F0E3FB002800D08CE79DE7492B9BD15B
:109F500030001CF056F803A919F0E2FB012F07D1DD
:109F6000206B1BF000F80399206B1AF0B1FFE3E7B8
:109F7000022F02D1206B1BF015F80399206B1AF009
:109F8000DAFFD9E703A928001CF040F8039906007E
:109F900019F0BBFB002800D076E7002F36D1350042
:109FA00003A928001CF032F806001CF025F80378FD
:109FB000A92B1BD100231A00310013E0002F25D15B
:109FC00003A928001CF022F80399050019F09DFB55
:109FD000021E02D03B003A0066E72B78A62BDFD0AA
:109FE000030029002000FFF7B3FE3BE7AA2B05D1B1
:109FF00003A91CF00BF8039B0200DDE7C12B00D185
:10A0000042E71BF0F9FF320003004DE7044A290044
:10A010002000FFF71FFD25E73C3503005435030002
:10A020006F350300F0B5170085B0040008000D007F
:10A030001BF0E2FF3900060019F067FB01900028D1
:10A040001FD02379002B17D0E36A1E78002E13D17E
:10A05000F6212000FF31FFF725FC29002000FFF743
:10A0600033FC330032000121206B1BF056F9206BCA
:10A070001AF08DFF05B0F0BD29002000FFF724FC89
:10A08000F5E733786D2B1DD1290001222000FFF761
:10A09000D3FE30001BF0B5FF4378811C4E3BDBB292
:10A0A00018260A2B01D8234AD65C2000FFF70CFCA7
:10A0B0003100206B1BF060F8022229002000FFF71E
:10A0C000BBFED7E76E2B2ED1300003A91BF09EFFFD
:10A0D00006000700039BBB421FD101992000FFF738
:10A0E000F3FB206B1AF03FFF002229002000FFF74E
:10A0F000A3FE019BB342BDD030001BF07DFF019B4E
:10A100000500834202D0206B1AF02DFF310000229F
:10A110002000FFF791FE2E00EBE738001BF06CFFEC
:10A1200001970700D6E731002000FFF7CDFB019A29
:10A13000C3E7C04631350300F0B50B788FB00A3B5A
:10A140000400019103920F2B00D906E108001BF0D7
:10A1500053FF0378432B00D0FFE001981BF04CFF26
:10A160000BA91BF053FF037842780A3B1B021343F1
:10A17000A14A934200D0F0E01BF03EFF03780500B7
:10A18000472B00D0E9E01BF07CFF002800D0E4E082
:10A1900028001BF031FF0B9B984200D0DDE0280027
:10A1A0001BF02FFF9F210C900CA81BF03EFF0C9B77
:10A1B00007000293012302980D931BF01DFF050079
:10A1C0000C90B84200D1BDE01BF016FF0C90B842D5
:10A1D0000ED00378032B00D0BFE00DA91BF0D1FEF9
:10A1E0000D9B0C90002B00D1B7E0B84200D0B4E03A
:10A1F000029B1B784533DBB2022B00D8ADE02B78F5
:10A200004533DBB2022B00D8A7E00B9B1800059367
:10A210001BF0F2FE039B0700984200D100270D9B24
:10A2200026690493238B26830693638B0793E38B22
:10A230000893731C6383A38BE383331D23612B7803
:10A24000D91E03930B00591E8B410993039B032BCB
:10A2500003D029002000FFF737FB02992000FFF709
:10A2600033FBF11C206B1AF0C9FEB11C206B1AF0F5
:10A2700088FD206B1AF077FE002201992000FFF77D
:10A28000DBFD05992000FFF71FFB711C206B1AF006
:10A2900078FD0499206B1AF0A8FD1221206B1AF0AA
:10A2A0006BFF206BF11C1AF06CFD039B206B032BE2
:10A2B0004CD01AF062FE206B1AF074FE049B206BE7
:10A2C0001921002B00DA1A2100251AF055FFB21CC3
:10A2D0000121206B1AF09EFE069B2383079B63835C
:10A2E000089BE383AF4218D0206B1AF050FE039B0B
:10A2F000032B02D0206B1AF04AFE39002000FFF732
:10A30000E3FA2569206B6B1C290023611AF076FEA5
:10A310000999206B01311AF07AFC3100206B1AF098
:10A3200030FD206B1AF033FE039B032B02D0206B11
:10A330001AF02DFE002F03D02900206B1AF021FD0A
:10A340000FB0F0BD2D4B029D029351E71AF00BFEAA
:10A3500029002000FFF7B8FAB0E7238B25690293A4
:10A36000638B6E1C0493E38B66830593AB1C06938F
:10A37000A38B0198E383224B2B432383EB1C2361A4
:10A380001BF03AFE01002000FFF79EFA07000121B2
:10A39000206B1AF090FE3100206B1AF0F2FCA91C21
:10A3A000206B1AF09BFE002201992000FFF744FD6C
:10A3B00039002000FFF788FA0700206B1AF022FC12
:10A3C000002803D13100206B1AF018FEA91C206B65
:10A3D0001AF0D7FC206B1AF08DFE029B2383049B9E
:10A3E0006383059BE383039BBB42A5D03900200018
:10A3F000FFF76AFAA0E7C046A20200001A6D030048
:10A400000080FFFFF0B589B005000591049200932C
:10A410000191002904D09F2105A81BF006FE0190A0
:10A4200000231E001F00059C03930293019BA3427F
:10A430001AD1002E0DD0029B002B00D079E0286BA2
:10A440001AF03CFD039B002B00D077E0286B1AF03C
:10A4500035FD049B286B002B00D174E033003A00DB
:10A4600000991AF063FF0AE02378BB2B14D1BA3BA2
:10A470001E4206D0374A21002800FFF7EBFA09B048
:10A48000F0BD012320001E431BF0BBFD0290200005
:10A490001BF0B2FD0400C9E7BC2B0BD1BA3B1E4236
:10A4A00001D02D4AE7E7022320001E431BF0A9FD3F
:10A4B0000390ECE7BD2B2AD120001BF0A2FD040085
:10A4C0001BF09AFD0378C12B0BD128000622210036
:10A4D00019F031FA009B2000013300931BF08CFD32
:10A4E000D6E723780A3B0F2B01D91C4AC3E707A9FB
:10A4F000200019F015F904000799286B1AF0BDFC2B
:10A5000021002800FFF7E0F9013704008EE7002E54
:10A5100001D0134AAFE7002F01D0124AABE7210068
:10A520002800FFF7D1F9009B0400013300933E009F
:10A530007CE702992800FFF7C7F983E70399280011
:10A54000FFF7C2F985E733003A0000991AF0E5FEFB
:10A5500095E7C0468D380300A4380300BC380300DB
:10A56000DD380300F8380300F0B589B0040003912A
:10A5700003A83D211BF059FD0027E36A02905E7D90
:10A580000398029B984215D118001BF03AFD029BDC
:10A5900003901B780100320020001D2B59D119F0C7
:10A5A00075F90500013F57D229002000FFF72EFA68
:10A5B00009B0F0BD05A91BF029FD6821039003A88F
:10A5C0001BF033FD06A90500039819F0A9F896239E
:10A5D000069AFF3301909A4213D003992000FFF7A7
:10A5E00073F9013703900398A84229D105992800EF
:10A5F00019F08BF800280CD129002000FFF764F92E
:10A6000007E0019B9D4207D8174A00212000FFF771
:10A6100021FA059B0393B3E701981BF0EDFC8542FB
:10A62000F2D107A9019819F07BF8079B0F4A9342D2
:10A6300004D00F4A9342E7D10426EAE70126E8E76F
:10A6400007A919F06DF807990390206B1AF040FCE8
:10A65000C9E719F065FBA4E7002301211A00206B6C
:10A660001AF05BFE9EE7C04654360300110200005C
:10A6700006020000F7B50A780E00130008215D3BC2
:10A680008B43DBB20400002B02D101338371F7BD91
:10A6900013005E3B8B43DBB2002BF8D013000A3B68
:10A6A0000F2B2FD95C2A11D101A930001BF0AEFC71
:10A6B00007001BF0A1FC019B834205D01BF09CFC12
:10A6C000019B0500834208D1002506E030001BF005
:10A6D00098FC07001BF090FC050001A9380019F058
:10A6E0001FF8A379002D02D02A78002A0CD1002B64
:10A6F000CDD1E38A002BCAD0184A31002000FFF7E1
:10A70000A9F9C4E73700DFE7002B1ED0A38A013385
:10A710009BB2A382012B09D1E18A206B002911D0C1
:10A720001AF04CFD0021206B1AF062FD2900200078
:10A73000FFF7CAF8206B01991AF09FFB206B1AF003
:10A7400063FDA4E71AF0BAFBECE7E38A29000133C2
:10A75000E3822000FFF7B8F899E7C046723603009D
:10A76000F0B504000E00056987B002936B1C0393DB
:10A77000AB1C03612900006B17001AF079FC200064
:10A7800018F0D6FF31002000FFF79EF8206B1AF07A
:10A79000B7FC691C206B1AF031FC2900206B1AF001
:10A7A000F0FA206B1AF006FE2669731C2361029BE7
:10A7B0009F4218D1A38B206B013BA3831AF070FC3E
:10A7C000206B1AF0FCFD0399206B1AF0DAFA0C9B4F
:10A7D000002B03D019002000FFF776F83100206B22
:10A7E0001AF0CFFA1BE038001BF00BFC0023059396
:10A7F000236905000193013323610378002B10D1F5
:10A800001BF0FAFB1BF0F8FB029B984224D03C4A59
:10A8100029002000FFF71EF9A38B013BA38307B09B
:10A82000F0BD07008B2B07D11BF0EBFB07001BF0E3
:10A83000E3FB05A918F074FF206B1AF094FB3900B4
:10A840002000FFF741F82121206B1AF095FC019AB6
:10A850000021206B1AF0DEFB28001BF0CDFB0599D0
:10A860000700002948D1206B1AF091FB0025059BB9
:10A87000AB4209D02569206B6B1C236129001AF0BB
:10A8800003FC200018F054FF39002000FFF71CF8EB
:10A89000059B0700002B02D0206B1AF031FC206BC7
:10A8A0001AF053FC059B002B19D00E21206B04F0ED
:10A8B00019FA2900206B1AF064FA0E21206B04F0BB
:10A8C00011FA05992000FFF7A1F820000599FFF77C
:10A8D000AFF8A38B206B013BA3831AF0E1FB31009F
:10A8E000206B1AF08BFB0199206B1AF04AFA0121B8
:10A8F000206B1AF08CF95AE72000FFF787F8B5E7CC
:10A900001A390300F0B587B0039143790400012B95
:10A9100007D1C36A0D001B78002B04D1194AFFF739
:10A9200099F807B0F0BD692103A81BF07EFB0290E7
:10A930000398029B9842F4D005A90B2718F0F0FE6B
:10A94000059B0390019302ABFF183A000199E06A5E
:10A9500018F0FEFB3B780600002B0DD0019A010099
:10A96000E06A18F020FC3378074A002BE0D1290078
:10A970002000FFF76FF8DBE70378042BD8D0034AF9
:10A98000F5E7C046BF360300E43603000237030094
:10A99000F0B587B0039144790500012C09D10191EC
:10A9A00003A869211BF041FB02900398029B984287
:10A9B00001D107B0F0BD05A90B2718F0B1FE02AB1D
:10A9C000059EFF1803903A003100E86A18F0C0FBBA
:10A9D0003B78002B08D10378012B05D0074A019959
:10A9E0002800FFF737F8E0E704703100E86A18F054
:10A9F000D1FB0028D9D00470D7E7C046A0360300A9
:10AA000010B5084B428B04009A4202D1064AFFF768
:10AA100021F8A28BE38B618BD21A206B04F088F9AA
:10AA200010BDC046FFFF00003C36030010B5084BC8
:10AA3000028B04009A4202D1064AFFF70BF8A28B60
:10AA4000E38B218BD21A206B04F072F910BDC04643
:10AA5000FFFF000027360300F7B50B7804001A004B
:10AA60000A3A0E000F2A08D801A9300018F058FE43
:10AA700001992000FEF7DCFFF7BD432B44D1694666
:10AA800030001BF0C3FA01002000FEF71DFF037821
:10AA90000500A22B10D101A91BF0B8FA050028006F
:10AAA0001BF0AAFA019B0700834205D02900200071
:10AAB000FEF70AFF3D00F2E72B78482B16D128005D
:10AAC0001BF09FFA01002000FEF7FEFE0500206B40
:10AAD0001AF089FA0099280018F017FE0028CBD147
:10AAE000214A31002000FEF7B5FFC5E7492BF7D119
:10AAF00028001BF086FA01A918F012FE0199050042
:10AB0000206B1AF059FAE5E7442BE9D108001BF055
:10AB1000B8FA0028E4D130001BF073FA06001BF0ED
:10AB200070FA050001002000FFF796FF28001BF0D7
:10AB300063FA0378A92B9FD0AA2B0ED101A91BF091
:10AB400065FA019B0500834296D020002900FFF79B
:10AB500083FF28001BF050FAF3E7C12BC0D001009F
:10AB60002000FFF779FF87E7B5350300F7B5022628
:10AB70000D00C16A0400097D314005D0344A290026
:10AB80002000FEF767FFF7BD0191297808000A3819
:10AB90000F281DD8280001A918F0C2FDA279E36A88
:10ABA000002A03D01A8B01321A8302E0DA8A0132BA
:10ABB000DA82012601990029E5D06B46DF1C3A00B4
:10ABC000E06A18F0C5FA3B78002B3CD1214AD6E761
:10ABD0001A32914204D128001BF013FA01A9DBE7D5
:10ABE0001A33994223D1A379002BC7D1012728001A
:10ABF000A7711BF046FA03260028DBD128001BF0C2
:10AC000000FA0278E36A0A3A0F2A09D828001A7D66
:10AC100017431F751BF0F5F901A918F081FDC9E76D
:10AC20001A7D280017431F751BF0EBF9F2E7280087
:10AC30001BF0E7F901A918F073FDE36A1A7D1643CA
:10AC40001E750526B6E70223467003709BE7C046D3
:10AC50003D3703004C370300C36A70B51B7804000E
:10AC60000D00072B04D00C4A0021FEF7F3FE70BD47
:10AC70001100280018F049FD002807D00E21206B94
:10AC800004F030F8206B1AF05BFBF0E7290020009D
:10AC9000FEF71AFEF6E7C04623370300C36A70B515
:10ACA0001B7804000D00072B06D0022B04D0174A96
:10ACB0000021FEF7CFFE70BD1100280018F025FD21
:10ACC000061E07D00E21206B04F00CF8206B1AF042
:10ACD00052FBF0E72B78C42B12D128001BF091F91E
:10ACE00001002000FEF7F0FD3100206B1AF0E3F9BF
:10ACF000206B0E2103F0F6FF206B1AF04BFBDAE716
:10AD000029002000FEF7E0FDE0E7C04639390300E6
:10AD1000F0B50D0085B004001100280018F0F5FC16
:10AD2000071E05D00021206B1AF062FA05B0F0BDB5
:10AD30002B784E2B0BD1206B01211AF059FA2900E8
:10AD40002000FEF7C1FD206B1AF05EFAEEE7B32B90
:10AD500061D128001BF055F905001BF04DF9029058
:10AD60000378B62B4DD103A91BF050F9039B029039
:10AD7000984203D09D2102A81BF057F92B784E2B47
:10AD800020D103990298266B1BF02AF9411C300050
:10AD90001AF02EFA29002000FEF796FD206B1AF01B
:10ADA00033FA0127029E039B9E4210D1002FBDD192
:10ADB00031000298246B1BF013F9411C20001AF09B
:10ADC0002EFAB3E729002000FEF77EFDEAE733788C
:10ADD000310020000193FEF777FD019B0600002F54
:10ADE0000BD04E2B05D00F4A29002000FEF732FE73
:10ADF0009CE7206B1AF008FAD5E74E2BD3D10A4A0C
:10AE0000F2E72B7804224E2B00D0052229002000E7
:10AE100018F091FD8AE729002000FEF755FD012179
:10AE2000206BCCE7CD350300F0350300F0B504000E
:10AE30000D00002662711100C56206612A0087B00C
:10AE4000006B03F071FE6279012A01D1EE832E843A
:10AE5000AE683378542B0AD130001BF0D2F80100D1
:10AE60002000FEF731FD206B1AF06AFA2AE02B78F9
:10AE7000002B08D131002000FEF726FD0E21206BAB
:10AE800003F030FFEFE7072B21D130001BF0B4F8BF
:10AE900063790500012B07D100230100A371402233
:10AEA0005F4B200018F0B7FC28001BF0A5F81BF042
:10AEB000A3F801002000FEF707FD206B19F0A2FEA9
:10AEC0000028DBD0206B19F070FE07B0F0BD022B1C
:10AED00017D1012A07D100234732A3713100514B0A
:10AEE000200018F098FC30001BF086F801002000CC
:10AEF000FEF7EAFC2B7D5B07B5D5206B1AF047F80F
:10AF0000BCE7033B032B50D830001BF075F805A9B4
:10AF10001BF07CF81BF070F867790390012F09D1C2
:10AF20000B2202ABD2183900E06A18F011F90223A3
:10AF30000370EF822B78032B20D10021206B1AF0B5
:10AF40004AF92B78062B27D1206B19F0B7FF012186
:10AF50002000FEF7A7FC206B19F0B0FF206B19F062
:10AF6000ADFF0023059A009303993300200019F0E8
:10AF700096F92B78062B00D075E77FE7042B04D1D8
:10AF80000021206B1AF034F9DBE7052BD9D1002121
:10AF9000206B1AF044F9D4E720000121FEF782FC6F
:10AFA0000121206B1AF087F8DBE7012A07D1DE21A7
:10AFB00005AAFF31280018F0CBF80223037005A979
:10AFC000A86818F0ADFBF82120004900FEF76AFCE4
:10AFD000F0212000FF31FEF719FDE989206B19F0FF
:10AFE0004CFFFA2120004900FEF710FDA8681BF075
:10AFF00003F81BF001F801002000FEF765FCDE21DC
:10B000002800FF3118F094F80378022B00D135E7BF
:10B01000DE214288FF31206B19F007FE23E7C0468E
:10B02000BF3E0200B33E0200F8B5164B0400A83341
:10B030001B681600002B24D1056901226B1C0361DB
:10B040002B0019F0B2F8BE210700FF31206B19F078
:10B0500019FE3100380018F058FB061E09D13900DE
:10B060002000FEF731FC330032000121206B1AF082
:10B0700054F90121206B1AF070F92900206B19F0A6
:10B0800080FEF8BD7C2E0020F0B585B005000E00D6
:10B090000192FEF719FC03780400A22B03D101A949
:10B0A0001AF0B4FF0400EB6A1B78072B00D070E0A5
:10B0B000337872780A3B1B021343504A934268D19B
:10B0C0002378472B65D120001AF0DBFF002860D0E1
:10B0D000DE212800FF31FEF7E5FB0121EA6A936AD1
:10B0E000928C002A06D1464A21002800FEF7B2FCC5
:10B0F00005B0F0BD5878084211D059682800FEF715
:10B10000D1FB019920001AF06BFF02280ADC002312
:10B11000286B1A0002211AF000F9200036E0013AEB
:10B120000833DEE720001AF067FF0378492BEED1E1
:10B1300020001AF061FF1AF05FFF0378472BE6D179
:10B1400020001AF059FF07001AF056FF06003800D9
:10B150001AF057FF03A918F0E3FA03990122286BAC
:10B1600019F0C2FE30001AF08CFF0021884203D192
:10B1700030001AF046FF0100002301222800FFF7EB
:10B1800041F920001AF038FF1AF036FF1AF034FFA8
:10B190000400019BA342ABD020001AF02DFF019BBD
:10B1A0000600834224D02378492B21D10378472BF2
:10B1B0001ED120001AF025FF070030001AF061FFB1
:10B1C0000024A04203D130001AF01BFF040003A9A1
:10B1D000380018F0A5FA00220399286B19F084FEB4
:10B1E0002800002301222100FFF70CF93000CDE7F1
:10B1F00021002800FEF768FBCAE7C046C70200002E
:10B200000F360300F0B59BB01500069038220F00F2
:10B210000CA800211E001DF0D8FD069B0BAC5B683E
:10B220000B97236201235B421193069B26711868DA
:10B230001AF0E2FE1AF0B4FE606280001BF04BF8D8
:10B240000022A06200950025069B11001B682000CB
:10B2500018F078FA19F093FC2B0003902063049502
:10B26000626A0792954202D2A268002A41D0002B5E
:10B270005DD10593059A079B934202D00D9A002A4F
:10B2800058D00499039819F07FFC0025149A0D9B5F
:10B290000592954200D213E1002B0CD0169B0EA80C
:10B2A000996818F0DAFC169B0E9A0493DB890B99C7
:10B2B0000D98FDF763F9039819F06EFC18980028B3
:10B2C00001D017F073FC002406981AF0E4FE159BD9
:10B2D0001B681D69149B159803939C4200D219E1C9
:10B2E0001BF016F80D99002900D11BE1080001F0B0
:10B2F000F5F9A16AAA005658002E13D03269002A27
:10B3000010D117F0C6FB737D30610122310020009F
:10B31000042B09D1FEF7BAFB2369049A9A4200D2A2
:10B320000493012301359BE7FFF780FDF4E7002339
:10B330001D0095E70599159B8900CB58002B37D048
:10B340000120998C8C46197D01421BD06446601EF9
:10B35000C000002C16D00226996A09184D78354293
:10B3600029D0002A0ED00F00508816780890506817
:10B370005578099011CF11C2089A0E704A80099A27
:10B380004D704A600021DE249983FF348C451ADC1D
:10B3900000218C4535DC5E68002E09D00021B28C7E
:10B3A00009920A00099881423BDB0020824263D166
:10B3B000059B01335DE7002A02D1012D00D10A006F
:10B3C000013C0838C5E7986ACA0082181878012835
:10B3D00004D15068A04208D10131D7E7157801287F
:10B3E00003D9002D01D1012010701078022803D05C
:10B3F000012550782842EFD0988B451C9D835080C2
:10B40000EAE7986ACA0082181078032807D1012455
:10B410005078204203D1988B5080001998830131D5
:10B42000B7E7B06ACD0040190890007803380128CA
:10B4300012D800240EE09F6AE00038180778042F25
:10B4400007D1089D6F683D004768BD4201D1428029
:10B4500001320134A445EEDC0131A3E79C6AC1004E
:10B4600061180C78042C03D101254C782C4202D0B1
:10B470004C88A4184C8001308445EFDCD98A92B204
:10B480005118D982998B52189A8391E7039B022213
:10B4900021000BA81793FFF7C9FC0D9B0593002B08
:10B4A00004D1032221000BA8FFF7C0FC0D9B0593DC
:10B4B000002B2DD1042221000BA8FFF7B7FC27E0B9
:10B4C000002B00D0EAE6159B0593059AAB009C582B
:10B4D000002C1DD0637D042BD8D1189B0593002B25
:10B4E00004D10499139817F04AFB1890002317937E
:10B4F0000F4B032221000BA81993FEF7C7FA0D9BEF
:10B500000593002B04D1042221000BA8FEF7BEFAFC
:10B510000135BBE6A3001858002801D017F0FFFD45
:10B520000134D7E60A00280017F0BFFA1BB0F0BDBF
:10B5300058980200F8B5124A0E00124B1249904278
:10B540001AD0C4688C4203D0012430602000F8BDBA
:10B55000406B002812D004689C42F0D10500002402
:10B5600047680835BF00EF19BD42EFD2310001CD69
:10B57000FFF7E0FF2418F7E70024E7E70400E5E71A
:10B580004CB202004CA002007DB60000F7B50500E9
:10B590000C00AB68002B0AD0344AE168914206D017
:10B5A000E358002B03D00422EB681A60F7BDA06BB0
:10B5B000002820D06B680430D900062300221943EC
:10B5C000FDF7DAFA002816D0297C4268EB68286873
:10B5D000002904D00100002001F0F0F9E6E700287E
:10B5E00007D02249E5688D4203D021498C4200D022
:10B5F00000692100F0E72B68002B16D1646B002C4A
:10B60000D4D01C4B22681A4F9A420BD12600636893
:10B61000194A08369B189B00F3180193019B346864
:10B620009E4216D3BC42B4D1C0E72A7C002AE5D1A1
:10B630000E4AE1689142E1D00D4A9442DED0186989
:10B64000EA68696801F014FAEB681B68002BD5D032
:10B65000ACE7BC4201D10436E0E721002800FFF747
:10B6600095FFEB681B68002BF5D09FE77DB60000C7
:10B670004CB202004CA00200FFFFFF3FF0B58FB0BC
:10B680000E0005A9019202930700FFF753FF041D66
:10B69000A40020001AF00DFE0500002180C017F064
:10B6A000C7FE22002800103A103000211DF08DFB4B
:10B6B000012E05D1029B1B680393042B00D189E066
:10B6C00007AC0822002120001DF07FFBF22200239E
:10B6D00009A8FF324260E63AFF3A39008260C4604E
:10B6E00003740993FFF752FF079804282FD1059898
:10B6F000029BC468019A3100A04728612800F7F72F
:10B70000D5F8B84266D1EA220023FF32390009A8F1
:10B71000089307930B9309950A92FFF737FF079B4E
:10B72000002B57D00198304336D107AA010019F0F9
:10B7300045F90400294B9C424CD0200016F077FFBD
:10B74000274902002748FCF7ADFE00F0C7FF00289C
:10B75000D4D0019A324306D106AB0121069701F0FD
:10B760000FF90500CAE7019B5D00AD190135AD0079
:10B7700028001AF09EFD2A1F0390029980C01DF038
:10B7800008FB711C039B019A206801F0F9F8050081
:10B7900003981AF0BDFDB1E7019B5C00A4190234C7
:10B7A000A40020001AF085FD22000700079B0299E3
:10B7B00003600393089B083A436008301DF0E9FAE0
:10B7C0003A000199300019F0F9F8040038001AF035
:10B7D0009FFDAFE728000FB0F0BDC046E4B3020004
:10B7E000A339030090AC0200F0B5146889B01700CB
:10B7F000002C0ED1436803AD82686960596B0392D7
:10B80000AC60EF602C74002905D111492800FFF7C6
:10B81000BDFE09B0F0BD0F4B0A689A4210D14B68CB
:10B8200008310E000193019B9C42EED0A300F15819
:10B830002800FFF7ABFE3B68002BEAD10134F2E7AA
:10B840002800FFF7A3FE3B68002BE2D1DDE7C046EE
:10B850004CB202004CA0020010B54A6801491BF02E
:10B86000D9FA10BD9D3A0300F0B58BB005000E006B
:10B8700014000021082268461DF0A7FA00211022BA
:10B8800006A81DF0A2FA202307936B46059508939E
:10B890002968E023002C02D0042C10D1E623FF33CA
:10B8A00005A80693FFF772FE0221009F042F0ED118
:10B8B000220031002869F7F769FA0BB0F0BDFC23CC
:10B8C00005A85B000693FFF761FE0321EDE7381E34
:10B8D000F3D002AB002202950396049401F050F8D5
:10B8E000042CEAD00048E8E7E4B30200F0B5204BAE
:10B8F0008BB08200D35803AF0C0008220021060051
:10B90000380001931DF061FA019B05AD6B601423B3
:10B91000AB600023280021680594EF602B74FFF7CB
:10B9200035FE0398042805D12169300000F0B6FFE8
:10B930000BB0F0BD00280AD0210019F037F8022E14
:10B94000F6D1F7F7C7F8440001202043F0E7022EB4
:10B9500001D00020ECE7E2232168FF3328006B6070
:10B96000FFF714FE3B68002BF3D16400ECE7C04600
:10B9700094B80200F0B55642564103238BB00C0038
:10B980000190002117007642082203A81E401DF0F6
:10B990001CFA0823079303AB0893002305ADF73681
:10B9A000FF36216828002B7405940696FFF7EEFDFC
:10B9B000039B002B09D1002F07D1F733FF332168F8
:10B9C00028006B60AF60FFF7E1FD039804281AD1EF
:10B9D0002069F6F76BFF154BC2689A4211D1002F10
:10B9E00007D02368586819F0C5FF010001981BF0C3
:10B9F00050F980223A4321690198F6F76FFF0BB0A6
:10BA0000F0BD3A00F7E7002805D0210018F0CEFF7E
:10BA100000220100F0E7200016F009FE23000200DA
:10BA2000034901981BF0F6F9E9E7C0466583000079
:10BA30005239030070B504000D000B491BF029F9C1
:10BA4000696800222000F6F749FF084920001BF032
:10BA500020F9A96800222000F6F740FF04492000E1
:10BA60001BF017F970BDC0465B3A030045FC0200AD
:10BA7000A83A030010B5C468002C06D142680449F6
:10BA80000448FCF70FFD00F029FEA04710BDC0469A
:10BA9000643A030090AC0200F0B5154B89B0160073
:10BAA0008200D5580C000C220021070068461DF0CA
:10BAB0008CF9182303A84560836000256B46216834
:10BAC000C36003940574FFF761FD009B042B06D14E
:10BAD00032002169380001F081FC09B0F0BD181E68
:10BAE000FBD06A4629000120029618F067FFF4E7B0
:10BAF0000CB70200F0B51700EE228DB004000393DE
:10BB0000002307A852004260CD3A05ADFF3A0E006F
:10BB100021688260C560037405936B600794FFF72A
:10BB200035FD0598002809D1200016F080FD0C494C
:10BB300002000C48FCF7B6FC00F0D0FD039B042883
:10BB400006D13A003100206900F01AFF0DB0F0BDB7
:10BB5000009332003B00696816F072FEF6E7C046BB
:10BB60008739030090AC0200F0B50D0085B001A943
:10BB700007001600280002AA17F055F900230199C2
:10BB8000029899422CD13C201AF0A5FB2A4B019A2D
:10BB900003602A4B04008360294B4760C360294B34
:10BBA0000361294B4361294B8361294BC361294BB5
:10BBB0000362294B4362294BC362002A06D0029BD1
:10BBC0001968096B0163012A18D94563A66303A9A3
:10BBD0002000FFF7AFFC012813D9214801F0BAFD7E
:10BBE0009A008258D468002C06D152681D491E481C
:10BBF000FCF758FC00F072FD0133C2E71B68436399
:10BC0000E4E7A36B0022181D1849FCF7B5FF051ED9
:10BC10000ED0032243681A400AD11968144B4968B0
:10BC2000994205D1031D0121124818F093FD686067
:10BC3000200005B0F0BDC04658B8020075B900003C
:10BC40007DB60000F5BA0000EDB8000099BA00001A
:10BC5000C746020069B8000047480200FD470200DD
:10BC60002D3A0300043A030090AC02008E0F00004E
:10BC700045020000E0B7020037B50D001C000023AC
:10BC80001100009301220333280006F015FB012D5B
:10BC900004D0032D06D0074801F05CFD2068F6F7BC
:10BCA00005FE3EBD2068F5F775F9A2686168FFF7EB
:10BCB0005BFFF6E7813A03001FB5064B0A000193CC
:10BCC0004B6802938B68010001A8039300F002FF08
:10BCD00005B000BD1CB80200F8B50E0003271349DB
:10BCE000134AB0421CD003003B401BD104688C4275
:10BCF0001AD1406B002814D003689342F1D105009B
:10BD000044680C4B0835E418A4002C192868A54297
:10BD1000E5D23100FFF7E0FF002802D10435F5E756
:10BD20000120F8BD0020FCE71800FAE758B802002F
:10BD30004CA00200FFFFFF3FF0B585B00500019168
:10BD400008008B0717D10B68134A93420BD10123CC
:10BD5000029301AB03930024029E039FA6420DD1E0
:10BD60000E4805B0F0BD0E4A934204D103AA02A9C1
:10BD700017F059F8EFE70B4801F0ECFCA300F95875
:10BD8000094B994206D02800FFF7A6FF002801D1F1
:10BD90000134E3E70548E4E758B80200C4E70200CD
:10BDA0004CA00200CB3903004CB20200CCE70200E9
:10BDB00010B5830703D1054B02689A4202D00448AC
:10BDC00001F0C8FCFFF7B8FF10BDC04658B802002C
:10BDD00064390300F0B58BB0079310AB10CB009023
:10BDE00001911B78062A12D8012A08D93F230B702B
:10BDF0000B0001330193002301990B7001E0002A2D
:10BE0000F9D101209042804140420BB0F0BD009931
:10BE1000002929DA019B01995F1C2D230B708021D9
:10BE200009068C46009B63440093019BFF21099304
:10BE3000009BC90518000840884222D120234E21CA
:10BE4000079AF81C1A4013001143009A540212D1A9
:10BE500049225A403A70462253407970BB70002301
:10BE6000FB70019BC01AD0E7019F002BDDD0390089
:10BE700001370B70D9E74124634039707B70B9708A
:10BE8000EDE7002C00DA06240199013A7D1A551BD2
:10BE90002022079911430291672940D1002C00D13B
:10BEA000CEE1002B79D0A64A934200D9D4E0A5492F
:10BEB00000980EF021F9431E9841002300263030EF
:10BEC00003932033059004939F4B039A0099D05815
:10BED0000EF008F9002808D0049B039AF6189B4B33
:10BEE0000098D1580EF07EFD0090049B5B100493E7
:10BEF000039B04330393182BE6D115330393009A65
:10BF00008F4B93425DD38F4900980EF0F5F80028CF
:10BF100051D0002E7CD0FE239B05009351E0002BD6
:10BF2000C1D1029B662B38D1631CAB4200DBAC1E37
:10BF3000029B651C049300231E0003930593E343B7
:10BF4000DB171C40049B652B00D0EEE0651C002332
:10BF50000693069B9D424CDD00980FF04FF87B1C2A
:10BF60000893030030333B70059A069B934205D13A
:10BF7000002C03D0BB1C08932E237B700FF05EF8BF
:10BF8000011C00980EF060FE71490EF02BFD069B1F
:10BF9000009001330693089FDBE7631DAB4200DB93
:10BFA000AC1F029B652B00D1AFE0002504930395E5
:10BFB00005952E00C3E7009865490EF013FD013684
:10BFC0000090029B662B03D0672B39D1042E37DCFF
:10BFD000059B3B70029B672B01D1731EE418631C09
:10BFE000AB4200DBAC1E002C15D166230137039455
:10BFF0000493029B662B00D0B0E0012E00DDDDE053
:10C00000544900980EF078F8002800D0ACE0D5E054
:10C010002B2303937FE72E23250030227B70BB1C4C
:10C02000013E1F00002E76D0002D05D1039501237F
:10C030005B42059367334DE01A70013D0133EFE732
:10C040006B1FA3426CDC029A672A66D01300AC1FF8
:10C0500000250493059572E70023002603932033FF
:10C0600004933A4B039A0099D0580EF031F8002807
:10C0700008D0049B039AF618334B0098D1580EF061
:10C08000B1FC0090049B5B100493039B0433039367
:10C09000182BE6D12E4900980EF02EF8002805D076
:10C0A00000982D490EF09EFC01360090029B662BF5
:10C0B00012D1AE4214DAA3190133AB4204DBAC1B3C
:10C0C000023C631C00D10024002335190393013581
:10C0D00005966633049332E7029B652B00D0B1E0EE
:10C0E0006B1FA34200DCAC1F2B2300250393059597
:10C0F0003A33EFE7231DAB4200DB6C1F029BA642E5
:10C1000000DBA3E0731CE41ADEE7029B0025049326
:10C110002B2303934CE7039689E71C00029B97E7C8
:10C120000025029B059504930CE7049B672B00D028
:10C130000DE7251E00D00AE701252C0007E7C046C1
:10C14000FFFF7F3FF8FF7F3FB0B80200C8B8020092
:10C15000000020410000A040CDCCCC3D3E490098DD
:10C160000DF0CAFF002824D030217B1E1A782E2A19
:10C170004FD010003038092842D901330193019B78
:10C180001B78302B15D1019A52782E2A45D104996B
:10C19000662942D001994B70039B0A702D2B3AD12E
:10C1A000013E002E3BD03B00019A9A423AD3312304
:10C1B0001370029B672B01D1002C39D1039B002BFC
:10C1C00019D02022079B0A2113401A00452313434C
:10C1D0003B70039B30007B700DF034FE0A210DF0A4
:10C1E00017FF3031B97030000A210DF011FF3C1DEE
:10C1F0003031F970270000233B70099BF81A04E6E0
:10C20000392A02D001321A70B8E7019A19709342A4
:10C21000B5D0013BAAE70136C5E70137C3E72B23B9
:10C220000393C0E75A1E117819701300BCE71F0072
:10C230007B1E1A78302AFAD02E2ABFD11F00BDE704
:10C2400001242EE6029B672B00D153E704932B2396
:10C2500000250393FEE6C0460000A040F8B50700A5
:10C2600008680C0016F026FE05006068F6F744FD2D
:10C270000600022F0AD9A068F6F700FC0200310080
:10C28000280018F03CFB19F01BFAF8BD004AF6E74D
:10C2900040420F00F0B5486887B00F00F6F7EEFB9C
:10C2A000041E02DA002001F091F8BB68164A0193DF
:10C2B0009D186B1E9D41010002A81AF035FF049ED7
:10C2C0002200002130001CF080FD3868EDB2C30769
:10C2D0000AD433002200290019F0BFF902A90B4843
:10C2E000F4F700FE07B0F0BD43102000042C00D985
:10C2F00004200749019F00228F4200D0221AB21861
:10C3000029001AF001FCE9E75AECFFFFA0920200B5
:10C31000A6130000F0B50C0087B0012203A96068E5
:10C32000F6F766FDA3681349039A8B420DD10126E7
:10C33000049976424C1E01911419049900200D00B5
:10C34000002D05D119F0D7F90DE014000126F4E70E
:10C35000094F013DB84208D908481B18581E8341AF
:10C36000D8B219F06BF907B0F0BD27780002384356
:10C37000A419E5E7A6130000FFFF3F005AECFFFFFA
:10C3800070B546007508041C291C281C0EF020FE00
:10C3900000280BD11649281C0DF0A4FE002808D057
:10C3A0001449154816F03EFF00F098F9134801F0C3
:10C3B0000DF8002C11DA002E12D0FF23DB05E31854
:10C3C0009C22D20593420BD903F03EFA211C0500B2
:10C3D000043015F0B1FA280070BDE30DDB05EFE77E
:10C3E000201C0EF00BFE012540000543F3E7C0467C
:10C3F000FFFF7F7FBA3A030064AB0200D33A030029
:10C40000F0B50C00002585B0110020001E0000953D
:10C4100002232A0005F050FF0120AC422BD08442B9
:10C4200031D13068204226D103230340AB4203D1EF
:10C430001C4A016891421ED01B4A0240062A06D0BF
:10C44000002B0DD10268194B92699A4208D103A9B9
:10C45000F5F7D6F900231A000399F6F77FF80AE0FA
:10C46000032302001A40022A07D1FF22D2058018B6
:10C470009843FFF785FF05B0F0BDF6F7FFFA0123FB
:10C4800040001843F7E703A93068F5F7B9F904004D
:10C490007068039FF6F7F2FA2B00020039002000C3
:10C4A000DBE7C0462CB90200070080FF9D1D00009D
:10C4B000F8B51F000B4B15005918013909780DF01C
:10C4C00037FC00260400B74204D0013003210DF0F0
:10C4D0002FFC0600281E01D01CF0CBFC0334A4194D
:10C4E0002018F8BDAA3A0300F0B58DB00A9214AA3C
:10C4F000147815AA127806000F000792DA0742D5C1
:10C500005D100023002D01DA2D236D420693139A4E
:10C51000079B12992020FFF7CBFF3B6805908342D1
:10C5200004D219F0C6FE059B30603B6000213768DD
:10C53000059BFB185A1E11708D4240D00A3C09928F
:10C5400008920B94129928000DF078FC0B00303300
:10C55000092901D90B9B5B18089A541E2370079B6D
:10C56000002B48D000282DD0A7422BD2099B1B1BA3
:10C57000032B05D1079B013C2370A74222D20994CB
:10C5800005000894DEE79A0712D1244A19689142FF
:10C590000ED1079A02940392139A39000192129ACB
:10C5A00000920A9A19F020F8040020000DB0F0BDA6
:10C5B0000023326813700A9A34681360F5E79C1EF2
:10C5C00030232370139B002B05D018001CF051FC66
:10C5D000201A87421FD3069B002B04D0BC4202D9ED
:10C5E000069B013C23703368059A9B181B1B0A9A13
:10C5F000013B1360D9E7A742E4D20028C0D1E1E7AC
:10C60000C2540133139AD25C002AF9D1069B04006C
:10C61000002BE5D1E7E70023F4E7C0462CB9020080
:10C620001300144A10B50400934204D101222000E3
:10C6300000F0D4FE10BD104A934201D10322F6E768
:10C640000020072CF6D10D4A1A40062A0ED09A0770
:10C65000F0D11A680A4CA24208D00A4CA24205D076
:10C66000094CA24202D0094CA242E3D10A000720A1
:10C670001900DDE7C4E70200CCE70200070080FFF5
:10C680000C9A0200A09202004CA0020088E702006F
:10C69000C4600561466187614146C16149460162E6
:10C6A00051464162594681626946C1627146816064
:10C6B00000490847BDC600000020C046024B9A68EA
:10C6C00002609860002070477C2E0020024B9A6820
:10C6D00012689A607047C0467C2E00200E4A93680C
:10C6E000002B01D116F0AAF8196858609160181C47
:10C6F000C468056946698769C1698846016A8946CF
:10C70000416A8A46816A8B46C16A8D4681688E4637
:10C7100001207047FEE7C0467C2E002070B504F073
:10C720008DF90F4C0F4B0025A3620F4BE56263633D
:10C7300023002563A83303210C481D60A56403F082
:10C740003FFC0B4E0121300003F03AFC3000094A57
:10C75000094919F091F826606660E56570BDC0462C
:10C760007C2E0020FCA9020044A00200B42E002070
:10C77000C82E0020760F0000860F000070B506243A
:10C78000134EC3001C437368002205002100181DCE
:10C79000FCF7F2F9021E18D1F06D002807D0043022
:10C7A0002100FCF7E9F9002801D0406870BD0022A3
:10C7B00021000848FCF7E0F9021E06D12A000649CC
:10C7C0000648FBF76FFEFFF789FF5068EEE7C046AB
:10C7D0007C2E0020689D0200E63B0300B0AA020008
:10C7E0000A4B10B5040018685B6898420AD006210D
:10C7F000E300194304300022FCF7BEF9002801D001
:10C80000406810BD2000FFF7B9FFFAE77C2E00203A
:10C81000074B10B5D86D002801D1064810BD043073
:10C8200000220549FCF7A8F90028F6D04068F5E792
:10C830007C2E0020309C0200DE0E00000A00C100A9
:10C84000062010B5024B0143186819F015F810BD09
:10C850007C2E0020062110B5034BC0000143186850
:10C8600019F014F810BDC0467C2E00200A00C1004B
:10C87000062010B5024B0143586818F0FDFF10BDAB
:10C880007C2E0020062110B5034BC00001435868E0
:10C8900018F0FCFF10BDC0467C2E002037B5050007
:10C8A0000C00062806D10800F6F726FA00280DD05D
:10C8B0002C483EBDCB071BD54B10042816D80DF0D5
:10C8C00023FA03154E4E0700002BF1D02648F0E75F
:10C8D000C0221206934204D18020C00518F0F0FE59
:10C8E000E7E75B425B0001201843E2E7DB43F9E73F
:10C8F00002281AD11D4B0B40062B08D08B0714D1F0
:10C900000A681B4B92699A420FD1486802E0C80836
:10C9100019F026F8002806D101A92000F4F752FBEF
:10C92000019904F079F84300DDE72000F5F7BEFF38
:10C930004369002B0DD10F4BAD002000ED5815F0D1
:10C9400076FE2A0003000C490C48FBF7ABFDFFF70D
:10C95000C5FE2100280098470028AAD1EBE708006F
:10C96000A7E7C046C4E70200CCE70200070080FF4B
:10C970009D1D000094B80200723C030090AC0200C0
:10C98000F7B50400019116001F00F5F78FFF056948
:10C99000002D09D1200015F04AFE06490200064884
:10C9A000FBF780FDFFF79AFE3B0032000199200063
:10C9B000A847FEBD8739030090AC0200F8B50E0011
:10C9C00015001C00930714D113681E4A934202D12C
:10C9D0006B682360F8BD1C4A934207D1002802D03F
:10C9E000F5F764FF06006B6848C4F3E7174A934203
:10C9F00001D12560EEE75A68022117008F431449E0
:10CA00008F4202D013498A42F3D1002817D1124A2B
:10CA100093420BD0114A934208D0114A934205D059
:10CA2000104A934202D0104A934208D10C2019F0C8
:10CA300040FC0E4B4660036085602060CAE72560BD
:10CA40006060C7E7E0B70200A4B7020058B8020070
:10CA5000450200001A0200003CEA020078EA0200E7
:10CA6000B4EA0200F0EA02002CEB020070B9020006
:10CA7000F8B500231360536006000D001400F5F7AD
:10CA800015FFF92307005B009D4205D1836A002B47
:10CA900002D00F4B48C4F8BDFB69002B04D0220024
:10CAA000290030009847F6E7B86B0028F3D006213C
:10CAB000ED00294304301A00FCF75EF80028EAD0A4
:10CAC0004268230039003000FFF778FFE3E7C046F3
:10CAD000F89C020070B5160004000D00FFF7C8FFB7
:10CAE0003368002B15D10B4EA3070BD10A4B2268DC
:10CAF0009A4207D12B00626808493000FBF7D2FC4C
:10CB0000FFF7ECFD200015F092FD2B000200044918
:10CB1000F3E770BDE0A7020058B80200FF3B030036
:10CB2000263C030073B504000D001600F5F7BEFEA9
:10CB3000C369002B09D004220196009229006A469D
:10CB400020009847009B002B0AD0200015F06FFDB5
:10CB50002B00020003490448FBF7A4FCFFF7BEFDCD
:10CB600073BDC046263C0300E0A7020073B5040075
:10CB70000D00F5F79BFE174B426A06009A4226D03D
:10CB8000002D03D1102019F094FB0500736A002BCF
:10CB900012D1E6216A46FF312000FFF769FF009BB2
:10CBA000002B0FD1200015F042FD0B4902000B486D
:10CBB000FBF778FCFFF792FD29002000984700283A
:10CBC000E7D076BD29006846FCF742FDF9E7200072
:10CBD000F7E7C0465B260200953B030090AC0200DD
:10CBE00037B50400F5F762FE856A002D02D02000FB
:10CBF000A8473EBDF9216A4649002000FFF738FFEB
:10CC0000009B002B05D06A462900280017F0D6FEAD
:10CC1000EFE7200015F00BFD034902000348FBF786
:10CC200041FCFFF75BFDC046C73B030090AC020030
:10CC300030B505008FB003F0A3FE2800F5F736FEEF
:10CC4000846A002C05D02800A047040020000FB003
:10CC500030BDF9216A4649002800FFF709FF009B13
:10CC6000002B16D002A8FFF713FD002807D16A4653
:10CC7000010017F0A3FE0400FFF728FDE6E7039B81
:10CC800008491868FFF728F80028DFD10398FFF754
:10CC900025FD280015F0CBFC034902000348FBF7F3
:10CCA00001FCF4E7DCAB0200C73B030090AC0200E0
:10CCB000F0B513688FB00793002800D073E004002C
:10CCC000131D0393FF220B00090A13401140019327
:10CCD0004B000693069A019B05919B18039A9B00B3
:10CCE000D2580492039AD3185F68381E09D00020E6
:10CCF000BB0706D1944B3A689A4202D1380018F02B
:10CD0000B8FD059B1818049B4600002B50D1019BD1
:10CD1000581C83199800009319F0CBFA26000500DF
:10CD2000002C01D001260460019BB0009A00281855
:10CD300003991CF02EF8019B9B190293029B98000B
:10CD4000059B2818DA00019B9900039B59181CF0D9
:10CD500020F8029A069B944663440193002F12D058
:10CD600003243C4000D0A9E0774B3A689A4200D0B7
:10CD7000A4E0380018F095FD0323060000937368C3
:10CD80009C4200D27DE0019B029A02999A1A5208B5
:10CD90002B000798FFF7F4FD0400280019F0B8FAFB
:10CDA00020000FB0F0BD130008330393546889E7E7
:10CDB000049B9B072FD1049B644A1B68934202D0BB
:10CDC000634A934227D10AAA09A90498F5F7F8FE05
:10CDD000099B581C019BC01883199800009319F0F7
:10CDE00068FA26000500002C01D001260460019B92
:10CDF000B0009A00039928181BF0CBFF019B0A99F9
:10CE00009819099B80009A0028181BF0C2FF019B0B
:10CE1000099A9B1890E7019B181D831998000093AD
:10CE200019F047FA26000500002C01D00126046005
:10CE3000019BB0009A00039928181BF0AAFF019BE0
:10CE40000AA99B1904980293FFF790FE029B049095
:10CE50009C000498FFF7ECFE061E00D16EE7009BD5
:10CE6000029A934207D8D900280019F040FA050029
:10CE7000009B5B000093029B2E510133029304340C
:10CE8000E7E7B368E700D859002815D0042813D085
:10CE9000009B184205D12F4B02689A4201D115F030
:10CEA000BAFB019B019A9B00E85002320192B268E2
:10CEB000EB18D7197A685A60013460E70AAA264944
:10CEC0003800FFF707FE00210AAA080017F076FDD8
:10CED0000021FFF74BFE019B03909E000398FFF794
:10CEE000A7FE041E00D14EE7019B009A01339A422F
:10CEF0000BD853000093042B01D204230093009B12
:10CF00002800990019F0F3F9050003231C4207D10A
:10CF1000104B22689A4203D1200015F07CFB0400DC
:10CF2000E6210AAAFF313800FFF7D4FD0AAA002142
:10CF300001200C9417F042FD019BAC510233019388
:10CF4000AB1958600836C9E774C202004CA0020051
:10CF500088E702000C9A02006B02000070B50C001A
:10CF600086B0160083071CD10368204A934202D082
:10CF70001F4A934215D102AA01A9F5F721FE019B90
:10CF8000A3422CD31BD80023029DA000A34201D1B1
:10CF900006B070BD9900421A043AAA580133725083
:10CFA000F4E702A9FFF7E2FD002305000193019BCE
:10CFB0002800A34206D3FFF73BFE0028E8D022005A
:10CFC0000C490EE0FFF734FE002808D0019A0A4908
:10CFD000A31A5B189B00013298510192E7E7019A6E
:10CFE00006490748FBF75EFAFFF778FB4CA0020002
:10CFF00088E70200B33C0300FFFFFF3F903C0300C3
:10D0000008AD0200F7B5FF240E00090A26401500FE
:10D010000C40830731D10368384A934202D0384A22
:10D0200093422AD101AA6946F5F7CAFD009833193F
:10D0300083425BD883009C46002301999A00A34257
:10D040000FD1B400801B0919C01AAD1819F008FDE2
:10D05000019B28601C190023013601339E4207D131
:10D06000F7BD6746BF1A043FCF590133AF50E5E71C
:10D070009A0051426158A950EFE70021FFF776FD71
:10D08000002307000093009BB34218D3002108003F
:10D0900019F0E6FC06003800FFF7CAFD011E1BD19F
:10D0A000B168A14222D3A3008A00EB181E60AA181F
:10D0B000091B9D4214D1300019F0EEFCD0E7380076
:10D0C000FFF7B6FD002811D0009AB31A1B199B0078
:10D0D000013258510092D6E7300007F07DF8DAE7C8
:10D0E000F468D01A2058043B1860E2E7009A05491A
:10D0F0000548FBF7D7F9FFF7F1FAC0464CA002004C
:10D1000088E70200903C030008AD0200F0B591B042
:10D110001D0006000C001700F5F7C8FB334B9842C2
:10D1200007D12B003A002100300004F0E3FA11B0DF
:10D13000F0BD826A2E4B002A08D09C4230D13000CC
:10D14000904728600028F2D00120F0E79C4227D1C8
:10D15000F92101AA49003000FFF78AFC019B002B4E
:10D160000DD1D72101AA49003000FFF7B3FC039489
:10D1700001AA0021012017F021FC2860E4E704A89F
:10D18000FFF786FA002807D101AA010017F016FC64
:10D190002860FFF79BFAD7E7059B2B600220C6E7C4
:10D1A000002CDED13800F5F781FB1249FEF794FD23
:10D1B00001AA00280ED010493000FFF759FC019B4E
:10D1C000002B10D001AA2100200017F0F7FB2860E7
:10D1D0002000ACE709493000FFF74AFC019B002B17
:10D1E00001D00397C4E72F60D8E7C04634D20200CD
:10D1F000E4B30200D0A8020019020000CD02000032
:10D2000010B50400FBF794F9002808D00023200093
:10D210001A001900FFF7B4FB0400200010BD200025
:10D2200016F004F80028F8D10249034815F0FAFF77
:10D23000F2E7C046483C030090AC02007FB5C30053
:10D2400006201843054B01900491052001A9029383
:10D2500003930592FAF72AFB07B000BDE4B302007E
:10D260001423F0B58DB000AFFA1805000C00FFF7DD
:10D27000FFFBBB69002B06D022002C492C48FBF792
:10D2800011F9FFF72BFA786900284CD1280015F026
:10D2900065FE0028F0D01423F821FA182800490070
:10D2A000FFF7E6FB10227869B918F4F7A9FAB8601D
:10D2B000200018F05AFB6A463E69B968731C7B600F
:10D2C000C318FB600E33DB08DB00D31A9D466D46A6
:10D2D000320028001BF05DFD2E23AB557B6820003B
:10D2E000EB18BB6018F046FB0600200018F03DFB71
:10D2F00031000200B8681BF04CFDF968280003F00B
:10D30000DBFBC300062018430A4B10223B627B6202
:10D31000094BBA18BB620123FB620B33F861D118C9
:10D320000520FAF7C3FABD460DB0F0BDB13B0300CE
:10D330000CA90200E4B30200CCE70200F0B5174CE0
:10D340000F00616895B003912168060008A8049158
:10D3500062602360FFF79CF9051E06D0039B0998C5
:10D360006360049B2360FFF7B9F933683A0031002A
:10D3700005A8019304F06EFC2B002A00019905A872
:10D38000FDF740FF17F00BFB0500FFF79FF92800A2
:10D39000039B6360049B236015B0F0BD7C2E0020CE
:10D3A00010B5040000F004FD031E054802D0054935
:10D3B00017F040FB22000449FBF774F8FFF78EF9E1
:10D3C00074AA0200043B03002D3B0300010010B5CA
:10D3D000014817F02FFBC04608AD0200F0B58BB036
:10D3E00004900F000392202803D191420FD0AF4E3A
:10D3F000BFE0049B1B2B01D01E2B0DD103993800DD
:10D40000F5F7EAFA049B002803D01B2BEFD1A84EB6
:10D41000AFE01B2BFBD1EAE7049B212B3FD1039804
:10D42000FBF786F8002806D00399380015F004FFB2
:10D430000028ECD1DBE70324039B1C4005D1039AB1
:10D440009C4B126805929A4223D0049B9A4A9B00F7
:10D4500038009C5815F0EBF80500039815F0E7F834
:10D460002B000090220095499548FBF71BF847E1F7
:10D47000039AA300D3189D682800FBF759F80028E9
:10D4800000D158E12900380015F0D6FE0028BED1A1
:10D490000134039B5B680593A342E9D8A7E7012603
:10D4A000314200D116E1039B4D101E4000D1E7E050
:10D4B0005C10049B1D2BC8D818000CF02FFC1E001C
:10D4C00028002A002D0045004C004E0050005D0051
:10D4D00066007B008300B4001E0028002A002D0097
:10D4E00045004C004E0050005D0066007B0083004C
:10D4F000CC00D000C6FFD400D80025432E00700019
:10D500000300734000D5B6E00126064331E06540D4
:10D51000F4E72C402600F2E7002C02DA6948FFF716
:10D5200055FF1F2C08DC684B2341AB4204DBC023B2
:10D530001B062341AB4205DDE917280018F0B1F8BE
:10D5400007004BE0A540D9E7002CE7DB1F2C00DDEE
:10D550001F242541D2E72E19D1E72E1BCFE721004A
:10D560002800FAF751FC0028E6D1012665436D003A
:10D570002E4330000BB0F0BD002C00D1DDE02100C7
:10D58000280015F07DFD0600B9E7002C00D1D4E09D
:10D5900028000DF053FD051C20000DF04FFD011C6F
:10D5A000281C0DF047F8032302269843474B0643F7
:10D5B000F618DEE7002C00D1BFE02100280015F0AE
:10D5C0004FFDE0E72F00002C2ADA28000DF036FD91
:10D5D0000323022798433D4B0743FF183800F5F714
:10D5E00065F98369002B00D12FE7039A390004986D
:10D5F000984756E001231C4206D039003000FAF764
:10D6000003FC002898D17E43012C00D177E7390034
:10D6100038006410FAF7F8FB002800D08CE77F434D
:10D62000002CE7D16BE7002C00D186E0002102201E
:10D63000F9F720F821000600280015F021FD012748
:10D6400040003843B0602100280015F009FDB840C3
:10D650000743F7608DE7A54200DAD8E6C7E6A542A2
:10D6600000DDD4E6C3E6A54200DCD0E6BFE6A54275
:10D6700000DBCCE6BBE6300018F022F8060078E7C5
:10D680000323039A1340022B24D1114B1340062B82
:10D6900020D028000DF0D2FC039A011C0498FBF75F
:10D6A000E9F8061E00D064E7CFE6C046C4E70200F2
:10D6B000CCE702004CA002000CB70200703B030054
:10D6C00090AC02005B3B0300FFFFFF3F0000808047
:10D6D000070080FF049B1F2B00D07FE70398F5F71E
:10D6E000E5F883690400002B0CD1636A002B11D18B
:10D6F000039814F09CFF134902001348FAF7D2FE76
:10D70000FEF7ECFF3A00039904989847061E00D0F4
:10D710002FE7EAE706A90398FFF728FA040020009C
:10D72000FFF786FA002800D161E63900F5F754F9D1
:10D730000028F4D06BE6039587E60449044817F007
:10D7400079F9C046953B030090AC0200E40D03005C
:10D7500044AD0200010010B5014817F06BF9C04656
:10D7600090AC0200F8B504000D0017001E0000295F
:10D7700008D01868F5F79AF86368834202D0054824
:10D78000FFF7E8FF33003A002900A068FFF7F8F838
:10D79000F8BDC046EC3A030001214000014310B53A
:10D7A000024815F038FDFEF799FFC04628AB02008D
:10D7B000010010B5014817F03DF9C046ECAA02007F
:10D7C00010B5034A0349044819F024FB034810BD6F
:10D7D000B33D0300590D030084E80200E4B30200E6
:10D7E00010B5034A0349044819F014FB034810BD5F
:10D7F000DB3C0300590D030084E80200E4B302009F
:10D80000F7B50600194D0C00280013F023F931007C
:10D81000174813F0A5F8174813F01CF9164813F031
:10D8200019F9FF239B00E61821787F2901D0A64231
:10D8300006D1280013F00EF9104813F00BF9F7BDCC
:10D840006278A37850290CD80D48475C0D48405C9D
:10D85000019300923B0002000B4813F081F804345E
:10D86000E2E70A4813F07CF8F9E7C046AA3F030054
:10D87000D73F0300DF3F0300683F0300863F0300FC
:10D88000940C0300430C03000040030023400300FA
:10D89000F0B51D0087B006001A4817000C0013F001
:10D8A000D9F82900184813F05BF8184813F0D2F89B
:10D8B000174813F0CFF8AD006519AC4204D11148F8
:10D8C00013F0C8F807B0F0BD3878A278049020684B
:10D8D00023780003400E0390E0789B060009029035
:10D8E00020883178C004400E0190E0789B0E00073C
:10D8F000000F00901209074813F032F80434013683
:10D900000137DAE7AA3F0300F73E0300243F030094
:10D91000563F0300883F0300F7B50020214A224EFE
:10D9200012783368111D4900CC5A5F18598801904C
:10D93000A020C00584466405640D4C431B49A41215
:10D940000968787807270500BD43F82D1DD001250B
:10D95000C00885402800A1256746ED0001327851B6
:10D96000D2B2101D4000C55A1F186D0558886D0DA4
:10D9700068438012001BE4D00A4C2270019A002AEE
:10D9800002D00A4A33601160FEBD6046084A5C68F6
:10D990008450002903D001220B00002101920A00CB
:10D9A0000C00DEE7312E0020BC2A0020C02A002017
:10D9B0000C05000010B572B600220F4B18681A60F3
:10D9C00062B6904210D10D4B0D4A1B680D48934230
:10D9D00000D010001A7802705A8842805A6842605B
:10D9E000002219788A4200D310BD510044185918FA
:10D9F000098901322181F4E7C02A0020BC2A0020D5
:10DA0000C42A0020F42A0020044B054A1A6000238F
:10DA1000044A1360044A13707047C046BC2A0020B1
:10DA20004CBA0200C02A0020312E002010B5782206
:10DA30000249022000F068FF10BDC04619D900005D
:10DA4000421E084BFF3A10B504009A4207D8FFF770
:10DA5000B1FF054B241144801860002010BD012047
:10DA60004042FBE740410F00C02A0020044B1B68E6
:10DA7000002B01D1034B1B68588800017047C0463A
:10DA8000C02A0020BC2A0020F7B53D4A04000D0042
:10DA90000B00914200D913008022D200D31A0193C7
:10DAA000FFF788FF0122A24046680092164207D184
:10DAB0002300A0210327C133FF339B00C9055F501A
:10DAC000002703789F4206DB002D01D0132B0BD9D2
:10DAD0002C4B1860F7BD391D490042185278D20806
:10DAE000A24243D00137EDE7009A191D324342604C
:10DAF000019A490055050A5A6D0DD20AD2022A43ED
:10DB00000A525205E400520F4118144301334C707D
:10DB10000370851C012225E0009A013BDBB296438D
:10DB200003704660BB42F4DD04335B001B5A0B52AA
:10DB3000EFE72F00131D5B00195A2E894905490D87
:10DB4000531E1C1D6400245A6405640D8C4204D9C4
:10DB5000FC88023F7C81013BF3D205335B001E52FF
:10DB60000132023503789A42E3DBB1E7002DD3D0CE
:10DB7000019B5A050B5A520DDB0ADB021343D6E711
:10DB8000FF030000C02A002070B500210400FFF749
:10DB90007BFF00210D4B18680578A94200DB70BDA2
:10DBA0000B1D5B00C3185A78161CD208944201D092
:10DBB0000131F2E70822524232435A700123A02178
:10DBC000A340034AC9058B50E9E7C046BC2A0020A0
:10DBD0000C05000010B50C0017F0AFFD631E1842D5
:10DBE00007D00200230003490348FAF75BFCFEF765
:10DBF00075FD10BD4440030008AD020010B54A6831
:10DC00000249D20019F006F910BDC0466C4003006D
:10DC100070B50B0006001400101E0FD071681800BC
:10DC2000042A0ED1FFF7D6FF7368012B03D0022B15
:10DC300005D0006800E0007817F042FD70BD008854
:10DC4000FAE7FFF7C7FF05002000F4F743FF72680B
:10DC500003000548012A03D0022A03D02B60EDE718
:10DC60002B70EBE72B80E9E7E4B30200F7B52D4F0B
:10DC7000B43701972B4A2C49FC32536C8B4200D8A5
:10DC8000F7BD0325043B53641A68264B501CAC3384
:10DC90001E6804008108715C2C4064002141831AD5
:10DCA000294001300229F4D00326019912010968A4
:10DCB0001B018A181B499B08002BDBD00F2014681E
:10DCC000044229D119480068A04225D80D00B83572
:10DCD0002D68A54220D9241A200900900800AC30F4
:10DCE0000068A409009D0419207835406D00844621
:10DCF0002841304001280FD13700AF403D00674632
:10DD00003D4325700D00FC356C6C094FBC4206D2BA
:10DD1000201D686400982060013B0432CCE70C00B1
:10DD2000BC34F8E77C2E00203C2F0020302F002050
:10DD3000BC2F00200F23994370B506000D00081A70
:10DD400041210BF0F5FF0F4C02002300B0331860A7
:10DD500023002100AC331E608301EB1AB4310B6049
:10DD600023003000B83300211D601BF02EF8802303
:10DD7000FC345B020122A36400235242E364226567
:10DD8000636570BD7C2E0020A222034952008B5A8D
:10DD900001338B527047C0467C2E0020A2220349DB
:10DDA00052008B5A013B8B527047C0467C2E00209C
:10DDB000A223034A5B00D05A431E9841C0B2704769
:10DDC0007C2E0020F7B50400032589004318019339
:10DDD000019B9C4200D1F7BD0F232168194229D134
:10DDE000184B1A00B43212688A4223D81800B8308F
:10DDF000006888421ED9891A1A000F093800AC320F
:10DE00001268890951180A78284040009446024156
:10DE10002A40012A0ED12E0086403000664630434B
:10DE200008701800FC30416C074EB14206D20B1D41
:10DE300043640F60FFF71AFF0434C9E7BC331A606C
:10DE4000F8E7C0467C2E0020BC2F0020A22210B58F
:10DE500008485200835A0100013383520300002214
:10DE6000FC33BC310A60DA64034A27215A64FFF7A5
:10DE7000A9FF10BD7C2E00203C2F0020F8B5032602
:10DE80002E4C00252200BC321368AB4213D1022273
:10DE90001900032794462200B03212689200914282
:10DEA0002AD323000022FC335A654532FF32A35A9D
:10DEB000013BA352F8BD23001560214AFC335A648C
:10DEC0002300B0331B689B009D42D9D22200AC32A4
:10DED0001268AB08D35C2A00324052001341334031
:10DEE000032B07D12200FC32536C191D51641D60B5
:10DEF000FFF7BCFE0135E3E72000AC3000688A087C
:10DF0000801802780D0016003D406D002E413E4005
:10DF1000022E09D0032E0BD0012E07D13B00AB40BF
:10DF20009A430270012301E0002BF7D10131B2E7DF
:10DF30006346AB409A4302700023F7E77C2E002033
:10DF40003C2F0020334BF0B51A001900B832B43121
:10DF500009681268521A1900B0331E680260032360
:10DF60000022AC310F68140011009C4642608260B0
:10DF7000C260026142618261B60065468B08FB5C4B
:10DF80000D406D002B4165462B404568012B33D079
:10DF9000002B2BD0022B32D001318E420AD06546A5
:10DFA0008B08FB5C0D406D002B4165462B4001D07A
:10DFB000012BE2D1012C26D1056901350561856966
:10DFC000A54200D284618E4201D0012BD5D1C36815
:10DFD000934200D2C2608E4206D143681B01436067
:10DFE00083681B018360F0BD0022C6E784680132AC
:10DFF000013484601C00CFE701354560FAE7013544
:10E0000045600134C8E7022CD9D145690135456125
:10E01000D5E7C0467C2E0020F7B50F3003090193E9
:10E0200002D100242000FEBDA223474A5B00D35A40
:10E03000002BF6D14733FF33D35A5E425E41002BAB
:10E0400007D0414BFC33DA6C1B6D9A4201D306F0CA
:10E0500071F8002430213F273B4A3B4BB032126815
:10E06000FC339446384A5B6DAC3210689C4505D849
:10E07000002ED6D106F05EF80136EBE70325C25C30
:10E080002A4231D1019D0134A5422ED89B00191B93
:10E090004E1C5A1C012C03D12B4C9708FC3467658D
:10E0A000B40800190324270037407F00A446023C2F
:10E0B000BC40077802313C43234F0470AC378B429D
:10E0C00034D22149204DB431FC350C68E96C330160
:10E0D0008C46E418019B921B63441201002120002E
:10E0E000EB641AF072FE9DE700240C252A4206D14B
:10E0F000019D0134A54203D89B000133C7E70024EA
:10E100000A4206D1019D0134A54203D89B00023387
:10E11000BDE70024BA4306D1019A0134A24203D8D4
:10E120009B000333B3E7002401339FE73C68880872
:10E130002018644602250C406400A5402C00057898
:10E1400001312C430470BAE77C2E0020A22230B5A6
:10E15000164B52009A5A002A26D1002824D01A00C1
:10E16000B4321268801A1A00FC32546D0109800919
:10E17000A04200D25065AC331800032204688B081B
:10E18000E3180C00150014406400A5401C78013110
:10E19000AC431C7004688B08E35C0C001440640002
:10E1A00023411340022BE9D030BDC0467C2E002015
:10E1B0000F2203000240002070B5824228D1154C86
:10E1C00010002100B4310968994221D82000B830EC
:10E1D000056810009D421BD9AC345B1A24681909EC
:10E1E0009B09E55C0800032318404000054110002E
:10E1F0001D40012D0CD14D1C2E00AA08A25C1E4012
:10E2000076003241681A1A400135022AF4D0000122
:10E2100070BDC0467C2E0020F0B585B007000D0013
:10E220000292002807D101002800FFF7F5FE060042
:10E23000300005B0F0BD002903D1FFF787FF2E00A5
:10E24000F6E70F2100260140B142F1D153480E00FC
:10E250000300B4331B68BB42EAD80200B83212682C
:10E26000BA42E5D9FB1A1A0900920200AC321268D0
:10E270009B090192D25C0323009C23405B001A415E
:10E2800003231A40012AD3D14233FF33C35A002B50
:10E29000CED129000F310909B0308C460168032620
:10E2A00089000391210014000131039A914212D296
:10E2B00001988A08825C08003040400002413240E8
:10E2C000022A02D101340131EFE7002A03D10133E0
:10E2D000E2186245F7D3644501D13E00A8E76445E2
:10E2E00021D9009B032663441900009B0800E21813
:10E2F000AC239C46294B9C44634605001B6884085C
:10E300001C19330035406D00AB40257801309D432A
:10E3100025709042F0D1214B8908FC335A6D91420F
:10E32000DBD25965D9E71B19634523D303250226A0
:10E330001A49009BAC31E3180191009A62449A4259
:10E3400009D86346191B090120010A003818002169
:10E350001AF03BFDC1E70199180009689A088A186C
:10E360003100284040008140080011780133084303
:10E370001070E2E7029E002E00D159E7002128002C
:10E38000FFF74AFE061E00D152E7220139001AF0BB
:10E3900000FD3800FFF7DAFE4AE7C0467C2E002079
:10E3A00010B58CB005A8FFF7CDFD079B0A4C039371
:10E3B0000093059A069B0949200018F02BFD089B45
:10E3C000099A01930B9B06490393009320000A9B33
:10E3D00018F020FD0CB010BD84E80200BB40030023
:10E3E000DE400300F8B5434E434F3300B4331A68A0
:10E3F0004249380018F00EFD00243300B0331B688A
:10E400009B00A34223D93F2214422CD13200250085
:10E41000AC3210680321AA08825C294049000A41F5
:10E4200003210A4202D10135AB42F3D12A1B7F2AD4
:10E4300012D992093249380018F0ECFC2C003F2325
:10E440009C433300B0331B689B00A34204D83800C0
:10E450002C4918F01EFCF8BD2B4B22011A402B4909
:10E46000380018F0D7FC3200AC321268A308D35C35
:10E470000322224052001341032213403A32022B5E
:10E4800031D03032032B2ED03F3A012B2BD1330029
:10E49000B4331B682201D3581D4954228B4222D029
:10E4A0001C49083A8B421ED01B49083A8B421AD0AD
:10E4B0001A490F328B4216D019498B4213D0194991
:10E4C000123A8B420FD018498B420CD017490532B3
:10E4D0008B4208D01649043A8B4204D015492632A3
:10E4E0008B4200D11B3A1449380018F093FC0134D8
:10E4F00083E7C0467C2E002084E802007C400300B5
:10E5000097400300654F0300F0FF0F00B340030086
:10E510004CA0020088E7020074C202000C9A0200BC
:10E52000A092020030B30200F4B2020088B00200F0
:10E5300000EA020098B1020082000300C379024899
:10E54000002B00D101487047CCE70200C4E702006D
:10E5500010B5F4F7A7FE014810BDC046E4B30200B1
:10E5600010B50868F4F79EFE004810BDE4B3020041
:10E5700073B50D00022836D1012601A96868F3F7AA
:10E580003FF976423400019BC318834212D101A99E
:10E590002868F3F735F97342734162426241DBB296
:10E5A000D2B20199F4F7C2FF002820D110491148D6
:10E5B00016F040FA0278722A01D0772A06D1611C3F
:10E5C0000ED1723A544254410130DEE7622A01D042
:10E5D000742A05D1711C03D1743A56425641F3E7AF
:10E5E0000548FEF7F3FE012676423400CFE776BDFC
:10E5F0001B04030028AB02002341030007224368E9
:10E6000004481B791340044AD35C002B00D0034814
:10E610007047C046CCE70200DA000020C4E70200E1
:10E6200010B50124037A05499B005A580448224238
:10E6300000D10448A243CA5010BDC046242B00207C
:10E64000CCE70200C4E7020070B5037A064C05006F
:10E650009B001859400817F033F801222B7A9B00D1
:10E6600019590A401A5170BD242B002030B5A2223E
:10E67000A025D200ED05AA580723CA401100164C68
:10E680000340E056421EC90700D5421C022A0ADC9C
:10E69000002082421ADB1149CD5C854201D0C8546A
:10E6A0000230E25430BD072A09DD0C2A10DC0B4988
:10E6B0000320CD5C002DF4D10238C854F1E707499E
:10E6C0000320C95C0029ECD10800EAE70200E8E772
:10E6D00003200C22E5E7C046E2000020DA0000201B
:10E6E0001D4B70B559791879FFF7C0FF022805D185
:10E6F0001A490B689A1C012313430B60184B597974
:10E700001879FFF7B3FF022805D114494B689A1C0A
:10E71000012313434B60134C2000FAF79DFB124D6D
:10E72000A84203D161792079FFF7A0FF0F4C2000A8
:10E73000FAF792FBA84203D161792079FFF796FF9F
:10E740000B4C2000FAF788FBA84203D161792079AD
:10E75000FFF78CFF70BDC0461CA30200242B0020D5
:10E76000BCA20200ACA2020020B20200F4A202008D
:10E7700004A30200072203791340014AD05C7047CA
:10E78000DA0000208022044B52001A600123034A61
:10E790001360034A1360704700E100E00C8C0040F6
:10E7A000008000408022054B5200DA67044BFF3A9C
:10E7B0005A600022034B1A607047C04604E100E033
:10E7C000008000400C8C004070B5002501261E4BD7
:10E7D0001E4C1D601E4B18601E4BE650C046FFF7D6
:10E7E000E1FF1D4B1D4AE660E25002221C4BFF2058
:10E7F000E5500433E25008339218E250C1238022DE
:10E800009B001203E250053BFF3BE550C22440222F
:10E81000144BA400195981430A4380211A510C3426
:10E820001A5909061202120A0A431A51C022043464
:10E83000195981430A431A51802212041A60802216
:10E8400052041A6070BDC046D02F002000800040E6
:10E850003C2B0020FC0F00004C050000701700004E
:10E860000405000000E100E070B51F4C1F4D636C13
:10E87000002B0AD0002363641D4B1B689847A82314
:10E88000DB00EA5800018018E850A36C002B09D087
:10E890000023A364164B5B689847164B0001EA58A7
:10E8A0008018E850E36C002B0AD00023E364104B7F
:10E8B0009B689847A923DB00EA5800018018E850BC
:10E8C000236D002B0ED000230B4A2365AB580B4958
:10E8D0005B18AB500A4A1368063313608022094B59
:10E8E00012045A6070BDC046FC80004000800040A9
:10E8F0000C000020440500004C05000070170000CB
:10E90000D02F0020FCE100E0F7B50191032823D8C7
:10E91000134B8000C758C223124D9B00EF500123B8
:10E9200044192364A8230F210F4EDB009C46E358B3
:10E93000AE59921BD218D3170B409A1801990B4B62
:10E940001211C150C1239B00EF50634600200132D9
:10E9500012019619E650FEBD01204042FBE7C04679
:10E9600084BC0200008000404C0500000C00002028
:10E9700003280BD8074B8000C158C223064A9B00CE
:10E98000D150064B064AC250002070470120404239
:10E99000FBE7C04684BC0200008000400C00002061
:10E9A000494A020010B5024B1B68984710BDC0468B
:10E9B0003C2B002010B50024054AA1008B58002BE9
:10E9C00002D00020885098470134042CF4D110BDA7
:10E9D0002C2B0020074A89008B58002B06D1885029
:10E9E00080211800044A49045160704701204042C8
:10E9F000FBE7C0462C2B0020FCE100E0F8B50E0040
:10EA000005001400FFF7CEFE330003272B433B42E3
:10EA10000BD1BC4209D9A208310028000AF0AEF897
:10EA20002300BB43ED18F6183C40002C04D0220014
:10EA30003100280019F0D7FD80220449D2008B58FC
:10EA4000002BFCD0FFF79EFEF8BDC04600E0014061
:10EA5000F0B5060000248BB0194B1A48E15804F0B9
:10EA600001F803AFE05104341C2CF5D11423002429
:10EA7000734301930025AB00F958134816F0ACFC22
:10EA80000135300014F025FE072DF4D1013DAB0017
:10EA90000D48F95816F0A0FC300014F01AFE013DA4
:10EAA000F5D20134082C03D100F0D4FD0BB0F0BD39
:10EAB00001231C42DED1019814F00BFEDAE7C046B8
:10EAC000F0BC02002CB502001C00002010B519207B
:10EAD000FFF7BEFF004810BDE4B3020070B515009B
:10EAE000040016F016F82A000249200015F0CFFFA6
:10EAF00070BDC046F54A020070B543790D00002490
:10EB0000032B06D9836A074C9200E41AC369D358D1
:10EB1000E418032115F0EEFF447024120570847090
:10EB200070BDC046FD7F0000F7B500230400617191
:10EB300083608371E260036101330F00150043615C
:10EB4000032906D80121836949429A00C0691AF055
:10EB50003CF90023A3622362AA8BEB8BD218002A14
:10EB600000D10132384E2000310015F090FF2A8C80
:10EB70003100200015F08BFFE3682000197D15F0AF
:10EB8000B2FFE3682000997D15F0ADFFE368200037
:10EB9000197E15F0A8FFE3682000997E15F0A3FF09
:10EBA000042F27D1636A226A31009A1A200015F0D7
:10EBB0006EFF3100EA89200015F069FF3100AA8953
:10EBC000200015F064FF0026AB8CB34217DCFF2158
:10EBD000200015F09EFF042F35D1EA8A2B8B0237D7
:10EBE000D31801930023019A9A422CD0AA8C0021B9
:10EBF000009223E00221200015F068FFD9E7AA6AFD
:10EC0000F300D3181A78032A03D19978200015F05D
:10EC100080FF0136D8E70126A86ACA00821850781A
:10EC200030420AD05088984207D15268D200606BB7
:10EC300099003A430A500133D5E70131009A8A42DC
:10EC4000E9DC0222F2E7F7BDCD4A0200F7B5234B1B
:10EC50000500A8331B680191022B0DD847698F422C
:10EC60000AD2836A0269CF1B9C1A3B00234304D15A
:10EC7000AB6A2B61019B6B61F7BD062F01D90F2C8D
:10EC800018D900941F2C01D91F230093009B002644
:10EC90009C4203D83E00032F00D9032601212800FF
:10ECA00015F014FF009A730113430370009BBF1B00
:10ECB000E41ADAE70A4B3E009F4200D91E00022107
:10ECC000280015F003FF702233091340F03A224365
:10ECD0001343037046700094E8E7C0467C2E002082
:10ECE000FF07000070B50D000121040015F08FFF33
:10ECF0000E2D14D00F2D17D010210D2D10D017214F
:10ED0000200015F006FF0322A36A04210333934376
:10ED1000A362200015F0EEFE044B036003E0112116
:10ED2000200015F0F6FE70BD1221F9E728900200D0
:10ED3000F8B5174F05000C0016000F40002A1AD135
:10ED4000110015F064FF23040FD53221280015F0BF
:10ED5000E0FE3221280015F0DCFE3221280015F0FB
:10ED6000D8FE3221280015F0D4FE3A0035212800C3
:10ED7000FFF7C2FEF8BD3A004621FFF7BDFE7F2334
:10ED8000210A99433143C9B2280015F0C2FEF1E7C8
:10ED9000FF7FFFFFF0B5124B87B003AD40C90138CC
:10EDA00000930195032303F0B7FA68680D4F1E2402
:10EDB000B84202D014F07EF844B2A8680023B842EA
:10EDC00002D014F077F843B270680399437104716C
:10EDD00009F00EFF70680AF075FA380007B0F0BD50
:10EDE000C0BD0200E4B3020030B5124B8BB003ACDF
:10EDF00020C9013800930194032303F08DFA616860
:10EE000006A818F091F9039B089A5900237A0093F9
:10EE10006868079B08F088FA021E05D00649074873
:10EE2000F9F740FBFDF75AFC06A90548F2F75AF836
:10EE30000BB030BDD8BD02003041030028AB02004A
:10EE4000A092020030B5114B89B002AC20C9013844
:10EE500000930194032303F05FFA012205A960687F
:10EE6000F3F7C6FF029B059A5900237A009368685E
:10EE7000069B08F069FA021E05D005490548F9F716
:10EE800011FBFDF72BFC044809B030BDF0BD0200BA
:10EE90004241030028AB0200E4B302000021F8B5B0
:10EEA0004768080017F0DCFD08250600B1223B6822
:10EEB000D2009D508022002092001900985001221B
:10EEC000FC319A6088605A61104A8868002803D132
:10EED000002A19D0013AF8E70024A24204D00C4AD3
:10EEE0009C5863425C41E4B238000AF0EBF9002C14
:10EEF00005D001216B001943300005F06DF9013593
:10EF0000782DD3D13000F8BD1400EDE710270000B4
:10EF1000C404000010B5040001F018FD074B020006
:10EF20001B690749074817F075FFFFF739FA012CED
:10EF300001D1FFF757FA044810BDC0467C2E0020CF
:10EF40005541030084E80200E4B3020010B5F3F772
:10EF500095FDF5F763F8014810BDC046E4B3020023
:10EF600010B5FEF71BFF014810BDC046E4B3020018
:10EF700010B5FEF709FF014810BDC046E4B302001A
:10EF800010B586B0040005AB04AA03A902A801F0DD
:10EF900003FE059B029A0193049B064900930648D1
:10EFA000039B17F037FF012C01D101F031FE03481C
:10EFB00006B010BD6A41030084E80200E4B3020019
:10EFC00010B5084C002805D1A834236801305B0037
:10EFD000184310BD0868F3F751FDA83420600248BB
:10EFE000F7E7C0467C2E0020E4B3020001220100B6
:10EFF00003001140100000290CD10800990709D125
:10F000001B68054910008B4204D00448181A43427B
:10F010005841C0B27047C0462CB90200D4E7020084
:10F020000023FA21094A89001360094A1370094A2A
:10F030001360094A1160094A1370094A111D083208
:10F04000D3670122CB67074B1A707047442B00200F
:10F05000322E0020402B002018000020332E0020EC
:10F060007C2E0020342E002010B5084B084A197859
:10F07000002907D1916C002902D0FFF7D1FF10BD04
:10F0800030BFF4E700221A70F9E7C046342E0020A2
:10F090007C2E0020837F0248002B00D1014870475E
:10F0A000CCE70200C4E702000023A022E02110B553
:10F0B00083770C4BD2050902D1500B48F9F7EAFED1
:10F0C0000A48F9F7E7FE0A48F9F7E4FE0948F9F7B4
:10F0D000E1FE0948F9F7DEFE0848F9F7DBFE0848CB
:10F0E00010BDC0460C0500000CA3020014A30200D2
:10F0F00024A302002CA302003CA30200B4A202003D
:10F10000E4B30200F8B5164C2368002B07D1482061
:10F1100019F0D5FD0500134908F0F8F925601248EB
:10F12000124902680B68D21A0123312A04D96233CA
:10F1300093429B415B420233002201260C4D2E700C
:10F140002F78032FFCD101329342F8D10368206855
:10F150000B6018F081FF430001201843F8BDC04642
:10F16000482B0020D8BE0200D02F00204C2B0020BE
:10F17000352E002030B50D4C87B02378012B13D1EC
:10F180000B4B02221D680621002302A818F0EDF89F
:10F19000082204A9684619F0FCFD039B029A280086
:10F1A00008F030F90223237007B030BD352E00205F
:10F1B000482B0020A02010B51049C0054B7F5A1CD9
:10F1C000002B09D14C8C0E4BA3430E4C03510E4B1C
:10F1D0004A775200D05A0FE010335B00CB185C889E
:10F1E000A123DB00C450092AF1D10120FFF7C0FBA5
:10F1F000FFF7C0FF0120404210BDC0461C000020A8
:10F20000F01F00000C050000F4F6020073B5041EA8
:10F2100009D11A4D2B78002B2CD01949194816F01A
:10F22000DBF82C7073BD184D2B1DDE6FF3F73EFB22
:10F23000164B2100984214D0154B2340062B05D0C5
:10F24000A30712D1134B22689A420ED101A92000C4
:10F25000F2F7D6FA019B012B0CD1007817F01FFBB7
:10F260000100300016F0B8F8DCE70B490B4813F04A
:10F27000D9FFA864FFF7D4FED4E7C046332E0020A0
:10F28000A8E402001C0000207C2E002008E50200FB
:10F29000070080FF0C9A02001E42030090AC02009F
:10F2A000F7B5A123A021214AC905DB00CA500123DB
:10F2B000C27F0D3293401E4A8B50C37F01920133AF
:10F2C000DBB2032B2FD0C3770200030000212233CF
:10F2D0003632198002339342FBD10424C17F154F8B
:10F2E0004D000522EB5D7E195343134A7678D318FF
:10F2F0009B190126A640B44662461B7901345B0087
:10F30000C3185E8C063516435E840D2CE9D10122AC
:10F310000D318A40A023A121DB05C9005A50828EFD
:10F3200001995A50F7BD0023CDE7C046F01F0000F9
:10F330000C050000B24103001C00002070B5394BE1
:10F340008CB01A78022A07D1A0223749D2008A58F5
:10F35000012A07D003221A70344DAB7F002B03D152
:10F36000FFF708FF0CB070BD2800FFF799FF304A87
:10F37000304913680968063313608B4207D30024B1
:10F380002D4B14601B78012B0FD0022B45D000238E
:10F390002A8C6B77FF33FF331A42E1D0E1222749F1
:10F3A000D2000120FFF7B0FADCE7254E331DDB6FFA
:10F3B000002B04D033000833DB6F002B02D1FFF7A2
:10F3C0002FFEE4E7FEF7E0FC6846FDF761F9002850
:10F3D0000CD11C4B1868FDF703FC0400FDF776F90F
:10F3E000FEF7DCFC2000FFF711FFD0E7FEF7D6FCAC
:10F3F000019B15491868FCF76FFC0028F2D10198B1
:10F40000F3F754FA114B984203D11149114817F000
:10F4100001FD019B0024B364E4E70F49280015F0C7
:10F42000DBFFCCE7352E0020007000401C000020E0
:10F43000402B002018000020322E0020B5F10000E3
:10F440007C2E0020442B0020DCAB020074AA0200BA
:10F450001609030084E80200A8E40200F0B50024C5
:10F4600085B0154D02930AAB1B782E1D0700083599
:10F470000800210001920393F467EC67FDF776FB27
:10F480000E4B019A18600E4BF7671A60029A0D4BEB
:10F49000E8671A700C4B1C70FDF7A2FBFFF7B6FE75
:10F4A00001220A4B1C600A4B1A70039BA34201D035
:10F4B000FFF7DAFD05B0F0BD7C2E0020442B0020C4
:10F4C00018000020332E0020342E0020402B002076
:10F4D000322E0020F0B50024384B8FB01D1D0833AC
:10F4E000DC67374BEC6709AD80C9013801950093A3
:10F4F000052302F011FF6B68099C049307942B7B92
:10F500002E7A05932B7C20000393FFF76FFD2D4D82
:10F51000002806D103232340022B09D12C40062CBE
:10F5200006D007AB002201212748F1F75BFD0790C9
:10F5300007980540062D05D0830730D1224B02687D
:10F540009A422CD108A9F2F75BF9089B002B23D033
:10F55000012B0DD1002E0BD1039B002B08D100787D
:10F5600017F09DF907900799380015F035FF13E063
:10F57000079803F05FFB079009AB1B7C002B03D0BF
:10F580000798F5F739FF0790059B049A00930799B0
:10F5900033003800FFF762FF0C480FB0F0BDF3F7FF
:10F5A00085F90B4B9842E7D1002E02D1039B002B2B
:10F5B000D9D007A90120F7F75DF8DCE77C2E002001
:10F5C00084BF0200070080FF0C9A0200E4B302002F
:10F5D00008E5020070B51B4B8AB005AD40C9013883
:10F5E00000930195052302F097FE059C20000494EA
:10F5F000FFF7FCFC002807D103232340022B0AD18C
:10F60000114B1C40062C06D004AB002201210F48F0
:10F61000F1F7E8FC049003A90498F2F7F1F82A7CCA
:10F620002B7B03990092059A03F0EEFA2B7A0100E6
:10F630000093300000236A68FFF710FF04480AB007
:10F6400070BDC046ACBF0200070080FF0C9A0200EC
:10F65000E4B302000022074B10B51A70064B0232C9
:10F660001A70064B064A1B68063B1360FFF7FCFC4A
:10F6700010BDC046342E0020322E0020180000207D
:10F68000402B002010B5FFF7E5FF014810BDC04634
:10F69000E4B3020010B5042901D8042A02D90948AC
:10F6A000FDF794FE092B01D90748F9E705246143CA
:10F6B00041188A18137101229A40038C1343038462
:10F6C00010BDC046480903002B420300F8B5486846
:10F6D0000C000D68F3F7D2F90600A068F3F7CEF935
:10F6E0000700E068F3F7CAF93A0003003100280088
:10F6F000FFF7D0FF0048F8BDE4B3020010B50429BD
:10F7000001D8042A02D90448FDF760FE05235943B5
:10F7100040188018007910BD4809030070B5104CDE
:10F72000050021000F48F9F7CBFB21000E48F9F73F
:10F73000C7FB21000D48F9F7C3FB21000C48F9F77E
:10F74000BFFB21000B48F9F7BBFB21000A48F9F782
:10F75000B7FB15F0C7FE01230848AB7770BDC04664
:10F7600000B202000CA3020014A3020024A30200B2
:10F770002CA302003CA30200B4A20200E4B30200E6
:10F7800070B50D00F3F7DEF9041C2800F3F7DAF981
:10F79000211C0BF059FA051C15F0B1FE011C281CA8
:10F7A0000BF020F9211C0AF0ABFD0323020002201C
:10F7B0009A43024B1043C01870BDC04600008080C1
:10F7C00010B515F09CFE0323020002209A43024B61
:10F7D0001043C01810BDC0460000808010B5074C13
:10F7E000002802D00868A04203D106F05DFC20008A
:10F7F00010BDF3F76FF906F077FCF8E7E4B3020009
:10F8000010B50400F3F7ACFAF3F738F9002803DC7D
:10F810000021064815F00EF906F020FC15F050FF07
:10F82000042201002000F3F7B1FA10BD84A9020000
:10F8300010B50400082016F03CFD024B4460036044
:10F8400010BDC046C0C0020010B5102016F031FD3A
:10F850000400034B08C011F0F6FF200010BDC046A5
:10F860002CB9020070B50C00052804D80AF04CFA37
:10F8700006030C04131C0024200070BD8B680E4C82
:10F88000002BF9D10D4CF7E7081D12F043FC0124C1
:10F8900040000443F0E7FFF7D7FF211D05000430C7
:10F8A00012F05EF92C00E7E7FFF7CEFF211D0500FF
:10F8B000043012F065F9F5E7CCE70200C4E7020076
:10F8C00070B5050083070CD1104B02689A4208D12D
:10F8D000FFF7BAFF291D0400043012F036F92000AA
:10F8E00070BD2800F3F7CAF8C0231B06984206D162
:10F8F00080200021C00515F0D4FE0400EFE70124AC
:10F90000C317C018584040000443E8E72CB9020070
:10F9100007B5C30701D540100EBD043001A9F1F7AA
:10F9200007FA002801D00198F6E70249024815F0CD
:10F9300081F8C0464442030064AB0200F0B58BB0CE
:10F94000019001200D00170008402BD04B1002221F
:10F9500003A904A811F0AFFF04AEFB072BD57B1061
:10F96000022203A904A811F0A6FF04AD019B092BF4
:10F9700001D0162B3FD16B68002B68D0300012F0FD
:10F9800024FC041C280012F020FC011C201C0AF09E
:10F9900051FE032302249843704B0443E4182000D3
:10F9A0000BB0F0BD03240C4023D16D4B0A689A4282
:10F9B000F5D10E1DD1E703231F4205D1684A3968EE
:10F9C000914201D13D1DD1E73B40022B0CD1654B4B
:10F9D0003B40062B08D0300012F0F7FB3A00011C28
:10F9E0000198F8F747FF04E03A0029000198FCF776
:10F9F00017FE0400D3E7019B182B00D98AE0FFF71C
:10FA000023FF040001980AF07FF9444A3E50500D4C
:10FA100013191F72336572444A3E50500D13191F5B
:10FA200072336500201D2A00310012F041F9B6E75B
:10FA3000201D2A00310012F075F9B0E7201D2A00C0
:10FA4000310012F0A2FAAAE76B68002B03D14649F5
:10FA5000464814F0EFFF07A811F0F5FE2B00320026
:10FA6000201D07A9F0F7FEFF07A811F0F1FE96E7A9
:10FA70006B68002BEBD007A811F0E5FE211D2B00D1
:10FA8000320007A8EEE7201D2A00310012F08BF9A2
:10FA900085E7201D2A00310012F001FA7FE7201DC2
:10FAA0002A003100F0F768FF79E73800FFF730FFF0
:10FAB000021E02DA2E48FDF789FC019B201D310051
:10FAC000032B01D0102B02D1F0F7EEFE67E712F006
:10FAD0008EF864E76B68002B03D02B78DB0700D52A
:10FAE00079E7201D2A00310012F0D2FA57E76B683F
:10FAF000002BACD0FFF7A8FE0700211D04302B001F
:10FB00003200F0F7AFFF07A9022007970894F6F735
:10FB1000B1FD6EE72900300011F0F4FF03000198F9
:10FB200000241938042800D939E7124C0AF0ECF8FF
:10FB30000308120B0F00002B00DB30E70E4C2EE702
:10FB4000002BFBDC2BE7002B00DD28E7F6E7002B82
:10FB5000F4DA24E7002B00D021E7EFE700008080F3
:10FB60002CB90200070080FFE40D030044AD020041
:10FB70005B3B0300C4E70200CCE70200044B886053
:10FB80000B60044B08004B600023CB607047C046FD
:10FB90006C9802009F570200044B0B60037A0B71B4
:10FBA000436808008B600023CB607047F0C10200FF
:10FBB00010B504000C2016F07CFB034B446003607E
:10FBC0000223037210BDC0462CC2020010B50430DF
:10FBD00013F049FC004810BDE4B30200002803D034
:10FBE000012808D0002005E007224B680448934311
:10FBF00000D1044870474B68DB085B001843F9E705
:10FC0000CCE70200C4E702000B6870B506000D00E7
:10FC1000181D49681400F8F7AFFF002802D04368A8
:10FC2000002B10D1022E08D1094B022C06D1696895
:10FC3000084813F0F0FAFCF751FDAB68012C00D135
:10FC40004360180070BD022CFBD100224260F8E72F
:10FC5000E4B30200C0A9020070B504000D000B7AE5
:10FC6000164A9B0086B0995817F013F814492000E3
:10FC700017F00FF8134B02AA02932B7A0126137187
:10FC80006B68019304930023059302A815F091FD7E
:10FC9000051E05D10C49200016F0FBFF06B070BD13
:10FCA000002E03D10949200016F0F3FF012229009C
:10FCB0002000F2F713FE0026E7E7C04668C2020004
:10FCC000BA420300F0C10200BD42030045FC02003D
:10FCD000F0B513681400012287B00F680D00009280
:10FCE000D9080223060002F0E7FA022E12D10323FC
:10FCF0006868034018D101682A4AC968914213D143
:10FD00002A68904206D0059305A9686815F032FD6F
:10FD1000061E01D100253EE0381D01223168F8F7AA
:10FD20002BFF73684360EFE70021FCF71FFF039090
:10FD30000398FCF77DFF0028ECD00021FCF716FFAC
:10FD40000500FCF775FF02902800FCF771FF060024
:10FD50002800FCF76DFF029B002B03D0002E01D082
:10FD6000002802D01048FDF731FB381D012202990E
:10FD7000F8F702FF4660DBE7A368EE009E193168E2
:10FD8000002907D0042905D0381D0122F8F7F4FE18
:10FD90007368436001356368AB42EDD8034807B030
:10FDA000F0BDC0461D00010094420300E4B3020010
:10FDB00030B5002585B001A90400019515F0DAFCE5
:10FDC000A84203D109490A4814F034FE636802A925
:10FDD000083B63600368029343680393042328C0CD
:10FDE0000220F6F747FC05B030BDC0467142030063
:10FDF000C0A90200F7B50C0015001B280DD0002388
:10FE00001F2808D1081D00222900F8F7B5FE2C4B49
:10FE1000002800D12B4B1800FEBD03222B001340FD
:10FE2000114225D1284922688A4221D1002BF1D1E3
:10FE3000296891421ED1009301936946200015F074
:10FE400099FC01A90700280015F094FC0600002F7A
:10FE500031D00028DED031683868F2F7BDFD0028C7
:10FE6000D8D071687868F2F7B7FD0028E5D1D1E7FE
:10FE7000002BCFD1154B2A689A42CBD16A686368B0
:10FE8000534007229343C5D1019301A9200015F0E7
:10FE900071FC061E01D10A4BBDE7281D0022316806
:10FEA000F8F76AFE0028B5D041687068F2F794FD53
:10FEB0000028EAD1AEE7024B0028ABD1ABE7C04641
:10FEC000CCE70200C4E70200B0C2020074C2020024
:10FED000F7B50B681C4A04000D00934203D05A6822
:10FEE0001A4916F097FF1A49200016F0D2FE002397
:10FEF0000127019301A9280015F03CFC061E0CD136
:10FF00001449200016F0C5FE2B680F4A934203D017
:10FF10001149200016F0BDFEF7BD002F03D10F4997
:10FF2000200016F0B6FE012231682000F2F7D6FC60
:10FF30000B49200016F0ADFE012271682000F2F797
:10FF4000CDFC0027D6E7C04674C2020090420300F1
:10FF500043FC02005E070300A002030045FC020010
:10FF6000613A030010B504000C2016F0A2F9034B0F
:10FF7000446003600023037210BDC0462CC202001F
:10FF800010B504000C2016F094F9034B4460036094
:10FF90000123037210BDC0462CC2020010B504300C
:10FFA00000220C00F8F7E8FD002805D121000348E5
:10FFB00013F031F9FCF792FB406810BDC0A90200B4
:10FFC00010B5024B08C013F033FA10BD74C2020022
:10FFD000F8B50E00070000217068FCF7C7FD0E4C55
:10FFE0000500022F00D9B4687068F2F761FE00289E
:10FFF00009D115F008FC06002800FCF719FE011EC7
:020000040001F9
:1000000003D13000F8BD4010F3E7331D0122180082
:10001000F8F7B2FD4460EFE7E4B30200F0B5070083
:1000200089B000201E000D00019215F0ECFB0E4B74
:10003000040007609F4203D1042302791343037134
:10004000019B2B430DD03368AA00B218019905A873
:100050000394049313F0FAF9681C05AA03A9FFF7A7
:1000600037FE200009B0F0BDB0C2020010B50C0090
:10007000002A03D115F00AFC0A480EE0042A0DD12B
:1000800004300022F8F778FD002805D12100064849
:1000900013F0C1F8FCF722FB406810BD15F0ECFB33
:1000A000EAE7C046E4B30200C0A9020010B50100AF
:1000B00083880120A0229840044BD205D050CA88E2
:1000C000083117F0E3F8024810BDC0460C050000E7
:1000D000E4B30200EFB5070008001500F98802003C
:1000E00000233868F2F7A2FD03267043002D14D0D8
:1000F0003F18042D14D101237A7A01A952001A4322
:1001000001923A7A30009A401A430292BA7A9A409F
:1001100013430393F6F7AEFA0500280004B0E0BDE0
:10012000310001AA2800F2F76DFD019B1868F2F773
:10013000A5FC019B06005868F2F7A0FC019B050096
:100140009868F2F79BFCFF2E03D8FF2D01D8FF28FB
:1001500002D90448FDF73AF93D727E72B872024D39
:10016000DBE7C046FA420300E4B30200F7B51C0027
:10017000002300930233080011001A0002F09CF8DB
:10018000206812F097FE47B26068F2F777FC041E11
:1001900002DC1048FDF71AF90326300060430830EE
:1001A00016F087F80C4BA2B20500878072430360FB
:1001B000C4800021083018F008FE3B00A022C133A3
:1001C000FF33D2059B009E500123BB40034928000A
:1001D0005350FEBDE142030044C302000C05000081
:1001E000032210B50400C38800215A43083018F0D8
:1001F000ECFD2000FFF75AFF004810BDE4B30200F9
:100200000523020070B5094C094D20684343094895
:100210009B189B0018582B682260C0180F231940A8
:1002200009012860F7F7BCFD70BDC046502B0020C7
:10023000442A002080C30200A839030000B508004A
:1002400006292ED809F060FD040A10161B2128008B
:100250009A18E223DB00D218107800BDC432920055
:10026000D05C8006800EF8E7C4329200D05AC004F9
:10027000400EF2E7C4329200D0580003F8E7C432CF
:1002800092009A1890780009E7E7C43292009A1811
:10029000D0780007000FE0E7C43292009A18D078B7
:1002A000F1E7024B024A00201A60D6E70400002062
:1002B00009430300A83910B504000800062949D8ED
:1002C00009F022FD040A141F2A343F00E221A2187B
:1002D000C9005218137010BD3F210B401800C432E2
:1002E0009200135D8B4303431355F4E77F21C4321F
:1002F000920019401948135B890103400B431353C3
:10030000E9E77F21C432920019401059144B490388
:1003100003400B431351DEE70F20C4329200A218B2
:100320001901937803400B439370D4E70F210B40DE
:100330001800C4329200A218D3788B430343D370C1
:10034000C9E70F20C4329200A218D1781B010140E6
:100350000B43F4E7034B044A1A60BCE73FE0FFFF9E
:10036000FF1FF0FF0400002027430300F0B5D2B2C6
:1003700085B00E000293072113000B40013BDBB256
:10038000042B02D9294C2A4D25608A431F02002ADA
:1003900024D1284B3578C45C274B2409E443E4B2CC
:1003A0002D1BDB19EDB2039308276319039ADBB207
:1003B000D35C5A00D2B25BB20192002B33DA1A211D
:1003C0000320013FFFB2FFF71BFF019B002FF0D17D
:1003D0000134E4B2002CE7D135701AE0D443174958
:1003E000E4B2CE5C0825144B1B19DB5D5A00D2B277
:1003F0005BB20192002B0FDA05210220FFF700FF0C
:10040000013DEDB2019B002DF0D10134E4B2002C8E
:10041000E8D1029805B0F0BD31000120FFF7F0FEF1
:10042000002EE9D0ECE706210420CAE704000020F2
:1004300014430300190700009F480300FA4E03000D
:100440000022F0B505000F00FF200F248BB008AB91
:10045000654EDA710100C431890069188B781A0978
:10046000B25C234012011343CA788B7013071B0F31
:10047000F35CA243234013431A09B25C23401201E8
:100480001343CB700138E5D2E223DB00EE5CB30806
:10049000F31ADBB20493554B1B68002B0BD0E222FE
:1004A000C4218120D200890000013B00AA186918EC
:1004B0002818FDF7EDF900244823029403930194D2
:1004C000009481222B1912019B181B7818000593A8
:1004D0000723984320D008A92300059A0731280054
:1004E000FFF744FF0230C4B2023FFFB2002F78D0C2
:1004F0002B780393013EF6B2002E47D1E2222B194E
:10050000D2009B181E78B308F31ADBB204930023C1
:10051000029301930093D4E7354B009A9C469A5C72
:100520002300C4339B00EB18997809090A43314929
:100530008A5C019907926246DB78525C1907090FC1
:100540000A432C491B098A5C2B490692029A8A5C51
:1005500006991343079A8A182649C95C012389180A
:10056000FF2A00DC031CC918882309061B06C918CA
:10057000090F0020FFF744FE039B013BDBB203930E
:10058000002BB7D10134E4B2013FAEE7049B013B3D
:10059000DBB20493002B02D1059B002B18D1220063
:1005A000C4329200535D00999B069B0ECB18DBB2C0
:1005B0000093535B0199DB045B0ECB18DBB2019314
:1005C0005359029A1B035B0ED318DBB2029378E7F0
:1005D00008A92300059A07312800FFF7C7FE040089
:1005E0008CE70BB0F0BDC04623440300582A00201E
:1005F000EF4D0300FB4503009F470300064B1B5CC8
:10060000002B05D0054B185C4843C011C0B27047A1
:10061000034B185CFBE7C0464B470300C44503008F
:1006200084440300064B1B5C002B05D0054B185C73
:100630004843C011C0B27047034B185CFBE7C0468B
:100640004B470300FF4E0300D4440300F0B5037A88
:100650008DB004007F2B00D157E103000700002577
:100660000933FF330837099301953E787F2E00D078
:1006700087E000230693019306998B00E318039308
:100680001A7A481C1B7BC0B206907F2B00D11BE15D
:100690009F49CE5C8D5C9F49AE4200D0F1E08D5CFD
:1006A000CB5C0493039B597A019B5918CBB20193FD
:1006B000049BEB18DBB20793023B1B06DCD4A82794
:1006C000019B5D1BEBB20593A82F00D0E1E0039BDB
:1006D000039A5B7A527B5B08520899180291019940
:1006E00001988A18E221C31AD2B2DBB2C900A2185B
:1006F000E31852185B18157818782D1AEDB27F227E
:100700002B006DB293430893EB17E81858400299F9
:1007100009F07EFC2800CBB20299099309F092FB04
:10072000059A00251600C3B20A93029B9B18DBB200
:100730000B93320039002000FFF77EFD0A9B013643
:100740000B9AC018F6B2C3B2964200D1B6E0099A2D
:10075000AD18029AEDB2AA420DD8AD1A20216A4610
:1007600052181278EDB252B2002A00DAA4E0002B3F
:1007700001D00133DBB2320039002000FFF79AFDCF
:10078000D7E7012E77D12B003100019A200015F018
:1007900092F8BA78604BA1789B185B78300001938F
:1007A000FB780893FFF72AFF3F23E17803403000EE
:1007B0000293FFF737FF7F22584B9B5D1A40584B3F
:1007C00003929A5D0F231A400492564A925D1A4092
:1007D0000592554A925D1A4006923F22534B9B5D0B
:1007E00007937B78EB18DBB20A93029B13400293CA
:1007F0007F23184083019C462A003F21C432920087
:10080000135D0F268B4302990B431355135B484925
:100810000B4061460B431353039B10595903454B3F
:1008200003400B430498190C314000011351084355
:10083000A21890701B0E0598B34306990343090153
:100840001E400E43D67081226319079912019A182F
:100850001170E222D2009B180899019A01355218B2
:100860001A700A9BEDB29D42C6D1099B0437BB4268
:1008700000D0FAE6FDE6022E8BD12B00019AFF2173
:1008800084E72D48AE4201D9C55C09E78D5C835CE5
:1008900007E7049B019A39009A18D2B22000FFF7AB
:1008A000CBFC059A050039002000FFF7C5FC079B2B
:1008B0002D1AEDB2029322E7013B5BE70137FFB24D
:1008C000AF2F00D000E7D7E6023189006118019B05
:1008D000497859186368C9B2002B13D1E2238122E9
:1008E0001648DB001201E318A518001B1A18C432C1
:1008F0009200125D1E789206D20EB21A1A7001335F
:100900009D42F3D12000FFF79BFD0DB0F0BDC04626
:1009100034440300FB460300EF4E0300244503006C
:100920003343030083430300D34303009F4D03007D
:100930003FE0FFFFFF1FF0FF74450300F0F8FFFFEB
:10094000014BD8607047C0467C2E0020034B82B01C
:10095000D86801ABC01A02B07047C0467C2E002098
:10096000014B18617047C0467C2E002010B54E2107
:10097000024812F050FCFBF7B1FEC046A0AB0200EB
:1009800007B5054A01ABD1681269CB1A9A4201D862
:10099000FFF7ECFF07BDC0467C2E0020074B5B69CC
:1009A000002B01D1180006E05A68824204D8801A50
:1009B00004308000C05870471B68F1E77C2E00208F
:1009C00070B5144D04006B699868DB68834215D3D9
:1009D0000230C00015F07AFC6B69002803D19868DA
:1009E0004000FCF7DDFC5A68D96803609B68521828
:1009F0005B00836000234260C36068616A69D368FA
:100A00005068591C04339B000138D16040189C5039
:100A100070BDC0467C2E0020074B4118884204D38D
:100A2000D8B2002800D1013070475A01D31802789B
:100A300001305340F2E7C04605150000034B044A5D
:100A40005A6100229C331A607047C0467C2E0020F9
:100A5000E4C30200F0B585B001900E00FFF7DCFFA3
:100A6000144B02905C69002C01D120001EE027008D
:100A700010373D00E3689B00FB180393039B9D42E6
:100A800001D32468EFE72868029A037893420FD1D4
:100A90004378B3420CD102303200019918F06AF960
:100AA000002805D1ED1B6068AD10281805B0F0BD19
:100AB0000435E3E77C2E0020F0B585B0039001916A
:100AC000FFF7C8FF002861D1314D019B2F009C37F3
:100AD000DC1C3B68002B18D02E002E4AA036126872
:100AE00031680292A2188A420FD9020061181800D8
:100AF00015F00AFC0290002822D1264B020019684A
:100B0000386815F001FC029B3B602B009C331B688E
:100B1000002B20D12600802C00D2802630002F0010
:100B200015F0D4FB9C37386000280DD1200015F05B
:100B3000CDFB26003860002806D12000FCF730FCF1
:100B400033681B193360E0E72B00A0331E602B00D5
:100B50000022A4331A602B00A4331A689C352D6838
:100B6000A41801990398AD181C60FFF755FF019B6D
:100B700028701A006B70A81C039918F00AF900225B
:100B8000019B2800EB189A70FFF71AFF05B0F0BD23
:100B90007C2E0020202F0020F7B51D00160000231A
:100BA000070003600B6033602B60174B00915C699A
:100BB000002C02D0154B9C4204D133682A68D3180C
:100BC0002B60F7BD3B6801333B60E268009B9446B5
:100BD0001B68009A0193634413602200E36810329B
:100BE0009B00D3189A4207D32000FDF7E1FA2B6847
:100BF000246818182860DBE702CA30684978033097
:100C000009183160EEE7C0467C2E0020E4C30200E4
:100C10000C4B70B55C69002C02D00B4B9C4200D190
:100C200070BD2600E36810369D007519AE4201D3F1
:100C30002468F0E704CE05490232054816F0EAF8C8
:100C4000F4E7C0467C2E0020E4C302003C4F0300C2
:100C500084E80200044B054A98331B6804481A6074
:100C6000044A9A807047C0467C2E00207800040019
:100C7000E4B3020004040000084A10B513009833DE
:100C80001B689979002908D0916C0029F9D00021BE
:100C900099711B695879FCF7F7FE10BD7C2E002076
:100CA00013B5084C98342368188814F009FD23689C
:100CB0000090588814F004FD694601900220F5F771
:100CC000D9FC16BD7C2E002010B50D4C002803D099
:100CD0000868F6F7ABFB04000A492000F8F7F0F8C3
:100CE00060790021FCF7D0FE2000F8F7D3F800224D
:100CF000054B064898331B681A619A7110BDC046AF
:100D0000ACA2020010B202007C2E0020E4B302006C
:100D10001FB50C4B02AC00930194022301F0FCFAC6
:100D2000029A002A03D0084B98331B685A806268E5
:100D3000002A03D0044B98331B681A80034804B080
:100D400010BDC046D4D002007C2E0020E4B30200C7
:100D5000F0B5254B89B004AC00930194042301F055
:100D6000DBFA224F224A3B0098331B6804989A8092
:100D7000204B0340062B06D0830730D102681E4B60
:100D800092699A422BD1012303940293002598374C
:100D90003B681869F8F77EF83B6860681D61F6F7F4
:100DA00045FB16490600F8F78BF83B68144A9D711D
:100DB000126802999A60227B9981DA71DD81039A27
:100DC000012900D112685A6101221E619A71237AA9
:100DD000002B01D0FFF750FF0A4809B0F0BD03AA6D
:100DE00002A9F1F7EDFED1E794D002007C2E00209D
:100DF00004040000070080FF9D1D000010B20200E7
:100E0000D02F0020E4B30200F0B5274B89B004AD29
:100E100001950093042301F07FFA6B68A868049E93
:100E20000393F6F703FB214F040098373B681869DA
:100E3000F8F730F800223B681D491A612000F8F7E6
:100E40003FF8607980212D7BFCF71EFE002E1CD11F
:100E50006079FCF799FE039B002B13DB0022134BF8
:100E6000144998331B6803989A710968DA7141181C
:100E7000DA605A61023299601C619A71002D01D0CA
:100E8000FFF7FAFE0C4809B0F0BD31000B4808F03E
:100E90004FFFFCF7D5FD0028DDD06079FCF774FE2C
:100EA0000748FCF793FAC046B4D002007C2E00201D
:100EB00010B20200D02F0020E4B3020040420F0025
:100EC000EB6A030010B5182015F0F3F9064B9833C0
:100ED0001860064B0360064B838000238371036117
:100EE0004361044810BDC0467C2E002078000400F9
:100EF00004040000E4B30200F0B56D4C87B0260096
:100F000098363368002B40D09A79002A3DD0694D3D
:100F100099682A68914238D89A79022A0BD11B69BC
:100F200000215879FCF7B0FD2B6832680A339360D2
:100F30000123937129E09A79012A26D19A89D989C6
:100F4000914204D3DD79002D19D00021D98158694F
:100F5000012A02D0DA8992001058574A904216D1DD
:100F60001B69002158799834FCF78EFD246853489A
:100F7000218808F067FF0123A060A37105E09D713F
:100F80001869F7F787FF33681D6107B0F0BD05A941
:100F9000F0F736FC9834236801901B69802158795A
:100FA0000293059EFCF770FD019B24681F781F23A8
:100FB000218842481F4008F045FF618808F042FF41
:100FC0007D1EEDB20390012E5AD9019B5B78232B35
:100FD0004DD0622B50D1002D4BD0023FFDB26A1E86
:100FE00053425A415242022E4ED00121022301980F
:100FF000C05C3A2803D00F27384020710133207994
:1010000084469E420ED90198C05C3A280AD1581CE9
:10101000864207D9019F0233385C0F2738409E4231
:1010200035D86071092D3DD86346043B9A1852B2F9
:101030006F00234B002900D1224BD85B002A2EDB06
:101040001041FCF7FDFC1A4B039998331A68537949
:1010500059430B0017490A3B09680A2B00DA0A2397
:101060005B189360D3890133D381022361E70022A7
:10107000B9E72A000625B6E7002101230A00B6E7F2
:10108000002101230A00BAE733000121B7E70A264D
:101090007043019E6071F65C3E408019C1E7524288
:1010A0009040CEE7029B00215879FCF7EDFCCAE79F
:1010B0007C2E0020D02F0020E4B3020060EA000064
:1010C00014F7020006F70200F7B5CC1CA4000700D5
:1010D00020000E00019215F0ECF822000500054BEF
:1010E0004760866003600C3A01990C3017F051FE9E
:1010F0002800FEBD2CD102000021F0B5070087B00A
:10110000816414F0DFFCFB693C6ABB637B6AFC63AF
:10111000002B05DA3A00062140321170013306E057
:10112000002B07D03A00052140321170013B7B6251
:1011300007B0F0BD002833D0BB6A002B30D1390096
:10114000043340310B703A6BAE4B786BD3185B00B5
:101150001B5A013C9C42EBD017D9F96A8A4207D34B
:101160000831490015F0C3F8FB6A78630833FB6265
:101170003B6B5A1C3A637A6B5B009C527B6ACDE7EF
:10118000013B3B637B6A013B7B623B6B9D4A9A1848
:101190005200125A9442F3D3CAD002230B70C7E70D
:1011A0003C69631C03D1002240373A70C0E7380025
:1011B00014F030FC0490002800D129E13B004033BA
:1011C00005930023059A13703B69752B5AD0622B47
:1011D00007D17B69722B5CD001240B230022019282
:1011E00008E0722B51D17B69622B52D0049B012401
:1011F00001930A23390040310A78002A4ED10B703E
:10120000002C07D0380014F02DFC022C02D138003D
:1012100014F028FC3B690293222B01D02723029370
:10122000380014F01FFC0123029A03933B69934298
:101230000BD113007A69934207D1380014F012FCE5
:10124000380014F00FFC0323039300263C69631C51
:1012500000D1CEE0039B012B02D10A2C00D1C8E0C3
:10126000039B9E421DD338003100443015F0EFFF40
:101270000121380014F026FC380014F0CBFB0028C4
:10128000A2D155E701240A23A8E700240A230194E8
:10129000B0E7049B022401930B23ABE79A42AFD043
:1012A00046E7029BA34209D13800190044300136B9
:1012B00004F0B2FD380014F0D5FBC7E75C2C00D079
:1012C00091E0380014F0CEFB019B3D69002B06D065
:1012D00038005C21443004F09FFD2C0071E0622D49
:1012E00051D030D84E2D77D01AD8222D29D0272D85
:1012F00027D000260A2DDDD02C00303C0326072CF9
:10130000E6D87B69303B072B5BD8013E002E58D0D6
:10131000380014F0A7FB3B69E400303B1C19F0E7F0
:101320005C2D0ED00724612D21D0552DE4D13B003A
:1013300040331B780B2B2ED138005C21443004F055
:101340006BFD2C0013E0742D1FD007D86E2D1ED01E
:10135000722D0BD0662DCFD10C2408E0762D18D03D
:10136000E5D30226782DC7D1002428E00D243B00C8
:1013700040331B780A2B32D138002100443004F06E
:101380004BFD002696E70824F1E70924EFE70A243D
:10139000EDE70B24EBE70826752DE5D1043EE3E7E6
:1013A000380014F05FFB3D692800F7F76DF900285D
:1013B00000D144E1280011F0BBFF24012418013EB4
:1013C000EED20026631C00D174E70F4B9C42CED9AD
:1013D0000122059B1A70D4E70C48FCF7E9F9FF2CB1
:1013E000F6D80B2BF4D13800E1B2443015F0EBFE07
:1013F000C7E7039B9E4200D335E73B0003224033FF
:101400001A7030E7FFFFFF7FFFFF10003A6B030009
:101410002000F7F721F9041E386903D15F2801D0B5
:101420007F2842D93D0007233C0040352B704434CF
:10143000C1B2200015F0C7FE380014F013FB386964
:10144000431C1BD1200015F0ACFE002406007E4F8B
:10145000A300F958300017F002FD00281ED10D340A
:10146000E4B22C70102C00D062E6784BA8331A68D6
:101470000D23002A00D102332B7059E6F7F7ECF860
:10148000002808D138695F2805D07F2803D8F7F7EE
:10149000EFF80028D6D03B69D9B2CAE7002800DAB5
:1014A00046E60134222CD3D142E6F7F7E1F80028D2
:1014B0000FD03E00396940362E2916D109233370EA
:1014C0003D004435280004F0A7FC380014F0CAFAA7
:1014D00031E03B692E2B04D17869F7F7C9F8002871
:1014E000E7D100255A4C02234AE008233370302903
:1014F000E6D17A6918331343623B0024162BDFD8F8
:10150000544CDC4001231C40DAE7002C17D10300C7
:1015100020229343452B12D13C3B33706521280098
:1015200004F07AFC380014F09DFA396902220B00AD
:101530002B3B9343C6D03869431CE6D1F8E5F7F757
:101540008BF8002805D039692E290BD10923337077
:10155000B8E73869F7F78CF80028F4D13B692E2BEF
:10156000F1D0E5E50B00202293434A2BAAD1EDE709
:10157000633E9E43F6B272425641A41901350134CE
:101580002678002E02D03A69B242F1D1380014F028
:1015900069FA002E02D14037012206E6212E08D139
:1015A0003B693D2BF7D1380014F05CFA40374122FB
:1015B000FBE52E2E12D13C003B6940342E2B02D18C
:1015C0007B692E2B02D04A232370B1E5380014F03A
:1015D00049FA380014F046FA0C23F5E72A000134E2
:1015E000267802213300633B8B43DBB2002B0ED104
:1015F000637839690135994207D1380014F032FA1D
:101600002A00652E03D00234EAE7632EFBD1124B89
:101610009B5C3A0040321370190004229143422926
:1016200001D0442B03D1BB6A0133BB6280E543295F
:1016300002D0452B00D07BE5BB6A013BF5E70122D8
:10164000059B04001A7092E668D102007C2E0020EF
:10165000F96A030001204000B66B0300F7B5456846
:101660001600A8681F00019111F0CEFA0400A868C6
:1016700011F0D0FA11F0C8FA0300032058430734E0
:101680000019800014F015FE074B040003606B681E
:101690003200436000238560C36001993B0008303D
:1016A000F3F780F92000FEBD34D2020070B50500CA
:1016B00088680C0015F07CFC230002000249280019
:1016C00015F0A8FB70BDC046006C030010B50248C1
:1016D00011F09BFDFBF702F8DCAB020010B5040033
:1016E000082014F0E6FD024B4460036010BDC046C4
:1016F00070D20200F7B5C56804001E00002D02D1AB
:101700001D602800FEBD03691830834205D1184BC7
:10171000994203D01748FCF71DF819602000164FB6
:1017200011007B680830019363687B6001F0A6FDBF
:10173000019B05007B60012807D002280CD0002304
:10174000E36023691B683360DBE723691B68336050
:10175000002BD6D1E360D4E7A368986811F054FA5F
:10176000002305308000E36024186368EBE7C0467F
:10177000E4B302001E6C03007C2E002013B501AB05
:10178000FFF7B8FF01280ED0104C02280DD0019BA6
:10179000A34219D0002B17D001AA01210C4811F047
:1017A0002EFDFAF79BFF019816BD0198F1F77EF820
:1017B0000749FAF791FA002801D10198F1E7019859
:1017C000F6F73CFEA042F8D10020EDE7E4B30200BA
:1017D000DCAB020010B50B00022808D14A680549AD
:1017E0001868FFF7CBFF002803D1FFF76FFF8A6867
:1017F000F5E710BDE4B3020010B500220149FFF780
:10180000BDFF10BDE4B3020013B5114C01AB114A8A
:101810002100FFF76FFF012803D0022805D0200028
:1018200016BD0D490D4813F005F90198F1F73EF882
:101830000B49FAF751FA0028F1D10198F1F736F87F
:101840000849FAF749FA0028E9D10198FAF746FF62
:10185000E4B3020048A70200E06B0300A0AB020063
:10186000D0A80200DCAB0200F0B585B00500160080
:10187000080003AB02AA01A911F011FC0398364F2E
:10188000B84209D0032807D0F1F7F8F8B060002873
:1018900004D13248FBF79AFD0123B3600198B842A6
:1018A00029D10024B368A34200DC6C1E0298B84220
:1018B00025D1B368002B47DD2800002C2ADA6419F3
:1018C00001D5B368DC17002834DA401901D50120AE
:1018D0004042B368002B00DA0130B368002B2DDDE5
:1018E000A04200DA2000013B706058425841C0B26B
:1018F000346005B0F0BDF1F7C1F80400D6E7F1F7A8
:10190000BDF8B368002801DBDA0F8018002CD6DBA5
:10191000002B03DDAC42D6D92C00D4E7002BD2D06B
:10192000A54200D86C1E002804DA4019D4D5012045
:101930004042D1E7A842D0D92800CEE7002BD2D030
:10194000A042D0DD601CCEE7002C01DA0020B6E713
:1019500000208342E4D1C0E7E4B30200546C0300EA
:10196000F0B5060085B017001B2805D10A9A9742EA
:1019700009D0002005B0F0BD19281AD01C281AD0B3
:101980000A9A0A9717001A000B0011000A9A01928E
:10199000BA4200D901971D000C0000230093009B60
:1019A000019A934209D10A9BBB4220D0E1D3012086
:1019B000E0E71A26EAE71D26E8E70295039401CD41
:1019C00002CCF1F709F8002802D0009B0133E5E7CB
:1019D0001B2ECED0039B30001A68029B1968FBF7C0
:1019E000FDFC044BC01A43425841C0B2C2E71A2E54
:1019F000DDD1BEE7CCE70200F0B51E0085B0039054
:101A000018680D001700F0F751FF736801900293FA
:101A10000024022F0ED90123B2682900F1F706F93C
:101A20000400032F06D029000123F2680198F1F782
:101A3000FDF80500A54202D80848FBF7C7FC039A49
:101A4000A3000299D058F0F7C7FF002801D1013454
:101A5000F0E701206400204305B0F0BD6E6C030088
:101A6000002313B5044A046A09050093890C8A58B7
:101A7000A16B14F0BCF913BDACD20200F0B587B075
:101A800000931B7804000F0002922A2B05D1826874
:101A9000525C002A01D0A62A14D11A00213A022A47
:101AA0002DD8A568E8190378032B5CD104A96668D2
:101AB00014F067FAAB19984206D1676004992000C8
:101AC00014F0C3F907B0F0BD0378032B4BD105A97F
:101AD00014F057FA009B1B78212B04D1049B059A24
:101AE00013430493E6E7222B03D1049B059A53404A
:101AF000F7E7232BDED1059B049A1340F1E71A0088
:101B0000243A022A00D986E0A368D8190193037801
:101B1000032B28D1636804A9039314F032FA06005A
:101B2000019B039A9B189E42C7D0B378B01C75786E
:101B3000032B18D105A914F024FA0600372D35D14E
:101B4000059A1F2A0FDC4249049B114199420ADB86
:101B5000C021090611418B4205DB93400493049A8E
:101B600053005340DCD500226368029DDB1B0193C8
:101B7000561CED0969D1019B0135DB09FCD102320C
:101B800052193900200015F033FB0400009B029A23
:101B90001B7831001A330370013014F0AAF8701C5E
:101BA0002018019A290014F0A4F88BE7392D08D1E8
:101BB000059B1F2B01DD1F230593049B059A1341F1
:101BC000CCE72F2D03D1049B059A9B18C6E7302D37
:101BD00003D1049B059A9B1AC0E7312D09D10599C1
:101BE0000498F6F711F90028BDD1059B049A5343D8
:101BF000B4E7332DB7D00599352D06D10029B2D0E1
